:1000000000800020BD01000005CE0000BDCD000035
:10001000BDCD0000BDCD0000BDCD0000BDCD0000B8
:10002000BDCD0000BDCD0000BDCD000005CE00005F
:1000300005CE0000BDCD000085C4000089C50000CC
:1000400005CE000005CE000005CE000005CE000064
:1000500005CE000005CE000005CE000005CE000054
:1000600005CE000005CE000005CE000005CE000044
:1000700005CE000005CE000005CE000005CE000034
:1000800005CE000005CE000005CE000005CE000024
:1000900005CE000005CE000005CE000005CE000014
:1000A000C1A90000CDA9000005CE000005CE0000CA
:1000B00005CE000005CE000005CE000005CE0000F4
:1000C00005CE000005CE000005CE000005CE0000E4
:1000D00005CE000005CE000005CE000005CE0000D4
:1000E00005CE000005CE000005CE000005CE0000C4
:1000F00005CE000071EE000005CE00009DEF00006F
:1001000005CE0000DDD7000005CE000005CE0000C2
:1001100005CE000005CE000005CE000005CE000093
:1001200005CE000005CE000005CE000005CE000083
:1001300005CE000005CE000005CE000005CE000073
:1001400005CE000005CE000005CE000005CE000063
:1001500075C6000089C600009DC60000B1C600003B
:1001600005CE0000F9DA000005CE000005CE000043
:1001700005CE000005CE000005CE000005CE000033
:1001800005CE000005CE000005CE000005CE000023
:1001900005CE000005CE000005CE000005CE000013
:1001A00005CE000005CE000005CE000005CE000003
:1001B00005CE000005CE000005CE0000564B4CF2E7
:1001C000205210B51A804DF628121A8000BF00BFC9
:1001D0000CF01CFE514B4FF010621A60504A9A60AE
:1001E000504ADA60504A136813F4807304D14F49BF
:1001F0000B604FF4A85313604D4B1A78110703D5C9
:100200001A7842F008021A704A4B4B492A221A7097
:100210004A4A4B4B8B4204D252F8040F43F8040B6A
:10022000F8E7484B484900228B4202D243F8042B9E
:10023000FAE74649464A002352F8230041F82300D2
:1002400001336F2BF8D1434B434A802103F8011B44
:100250009342FBD1414B3D4A1A60414B8A221A70AE
:10026000A3F5805324225A70A0221A709A7992071B
:10027000FCD59A79D406FCD43A4A937903F00C035E
:10028000082B384BF9D103221A7140225A719A79FE
:100290009006FCD5334A9179324B4906FBD5324A58
:1002A000324911600221516020221A709A7902F0BD
:1002B0000C020C2AFAD12E4B2E4A1A602E4B2F4AD2
:1002C0001A6000225A60072243F8042C2C4AC3F813
:1002D0000C2D62B60DF04AF9144B1B68DA0705D5F0
:1002E00028480CF017FF284B284A1A60284B1B7827
:1002F0005B0609D5244C254B22689A4204D121483B
:100300000CF008FF0023236010F002F90CF084FDCC
:100310000CF0B2FCFEE700BF0E2005403080044028
:10032000823F04000100002B10D0034014D0034092
:1003300002D0074000E00740C49BFF1F4C3D010076
:100340004088FF1FC49BFF1FD0A3FF1F0082FF1F19
:100350000000000000E400E05FE400E008ED00E0E1
:100360000050064000400640448004400000030165
:1003700004800440C010050014E000E0FF76010096
:1003800000002020D58A195F1CE00340A5C3945AC1
:1003900000F00740FFFFFFFFFFFFFFFFFFFFFFFF32
:1003A000FFFFFFFFFFFFFFFFFFFFFFFFFFFFFFFF5D
:1003B000FFFFFFFFFFFFFFFFFFFFFFFFFFFFFFFF4D
:1003C000FFFFFFFFFFFFFFFFFFFFFFFFFFFFFFFF3D
:1003D000FFFFFFFFFFFFFFFFFFFFFFFFFFFFFFFF2D
:1003E000FFFFFFFFFFFFFFFFFFFFFFFFFFFFFFFF1D
:1003F000FFFFFFFFFFFFFFFFFFFFFFFFFFFFFFFF0D
:10040000FFFFFFFFFFFFFFFFFFFFFFFFDEF9FFFF23
:1004100010B5054C237833B9044B13B10448AFF33E
:1004200000800123237010BDC49BFF1F000000004B
:10043000503D0100084B10B51BB108490848AFF307
:1004400000800848036803B910BD074B002BFBD0A0
:10045000BDE81040184700BF00000000C89BFF1F08
:10046000503D0100C49BFF1F0000000038B504464A
:10047000104621700A491D460FF02CFE01464FF030
:100480007E500FF0DBFE07490FF024FEE560606050
:10049000256165610CF0FAFFE061204638BD00BFC0
:1004A000DB0FC9400024744938B50446104621705A
:1004B00009491D460FF00EFE01464FF07E500FF029
:1004C000BDFE06490FF006FEE560606025616561CE
:1004D0000CF0DCFFE06138BDDB0FC940002474493B
:1004E00038B503780446032B20D8DFE803F01A1848
:1004F0001002C16840690FF0E3FC0D4905466068D1
:100500000FF09CFE014628460FF098FE38BD0849C2
:1005100040680FF093FEE1680FF0DCFD38BDC06865
:1005200038BDC16840690FF0CBFC38BD002038BD34
:100530000024744970B504460E460CF0A7FF05462A
:10054000E069281A0FF072FDE3682361E5616661D6
:10055000A061014660680FF071FE0146A06010487E
:100560000FF06CFE0FF042F90EF0E2FD0FF054FCBC
:10057000054601464FF07E500FF0A2FC61690FF076
:10058000A9FD2169064628460FF0A4FD0146304624
:100590000FF098FCE0602046BDE87040FFF7A0BF78
:1005A000000080BF38B50E201C4C0CF03FFA2188AB
:1005B0001B4B884205461A881DDA0023511AB1F5F3
:1005C000805FAABF1B03C3EB03330131142093FBED
:1005D000F1F10CF0B1FD134B1988F1B923889D425C
:1005E00010DAC3F57F630F33282091FBF3F1BDE8E8
:1005F00038400CF0A1BD9042D4BFC1EB0003C1EB69
:100600000203DBE740F6FF718D42D4BFC3EB050167
:10061000C3EB0101C1EB0131E3E738BDB09CFF1F23
:100620006A9EFF1F1C9EFF1F10B504460CF000F8C9
:10063000204610BD70B44C88A04220D9012301335C
:10064000DBB21CB2660031F8144084421D46F6D37A
:10065000A04211D005F10045013D965B31F815101F
:1006600032F81530401AF21A00FB02F0641A90FBBF
:10067000F4F4E01870BC7047905B70BC70470226C1
:100680000125E5E700280CDA064A434282FB0320F5
:10069000DA17C2EB600000EB4000A3EB8000C0F172
:1006A0000C007047ABAAAA2AF0B40E8886420DD27D
:1006B00003F10043013B31F81350854202D9F0BCED
:1006C000FFF7B8BF32F81300F0BC70471088F0BCD9
:1006D000704700BF094B1B880C2B09D8084A80B211
:1006E00052F8232028B143F6FE73984203D9108CA8
:1006F0007047108870470349FFF79CBF169CFF1F87
:1007000020180100BC190100374A38491088384ABE
:10071000F8B5384B12881B68834248DB9342A8BF68
:10072000134698420B60C8BF002342DD101AB0F593
:10073000804FAABF9B03C3EB8333013093FBF0F0E0
:10074000FFF7C8FF2C4B2D4F1C883B68C0F3C61524
:1007500005FB04F47F2CA8BF7F249D42064608D0E9
:10076000274B1B88002B38D1264B1B88002B30D100
:100770003D60254D2B689E4205D0214B1B885A1F9A
:10078000032A1DD92E60214D2B689C420ED0204B90
:10079000188848B11A4B1F4A1B88D35C834203D088
:1007A000C0B2E1B208F0C6FA2C60F8BDF8BD03464D
:1007B00008609A42D4BFC0EB0203C0EB0303B5E765
:1007C000144AD05C2030C0B206F07F0108F0B2FAC3
:1007D000D8E7284608F022FBCAE70E4A2946D05C33
:1007E00008F0A8FAC0E700BFB09CFF1FE89BFF1FFE
:1007F0006A9EFF1F189EFF1FFC9BFF1F589CFF1F38
:10080000049EFF1FA29CFF1F109CFF1FA49CFF1FA4
:10081000129EFF1F088AFF1F2DE9F04F012089B0AB
:100820000DF048F8AF4B186000200DF043F8AE4BC8
:10083000AE4A1B8810600C2B00F03B81AC4BAD4ADC
:1008400019880093AC4B52F8214000221A70AB4B30
:10085000AB4D1B88AB4A2E88013B32F91370002E3A
:100860005CD0A94BA94A1B88A9491278013B31F9F0
:100870001380002A40F0DF8011200DF01BF8A54BFB
:100880000193D3F800A00646B24540F3DF80A24BA7
:10089000DFF8A4921B88A14A012BD9F80030B2F8E6
:1008A00000B09F4A02922046C8EB030800F09A82EB
:1008B0000FF0BCFB029A52F82B100FF00BFC014614
:1008C00000200FF0FDFA0FF0CBFDCAEB0802B04597
:1008D000B8BFB0469042CAEB080880F2968200FB8F
:1008E0000888013298FBF2F08E4BDFF850820293B9
:1008F000D8F80030034403EBD3735B10C8F8003022
:100900002B88012B12D1884BDFF834B20393874B2D
:10091000DBF8005004934FF0000A47E07D4B019351
:10092000DFF814927F4BDFF8148202937E4B03931F
:100930001D460F200CF0BEFF2B689842824641DA1C
:10094000754A1288012A00F01D82744A05931288A4
:10095000734D049220460FF069FB049ADFF8E0B172
:1009600055F82210DBF800500FF0B4FB01460020D0
:100970000FF0A6FA0FF074FDEF1B059B5745A7EB90
:100980000302B8BF5746FF1A9042BABF013200FBBC
:100990000777474397FBF2F7D8F80020634B04939F
:1009A000BB1803EBD3735B10C8F80030604B1B8897
:1009B000013B032B00F2B082DFE813F06301A901D1
:1009C000C4008601594B04931B68984240F3C281CE
:1009D000514A1288012A00F0A682504A07931188D2
:1009E0004F4A0691204605920FF020FB059A069982
:1009F000DFF84CB152F82110DBF800500FF06AFB21
:100A00000FF02EFD079B2F445745A7EB0302A8BF0D
:100A10005746FF1AD8F800309042BABF00FB07775C
:100A20000132474397FBF2F73B4403EBD3735B1070
:100A3000C8F80030BAE715200BF0F8FF354B0193EA
:100A4000D3F800A00646B2453FF721AF354B0293DD
:100A5000D3F800A0B24580F289812F4BDFF8D890FF
:100A60001B882E4A012BD9F80030B2F800B02C4A6E
:100A700003922046984400F070820FF0D7FA039A50
:100A800052F82B100FF026FB0FF0EAFCB045CAEB32
:100A90000802A8BFB046CAEB08089042B6BF00FBE8
:100AA000088800FB08F8013298FBF2F0DFF88C8030
:100AB0001EE7204B1B78002B3FF4C0AE0C4B0D4AB9
:100AC000198800930C4B52F8210001221A700FF084
:100AD000ADFA4FF07C510FF0FDFA0FF0C1FC044667
:100AE000B5E600BF489CFF1F469EFF1F889EFF1F64
:100AF0004E9CFF1F8889FF1FF29BFF1F148AFF1F58
:100B0000BC9DFF1F041D0100648AFF1FD09DFF1FB5
:100B100074190100409CFF1F8E9CFF1F349CFF1F17
:100B20001C1D01007C9CFF1F389EFF1FB09DFF1FF6
:100B30005E89FF1F069CFF1FE09BFF1F4C9EFF1F4F
:100B4000349EFF1F28460FF071FAB2490FF0C2FA27
:100B5000054650460FF06AFAAF490FF0BBFA01465E
:100B600028460FF0AFF90FF07BFC0546CBF800509C
:100B7000D9F800000FF05AFAA6490FF0ABFA074671
:100B800030460FF053FAA4490FF0A4FA0146384654
:100B90000FF098F90FF064FCC9F800009F4AA04BD1
:100BA000168819889F4AA04B12681B889F4FC6EB76
:100BB000050E3544039EC6F800E0461A0844049921
:100BC0000D6001990E6002993E8808609A4280F299
:100BD00089810025C3EB060E954974450F6880F2A4
:100BE0007681611C9F4205FB01F50EF1010E95FB1C
:100BF000FEF5C0F2BE81BE42A8BF3E46F61A01FB1A
:100C000006F494FBFEF49A4200F33681BB42C0F234
:100C10003381884C20680FF009FA87490FF05AFA9F
:100C200086490FF04FF90FF01BFCA0F5FF531C3B5A
:100C3000082B98BF4FF40050D8F800301844002813
:100C40002060C0F24281B0F5804F80F252817C4B2F
:100C50001B781BB1B0F5005F40F05381794D2B78C4
:100C6000002B40F05481784D20682B68714C9842DD
:100C700004D080B208F03CF923682B6009B0BDE8CD
:100C8000F08F28460FF0D2F970490FF023FA05468D
:100C900050460FF0CBF96E490FF01CFA014628467A
:100CA0000FF010F90FF0DCFB0546CBF80050D9F837
:100CB00000000FF0BBF965490FF00CFA074630460B
:100CC0000FF0B4F962495FE728460FF0AFF95A49CF
:100CD0000FF000FA054650460FF0A8F95D490FF0F5
:100CE000F9F9014628460FF0EDF80FF0B9FB05467B
:100CF000CBF80050D9F800000FF098F94E490FF0EA
:100D0000E9F9074630460FF091F952493CE7284689
:100D10000FF08CF950490FF0DDF9054650460FF001
:100D200085F94E490FF0D6F9014628460FF0CAF86A
:100D30000FF096FB0546CBF80050D9F800000FF0F5
:100D400075F945490FF0C6F9074630460FF06EF9C0
:100D5000424919E7D8F80030DFF810B103EBD3733C
:100D60005B10DBF80050C8F800301FE6DFF80081A8
:100D7000DFF80091D8F8003003EBD3735B10C8F8AC
:100D80000030BDE5364A06931188364A0591204663
:100D90000492DFF8D8B00FF049F9049A0599DBF80E
:100DA000005052F821100FF095F90FF059FBEF1B8E
:100DB000069B5745A7EB0302B8BF5746FF1AD8F862
:100DC00000309042BABF013200FB0777474397FBE0
:100DD000F2F73B4403EBD373234A04925B10C8F849
:100DE0000030E3E50FF022F9029A52F82B100FF0D1
:100DF00071F90FF035FBCAEB0802B045B8BFB04639
:100E00008242CAEB08083FF76AAD00FB08F898FB7E
:100E1000F2F069E5CDCC4C3FCDCC4C3E168AFF1F9D
:100E20005C89FF1F489CFF1F149EFF1F2C9CFF1F07
:100E3000889EFF1FBC89FF1F9A99193FCDCC4C4556
:100E40003A9FFF1FA09CFF1F2089FF1F3333733F72
:100E5000CDCC4C3DCDCCCC3E6666663FCDCCCC3DBA
:100E6000349CFF1F1C1D0100B09DFF1F349EFF1FFF
:100E70004C9EFF1FE09BFF1F009B1B88002B3FF435
:100E8000C8AE2B1B002BB8BF5B42092B47DD05F515
:100E900000500130001B0FF0C9F83B493B4C0FF0EC
:100EA00019F9054620680FF0C1F839490FF012F919
:100EB000014628460FF006F80FF0D2FAD8F80030B5
:100EC000184400282060BFF6BEAE002213E09F4207
:100ED00005FB04F5B8BF002195FBFEF54BDA91FB4D
:100EE000FEF490E6B242D4BFC3EB0205C3EB0605A5
:100EF00070E643F6FF72274B22601B78002B3FF40D
:100F0000ADAE05F0DBF9244B01221A70ABE605F01B
:100F1000D1F900232B70A6E6D9F800003EE64FF485
:100F200000501A4C88E61D491D4A069320460D883C
:100F300005920FF07BF8059ADFF868B052F825109B
:100F4000DBF800500FF0C6F8014600200EF0B8FFA5
:100F50000FF086FA2F44069B56E50FF067F8039AC8
:100F600052F82B100FF0B6F8014600200EF0A8FF43
:100F70008AE51E4642E6B742D4BFC3EB0701C3EB86
:100F8000060104FB01F1AAE7CDCCCC3EBC89FF1FD2
:100F90009A99193F3A9FFF1FA09CFF1F349CFF1F87
:100FA0001C1D0100349EFF1F08B5244B1B88FBB19C
:100FB000234B1B78FBB1234B1B78E3B1224B1B78EF
:100FC000CBB1224B1B78B3B1214B22481A78C2B95E
:100FD000214A22490088128809680244B1EB620F55
:100FE00009DD01221A706420BDE8084005F07AB9D5
:100FF000174A117801B908BD1370BDE8084007F021
:1010000041BF154A16490088128809680244B1EBAD
:10101000620FF0DD00221A7007F034FF642005F043
:1010200061F9642005F05EF9642005F05BF94FF486
:101030001670BDE808400CF04BBA00BFBE9DFF1F04
:10104000669EFF1F679EFF1F689EFF1F699EFF1F12
:10105000149CFF1F2C9CFF1F149EFF1F489CFF1F0A
:10106000889EFF1F38B5114C232025780BF0DEFC3D
:101070000F4A42F82500131F02F1C400002253F862
:10108000041F83420A44FAD123780A4907480A4CCC
:101090000133DBB2322B81FB025108BF0023D21790
:1010A000C2EB21120370226038BD00BFFE9BFF1F00
:1010B000C09CFF1F1F85EB51309EFF1F2DE9F04F95
:1010C000B84CB94D2068B94F83B00EF0AFFFB849A6
:1010D0000FF000F8064610200CF0ECFB0EF0A6FF17
:1010E000B4490EF0F7FF31460EF0ECFE0FF0B8F900
:1010F0002988206088423B8843DA9E465B1A7F2B12
:101100004FF0000247DDD2015E1C92FBF6F2AA4EC0
:10111000DFF8C882B6F800C0C8F80020BCF1190F8B
:1011200000F0DF80BCF11A0F00F01781BCF11E0F38
:1011300000F020810126B146A04A1288002A00F062
:101140009D808842C0F207817045D4BFC1EB00008A
:10115000C1EB0E009A42BABF02FB000001335043BC
:1011600090FBF3F3964A1360964B1888C0B9964AE1
:101170001288AAB9954B197801B11A7003B0BDE86D
:10118000F08F9842D4BFC1EB0002C1EB03029E4630
:101190005B1A7F2BB7DCC2EBC21292FBF3F2B6E70D
:1011A0002988D4F800E0DFF80082DFF8F8A1714563
:1011B0006CDCDFF818C29CF80020002A2ED14FF01A
:1011C000010B04288CF800B028D1002E40F0948147
:1011D0007D4B18880028D1D0B9F1000FCED02368FC
:1011E0002C883A88A34280F265810023141B7E2C50
:1011F000774DD5BFC3EB8313C3EBC3135B0001343F
:1012000093FBF4F42B680134A34203D0C0B2E1B2E3
:1012100007F090FD2C6003B0BDE8F08F012800F0CE
:10122000F680022800F0EB800328D1D1694B1B889F
:10123000092BCDD0002ECBD023682E883A88B3421C
:1012400080F27B810023961B7E2EDFF88CA1D5BF18
:10125000C3EB8313C3EBC3135B00013693FBF6F6BA
:10126000DAF800300136B34203D0F1B24A2007F079
:1012700061FDCAF80060ABE716469146BCF11E0F4F
:101280007FF472AF0022DFF858817EE04F4B1A786E
:10129000002A3FF473AF002401281C7000F0A480E2
:1012A000022840F00E81002E00F0A3804A4D2B68EA
:1012B000002B00F09E800420214607F03BFD424BAE
:1012C0002C60188800283FF459AFB9F1000F3FF4A3
:1012D00055AFC0B2002107F02DFD3D4B00221A6032
:1012E0004CE7DFF8FC8098F80020C2B1DFF8D89016
:1012F000B9F800A0BAF1000F11D0DFF8E89099F822
:1013000000B0934578D05FFA8AF07F2107F012FD94
:1013100098F80030B6F800C089F8003010E0DFF827
:10132000C49099F800A0924566D0274B0021187808
:1013300007F000FD98F80030B6F800C089F80030DA
:101340001E4B1A88002A97D0BCF11E0F40F0068170
:101350000026B14619E00020FCE6DFF8848098F80A
:101360000020002A0BBF012600264FF000094FF095
:101370000109E1E6DFF86880104B98F800601A88F0
:10138000B6FA86F676094FF0000998F80030002B7F
:101390003FF4E8AE2988B7F800E02068C1EB0E03FF
:1013A000CFE600BF3C9CFF1FC49DFF1FC09DFF1FD9
:1013B0009A99193FCDCCCC3E469EFF1F709EFF1FD1
:1013C000B89CFF1F469CFF1F529EFF1F4B9EFF1F96
:1013D000209CFF1F049EFF1FBC9CFF1F2C9EFF1F15
:1013E000069CFF1F029CFF1F1EB1614D2B68002B46
:1013F0007BD1604B188865E70026B1469CE6002E3D
:101400003FF4E6AEDFF868A1DAF800202EE0002E07
:101410003FF4DEAEB7F80080F045D4BFC1EB080260
:10142000C1EB0E02C1EB0808B8F17E0FDFF840A156
:10143000D5BFC2EB8212C2EBC212520008F1010802
:1014400092FBF8F8DAF8002008F10108424506D0CE
:101450005FFA88F10120009307F06CFC009B18886C
:10146000CAF8008002287FF4DFAE42462168B5F852
:1014700000803888414559DA0021C8EB0008B8F1EE
:101480007E0FD3BFC1EB8111C1EBC11108F101087F
:10149000490091FBF8F808F10108904506D05FFA81
:1014A00088F10420009307F045FC009B1888CAF8D7
:1014B0000080B9E69342D4BFC4EB0303C4EB02033C
:1014C00094E6032827D12C4B1B88092B91D0002EA2
:1014D0008FD0274D2B68002B8BD04A20214607F058
:1014E00029FC244B2C601888ECE6214607F022FCEE
:1014F000204B2C601888E5E640207F218DE80C0009
:1015000007F018FC019B009A188858451CD0022847
:101510007FF48AAE76E704287FF46BAF002E3FF4A9
:1015200068AF2146402007F005FC62E78142D4BF46
:10153000C8EB0101C8EB00019FE79342D4BFC6EBA3
:101540000303C6EB02037EE6B8F80010DAF800E009
:10155000B7F800808E45FFF665AF5DE72988B7F8DC
:1015600000E020680026C1EB0E03B146E9E500BFAC
:10157000BC9CFF1F529EFF1F049EFF1F08B50F4B10
:101580001B88022B0FD0032B12D0042B03D00C4B43
:1015900001221A7008BD7F21092007F0CBFB084B00
:1015A00001221A7008BD7F21412007F0C3FBEEE73E
:1015B0004021092007F0BEFBE9E700BFB49CFF1FF4
:1015C0006A9CFF1F38B51C4B1B881D2B26D01B4B5C
:1015D0001B88012B25D01A4A1A4B14881B681A4AFB
:1015E000A342128818DB9342D4BFC4EB0303C4EBBD
:1015F0000203141B7F2CC6BFDB010134C3EBC313F2
:1016000093FBF4F4114D2B689C4203D0E1B205200A
:1016100007F090FB2C6038BD0023EAE70C4B1C88D8
:10162000F0E70C4B0C4A0D491B6812680C689B1ABA
:101630001C1B84F30704E5E7469EFF1FBC9DFF1FAC
:10164000669CFF1FF49BFF1F449EFF1FEC9BFF1F28
:10165000389CFF1F789EFF1F2889FF1FC89DFF1F12
:1016600010B50F4C23685BB90E4B1B88022B11D0B1
:10167000033B012B09D90C4A00231370236010BDD2
:101680000021052007F056FBEEE70021092007F0B6
:1016900051FBF0E70021412007F04CFBEBE700BFD6
:1016A000EC9BFF1FB49CFF1F6A9CFF1F08B5274BD4
:1016B0001B78ABB115200BF0B9F9254A254B1288E0
:1016C00018601D2A15D0244A1288EAB1012A25D0B3
:1016D000224B1B78002B34D0BDE80840FFF7C0BF79
:1016E00011200CF0E7F81A4A1A4B128818601D2ACC
:1016F000E9D11B4B1B78002BEAD0184B1B780BB39E
:10170000BDE80840FFF75EBF164A1288002ADFD006
:10171000154A1B6812889A42DADCEEE70F200CF0BB
:10172000C9F8104B114A1B88106033B1104B114A95
:101730001B6812689B1A9842DFDD084B1B78002B50
:10174000CAD108BDFFF71AFFDAE700BFD09DFF1F1F
:10175000469EFF1FF49BFF1FBC9DFF1F6A9CFF1F3F
:10176000069CFF1FB49CFF1F669CFF1FC89DFF1FA8
:10177000789EFF1F2889FF1FF8B510200CF09AF8FB
:10178000C830B0F5FA7F6EDBB0F57A6F0146A8BFBE
:101790004FF47A6101F51673B3F57A6FA8BF4FF471
:1017A0007A639BB289B27B4A7B4C118022202380D2
:1017B00007F044FC2188794D794C242007F03EFC49
:1017C0000E200BF033F940F6FF71C8308842A8BFF5
:1017D000084620EAE07000F5FA6283B28A42A8BFA8
:1017E0000A460220194622802B8007F027FC218818
:1017F000042007F023FC01200CF05CF804460020D4
:101800000CF058F8A042B8BF204600F1C801B1F56D
:10181000FA7FC0F2A480B1F57A6FA8BF4FF47A6165
:1018200001F54873B3F57A6FA8BF4FF47A639BB2A2
:1018300089B25C4A5C4C11800A20238007F0FEFBD1
:1018400021880C2007F0FAFB15200BF0EFF800F5CB
:101850009671B1F52F7F0BDB41F25C23994240F387
:101860008380194608E040F24C434FF4FA719AE73E
:1018700040F214534FF42F714C4A11804C4C4D4D93
:101880002380062007F0DAFB21884B4E082007F062
:10189000D5FB00274FF4AF74F9B2484809F004F9BA
:1018A00055F8043BC3F5967300FB03F086FB002359
:1018B000C017C0EB6310844207F10107A8BF0446BC
:1018C000062FE9D13E4F3C4E0025E9B23D4809F0D4
:1018D000EBF857F8043BC3F5967300FB03F086FB67
:1018E0000023C017C0EB6310844205F10105A8BFB7
:1018F00004460C2DE9D1344F2F4E0025E9B2334870
:1019000009F0D2F857F8043B2B4AC3F5967300FB55
:1019100003F086FB0013C017C0EB6310844205F18F
:101920000105A8BF04460C2DE8D1A4F1140131290A
:101930002BDD40F23A73A4F5B97403FB04F482FB87
:101940000432E417A4EB621289B232322048214BF0
:1019500001801A602A20BDE8F84007F06FBB40F212
:1019600014534FF4FA7164E7104A00F5617089B2BC
:10197000B0F52F7F1180B8BF4FF42F73FFF67EAF05
:101980008342A8BF03469BB278E740F26C723221D3
:10199000DCE700BFC49DFF1FC09DFF1FB09CFF1F61
:1019A0006A9EFF1F149EFF1F2C9CFF1F669CFF1F3B
:1019B000449EFF1F4C8AFF1FB5814E1B189CFF1FC2
:1019C0001C8AFF1F4C9CFF1F2C89FF1FA89CFF1F18
:1019D000649EFF1F048AFF1F2DE9F84F0C200AF0B8
:1019E000F1FF0C200BF0A6FCBF4914200BF0B2FC59
:1019F000BE49BF4808F0EAFC022103200BF040FD7D
:101A0000022104200BF03CFD022105200BF038FDE3
:101A1000022106200BF034FD01210A200BF030FDDD
:101A2000012109200BF02CFD01210D200BF028FDD8
:101A3000012128200BF024FD012114200BF020FDB2
:101A4000012116200BF01CFD172001210BF018FDC1
:101A500004200BF007FD00283DD005200BF002FD0F
:101A6000044600283ED000242046A24D287005F0F0
:101A700009FF2E785EBB204607F00AFB9E4B9F496C
:101A80001B880F889E4ADFF8DCE29E4DA3F5AF71FC
:101A900040F23A7303FB01F382FB0312DB17A3EB63
:101AA0006213323301210D20CEF800302F700BF07D
:101AB000D3FC64200BF00CFD4FF416710A200BF0E0
:101AC0003BFB5D21904809F02BF890B9FEE7BDE89B
:101AD000F84F08F08BBB06200BF0C4FC0028BCD1EB
:101AE0000124C2E703200BF0BDFCB0FA80F04009EE
:101AF000BBE764200BF0ECFC31460A200BF01CFB2A
:101B00004FF4967109200BF017FB5C217F4809F018
:101B100007F800B9FEE764200BF0DAFC3146092033
:101B20000BF00AFB4FF4967116200BF005FB5B21BE
:101B3000774808F0F5FF00B9FEE764200BF0C8FC19
:101B4000314616200BF0F8FA4FF4967117200BF07F
:101B5000F3FA64200BF0BCFC314617200BF0ECFAD2
:101B600064200BF0B5FC31460D200BF075FC694A82
:101B700069481268DFF8F0B1DFF8A4A1674FDFF819
:101B8000EC91DFF8EC8100230121FEF78DFC0123AD
:101B9000CAF800603E60C9F800608BF80030042687
:101BA0000F200BF087FED9F8003003440E20C9F84F
:101BB00000300AF03BFFDAF800309BF800200344C5
:101BC000CAF800301520002A7DD00AF02FFF3B68AC
:101BD0001844386006F0010080F0010004F072FB48
:101BE000B8F80030002B14BF4B20DC200BF070FC49
:101BF000013ED5D1D9F80030DAF8002048493868DC
:101C0000DFF870E1474E002BB8BF0333002AB8BF9E
:101C1000033292100A604449444A09881288002815
:101C2000B8BF03309B10801038605F1A19443160D0
:101C3000CEF800703E4E3F4F3F49C9F80030C2EB2E
:101C4000000E0244C7F800E032600B600CB1FFF7F1
:101C500093FDB8F800305BB94FF4FA7004F042FB22
:101C600004F02CFB06F00AF94FF4AF600BF030FCE7
:101C7000324B012404201C600BF0F4FB10B9304BF4
:101C800028701C702F4B1B881C2B23D02E4C04F16A
:101C9000C80523200AF0CAFE44F8040F01200BF007
:101CA00017FCA542F5D1294A294B1078187007F086
:101CB000F9F804F0FFFA45F6BF5226492648BDE878
:101CC000F84F0AF06BBC11200BF0F4FD3B68184490
:101CD00038607FE7214B18880028D7D0204BC0B24E
:101CE000197807F027F8D1E7001B374640420F006C
:101CF000D090FF1F1C9CFF1F649EFF1FDC9DFF1FD9
:101D0000B5814E1B789CFF1F189CFF1FA89CFF1FCE
:101D10004C9CFF1F2489FF1FE09DFF1FE09BFF1FBE
:101D2000F89BFF1FB09DFF1F168AFF1F5C89FF1FD6
:101D30007C9CFF1F409CFF1F789EFF1F409EFF1F43
:101D4000079CFF1F469EFF1FBC9CFF1FCC9DFF1FD3
:101D5000AB9DFF1FA50500005C9EFF1F809CFF1F21
:101D6000389CFF1F048AFF1FD09DFF1F349EFF1F5A
:101D70000E9EFF1F389EFF1F2DE9F04FAC4C2678BA
:101D8000012E95B000F04582C0F0FB81022E00F0DC
:101D9000CB80A849A84A91F800801178A74ADFF8BB
:101DA0002CE3A74DA74FA848A84B0292A84A00923F
:101DB000A84A9EF800B001922D78A74A3F7890F883
:101DC00000E01B78DFF80CA3DFF80CC3DFF80C93FE
:101DD0000392012E84BF00222270A04AA0481370F3
:101DE000A04A80F800B015709F48A04A077082F89A
:101DF00000809F489F4A03709CBF01362670117077
:101E0000BEF1000F40F009819B4A10880D2800F0B8
:101E1000A9819A4C00202070024604462DB19648B4
:101E20000088002840F0AA81054695480688254488
:101E3000002E40F057819348934C019E00783678ED
:101E400024780130A0EB4600002C40F04682039C31
:101E500094F800E0CEEB0004BEF1000F40F0668283
:101E60000026DFF864E202989EF800E00078A41BE8
:101E7000A4EB4E043C44CBEB040410B1B7FA87F05A
:101E800040099CF800602718BC1B1EB11EF100061B
:101E900018BF0126009F99F8000097F800909AF863
:101EA00000C07A4FC6EB040EC0EB0E00A0EB490059
:101EB0008044C3EB0803A3EB41010C2313FB0C117B
:101EC0003960734B734C744E1B8874482488376890
:101ED0000088734E033B03EB4303C4EBC40401EBE4
:101EE00083033C4403440C3B56F824001D44054442
:101EF0000AB16C4B19606C4B1A68954200F02E8148
:101F00006A4A6B4811680791079901601268089244
:101F10006848089A00881D60521A824284BF664A47
:101F2000156015B0BDE8F08FDFF8B481634E08AFDF
:101F30000025E9B2624808F0B7FD58F8043BC3F544
:101F4000967300FB03F086FB00230135C017C0EB3E
:101F500063100C2D47F8040BEBD15A4B3D4D019506
:101F60003D4DB3F800C00395109D09980F99464E5A
:101F7000DFF8D4A0DFF8C890DFF8D080654511AA5B
:101F80008CCAAE46ACBF4FF0000E4FF0010E844538
:101F9000D4BF0020012030708C452E480B9D254E6B
:101FA0008AF800E0D4BF00210121017094452A493C
:101FB000DFF820A1D4BF002201220A709C45424ACA
:101FC000D4BF00230123BC45AB46D4BF0027012763
:101FD0001370AC451B4B0C9D1F70D4BF4FF0000B12
:101FE0004FF0010B394B154A0292AC45DFF848C05F
:101FF000174A83F800B0D4BF0025012589F80050A6
:1020000098F800309CF8001096F80080DFF8C8C0FF
:102010002678DFF8C8900092DBE62D4A174814882E
:102020000122182C027040F260810024F6E600BF05
:10203000AA9DFF1F009EFF1F029EFF1F909CFF1F77
:10204000909EFF1F689CFF1F959EFF1F019EFF1F14
:10205000499EFF1F559EFF1F569EFF1F8F9EFF1F0D
:10206000C39DFF1F919EFF1F929EFF1F939EFF1F08
:10207000949EFF1F4A9EFF1F969EFF1F069CFF1FF8
:10208000F09BFF1F188AFF1F809EFF1F089EFF1FE7
:10209000209EFF1F3C9EFF1FB89CFF1F009CFF1F40
:1020A000341B01007C9EFF1F609CFF1F7C9FFF1F55
:1020B000509CFF1F509EFF1F849EFF1FB5814E1B2B
:1020C000A89CFF1F649EFF1F579EFF1F699CFF1F58
:1020D000469EFF1FB59DFF1F8E9EFF1F489EFF1F40
:1020E0002C89FF1F012E00F08F81022E00F0EE815F
:1020F000032EA74B00F01F811E78009B9CF800E088
:102100001C78019B99F800C01878029B93F8008016
:10211000039B1F78A6EB4E03A4EB8404CCEB030CCB
:10212000C0EB80760CEB0403C0EB8600034403EBAA
:10213000480303EB810327B196490978002940F051
:10214000608201269AF800109348C1F1060101EB64
:102150004101334403EB81010160B2E68F49904AAB
:102160000968D3E6002D3FF454AE8E4A8E4E148893
:102170000122182C327040F2B8807446A0F10D058F
:1021800053E6DFF87092894F0DF120080025E9B27F
:10219000874808F089FC59F8043BC3F5967300FBA7
:1021A00003F087FB00230135C017C0EB6310062D39
:1021B00048F8040BEBD17F4BDFF83CA219880D9B4C
:1021C00000228B428AF8002080F2A2807A4B8AF8A3
:1021D00000507A497A4A7B4891F8008011787A4A0F
:1021E0001D7002920378794ADFF810C2DFF810926E
:1021F0000092774A774E784D784892F800E0784A16
:102200000192784A96F800B02D78077826780392E4
:10221000DFE5DFF8F081654E08AF0025E9B27248CE
:1022200008F042FC58F8043BC3F5967300FB03F03A
:1022300086FB00230135C017C0EB63100C2D47F857
:10224000040BEBD15B4B0C9D1F885F4B02935F4BE4
:1022500000930B9B0A98099ADFF8A0C1089EDFF84B
:10226000A0910F99BB429E46ACBF4FF0000E4FF0BD
:10227000010EAF42D4BF002501258742109B8CF888
:102280000050D4BF00200120504D89F80000974233
:10229000D4BF00220122B742D4BF4FF000084FF054
:1022A00001082A709F42474A4448474E80F8008000
:1022B000D4BF002301231370129A414886F800E02E
:1022C0008F42D4BF00210121974201701ADC002205
:1022D0004648DFF824A102708BE7039C46B12678BC
:1022E000002E40F06081441EBBE50C3C012295E5C8
:1022F00094F800E00138CEEB0004BEF1000F7FF44B
:10230000B0ADADE5119A9742D4BF00220122DFE7BC
:102310000C9A374B9142CCBF012200221A7040F335
:10232000458105258AF80050234B52E7002E3FF4E3
:1023300097AD012695E51C78009B029893F80080E4
:10234000019B9CF800601B7890F800C099F8007021
:102350000398A4EB4604E71B90F800E0C3EB8374FA
:10236000A8EB88003844C3EB8403034403EB4C031D
:1023700003EB8103BEF1000F40F0488101269AF87B
:102380000010054833440C2414FB0131016098E52A
:10239000188AFF1F579EFF1F089EFF1F509CFF1F9C
:1023A0007C9FFF1F469EFF1F069CFF1FB5814E1B93
:1023B000189CFF1F649EFF1FC29DFF1F009EFF1FF2
:1023C000029EFF1F019EFF1F909CFF1F499EFF1F43
:1023D000959EFF1F699CFF1F909EFF1F689CFF1F1B
:1023E000559EFF1F569EFF1F4C9CFF1F329CFF1FD8
:1023F000699EFF1F4C8AFF1FB59DFF1F8E9EFF1F0A
:10240000489EFF1F1C8AFF1FA34CDFF89CE2207828
:1024100005909EF8004001980494059C0078019076
:102420000134A4EB40040498002840F0AF800398E6
:1024300090F800E00498261ACEEB06000390BEF157
:10244000000F40F09E8074460298944E00780290EF
:10245000039836780496041BA4EB460402983C4487
:10246000CBEB0404002800F08780B7FA87F040091E
:102470009CF800602044871B1EB10498061C18BFFE
:102480000126009C99F800002478BE1B301AA0EBAE
:10249000440080440198C3EB0803A3EB41030028E8
:1024A00067D1BEF1000F40F0BB807344002C5ED1B9
:1024B00000290CBF00206FF009009AF80010784C3A
:1024C00003440C2010FB01312160FAE4039E019CBF
:1024D00036780396009E2478019434786F4E7148C4
:1024E00099F800E0009496F800906F4C9DF80C600D
:1024F00086709DF80460067080F806E09DF8006024
:1025000080F803909CF800C02478DFF8B491DDF8DF
:1025100004E080F80880077180F805C0C671417238
:1025200044704FF000080120009500215D4C0D46DD
:102530005FFA88FC4F46764607E0022809D00A2950
:102540000BD014F8016F17F8010F864201F1010159
:10255000F3D101350A29EDB2F3D1092D72D808F172
:102560000108B8F1100F36D019F80A0FDDE7002086
:10257000A3E74FF0000E98E7029879E7CEEB04004E
:1025800003900198041C18BF01245DE701980028FE
:102590004ED0039890F800E0BEF1000FEED1601E1F
:1025A0000390744650E7841B01265AE40B9A3F4B74
:1025B0009142CCBF012200221A703EDC0A9A3C4BA9
:1025C0009142CCBF012200221A7052DD03258AF805
:1025D0000050384BFDE5304837490478C86B029904
:1025E000009D097801342044CBEB00000844002111
:1025F0009AF800402A4B401A0C2111FB0401196083
:102600005FE41BF1000618BF01269BE5234909780A
:1026100000293FF4B3AE1BF1000618BF0126AEE659
:10262000049800280CBF4FF0000E4FF0090E3CE755
:10263000039890F800E03046FDE604258AF8005043
:102640001C4BC6E514481C49047851F8280002992F
:10265000009D097801342044CBEB00006646084415
:10266000002BC4D0002EC2D1BBF1000FBFD001217E
:10267000BEE7099A114B9142CCBF012200221A7089
:1026800004DD02258AF800500A4BA2E5089B994216
:1026900018DD01259AE500BF188AFF1F579EFF1F0E
:1026A000089EFF1F849CFF1F809EFF1F689EFF1FC8
:1026B000679EFF1FC29DFF1FC489FF1F669EFF1FED
:1026C000E0190100134B1D78012D21D9124A8AF817
:1026D00000501288002A3FF47CAD104A1288013A5B
:1026E00092B2062A3FF675AD0D4A1278002A3FF4E1
:1026F00070AD0C4A1268012A7FF46BAD0A4A0B4E8A
:1027000010680C2290FBF2F102FB1102328060E5AE
:1027100035465EE5C29DFF1F8C9EFF1FCE9DFF1FAD
:10272000B29CFF1F409EFF1F849EFF1F0C9EFF1F39
:102730002DE9F04F3A4B1B788BB0002B6AD10E205D
:102740000AF074F90DF072FC01463648364E374DEA
:10275000FDF7F0FE3348FDF7C3FE0DF081FE80F378
:102760000C003060FFF708FB2C68012C7AD0022C9B
:1027700000F09F82032C00F0AD832D4E33682D4A6C
:102780002D4E0993099B316812882C4C591A013A35
:102790009142236000F28882294E32689A1A0D2AEB
:1027A00000F27B82274E32689A1A132A00F2708256
:1027B000254E32689A1A252A1AD9244B1B88002BD9
:1027C00040F05F81224B1B78002B40F05A81FEF7CE
:1027D00049FC204B1B881B3B9BB2022B04D81E4B91
:1027E0001B78002B40F0508103F08EFD236833608E
:1027F0001A4D2A689B1A502B00F20682184B1B8830
:10280000012B00F01E8206F029FB06F057F90BB0F1
:10281000BDE8F08F07F072FB0BB0BDE8F08F00BF92
:102820001C9CFF1FE09DFF1F189EFF1F409EFF1F67
:102830007C9FFF1FC089FF1FAC9CFF1FD89DFF1FFF
:10284000989CFF1F709CFF1F749CFF1FBE9DFF1F65
:10285000149CFF1F469EFF1F069CFF1FB89DFF1F75
:102860001C9EFF1FDFF810939E4AB9F800001378F2
:10287000834204D0C3B21846137006F02BFADFF877
:10288000F482994AB8F800301178994204D0974FF1
:102890003978002940F0F186954A33681288954EC0
:1028A0009A42C0F2F680944A1278002A40F0F180F1
:1028B000DFF8C8A2BAF8003023B9904B1B88002B70
:1028C00000F0EF848E4A8F4B11881B888E4A0B4490
:1028D00012685B1093428D4A126880F29184002145
:1028E0009342B4BF01230B4604910093ACBF4FF059
:1028F000010B8B4605910E200AF098F8844B854A0F
:102900001B68176803930133A7F25232002B8446E9
:10291000029240F3C386802BA8BF80237E4A7F4962
:1029200012780191002A00F0BE800978914200F0EF
:10293000BA80B8F80010DFF83CE2994201F09B80C1
:102940006A49AEF80030764B4FF0010E81F800E096
:102950001978DFF82CE2019B8EF800101A70009BAA
:10296000002B00F00F81BAF80030002B00F00A8134
:102970006C4B1B685A1C002A40F39486802A00F393
:102980009086694C69496A4824880988006821440E
:10299000B0EB610FC1F2E282A3F148020F2A02D824
:1029A000473BA9F800300E200AF040F86FF454734A
:1029B0001F44874202DC5F4B00221A705E4B1B886B
:1029C000002B00F015845D4B5D4A1B78117899420D
:1029D00040D0002B3ED05B490C78002C00F01487CF
:1029E000594991F800C0BCF1000F40F00B87574FD8
:1029F0000097574F57480297544F007887F800C008
:102A0000534F4FF0010E87F800C081F800E0002816
:102A100041F0B18050490978002900F0D5874F492D
:102A200003910C460978002940F0CB874C48484F69
:102A30000078397001210297217058B1434842490A
:102A40000090002008700099029F087003990124EB
:102A50003C7008701370434B1B88A3F11B02012AC2
:102A600040F2E6851D2B7FF489AE3D4F3B78002B6D
:102A700041F048803C4C2378002B40F08684237042
:102A80007CE6FEF791FAA2E62B68012B7FF4ACAE50
:102A9000ACE63168354A0691069835491060022245
:102AA0000B602A6004E71E49DFF8D4E009780029AA
:102AB0003FF451AF9EF8000081423FF44CAF0398C1
:102AC0004B2840F39F871833802BB8F80000A8BF2D
:102AD000802398423FF43FAF2648038003480123F8
:102AE000037038E7AB9DFF1F789CFF1F079CFF1FFB
:102AF000B09CFF1F7C9FFF1F149CFF1F9E9CFF1F0D
:102B00002C9CFF1F149EFF1F489CFF1F889EFF1FC9
:102B10007C9EFF1FF89BFF1F729EFF1F5C9CFF1F88
:102B2000739EFF1F089EFF1FC49DFF1FC09DFF1FB8
:102B30003C9CFF1FB49DFF1FCE9DFF1F329CFF1FBB
:102B4000E49BFF1F929EFF1F109EFF1F549EFF1FBE
:102B5000B29CFF1F939EFF1F8F9EFF1FE59BFF1FD1
:102B6000069CFF1F469EFF1F029CFF1F6C9CFF1FC1
:102B7000D49DFF1FDC9DFF1FCC9DFF1F649CFF1F8A
:102B80005D9CFF1F029B9C45BFF60DAF864B1B88CB
:102B9000002B3FF408AFBBF1000F7FF4E9AE834B8D
:102BA0001B881BB1059B002B7FF4E2AE049B002B1E
:102BB0003FF4F9AE7E4B1A78002A7FF4F4AEDFF8CA
:102BC000649299F8004001221A70002C40F036837C
:102BD000784B1B78002B02F03780774B1B78002B4B
:102BE00002F00283754B1B78002B7FF4DCAE744B34
:102BF0001B78002B3FF4D7AEB8F8003071490A3B80
:102C0000A8F800300A70CEE604F084FE6E4B1B7804
:102C100073B96E4B1B785BB96D4B1B7843B96D4B29
:102C20001B782BB96C4B1B7813B903F043FB01E005
:102C300003F04CFB23682B60684B1B88012B7FF44F
:102C4000E2AD674A674B116867481A78A1F118032B
:102C50002A2101FB03F10160002A00F0B382634CDA
:102C60002368994200F35C8310DA61480278002AF5
:102C700040F03E875F4A1068D0F17F0048BF0330C4
:102C8000801001301B1A994242F3428621609BE278
:102C9000FEF70CFD236833608AE5FDF7BDFDFEF706
:102CA0000DFA236833607DE5FDF72EFD2368336060
:102CB00072E5514A34681188A14204DB464B1B7807
:102CC000002B00F05D834D4E4D48336807934D4B0C
:102CD000079A00681B88121A9A4200F2A980002BFA
:102CE00000F0A680484B1A88002A3FF447AD474BB6
:102CF00047481B680088A342B8BF2346994241F366
:102D00002681444B1960DFF8208188F80020344F79
:102D1000FDF7FAFC38687F2840F370853E4B7F381A
:102D200083FB0032C317C3EB620303EB4303A0EB47
:102D300083007330394B01931B883860002B40F0BF
:102D40008C86234B00931B78002B00F0CD83344CF2
:102D50002378002B00F0C883DFF8D090DFF8B8A00C
:102D60004FF0000B0CE003F17300C0B298F80010B4
:102D700006F008F823780BF1010B5B4540F3B483B0
:102D80003B6859F8040F1844A0F17F038AFB032124
:102D9000DA17C2EB610202EB42027F28A3EB820347
:102DA000E1DCFDF76FFCE0E79E9CFF1FD29DFF1F5B
:102DB000B49DFF1F8F9EFF1FC39DFF1F919EFF1F8E
:102DC000929EFF1F079CFF1FB29CFF1F109EFF1FBC
:102DD000549EFF1FE59BFF1F149CFF1F1C9EFF1F9F
:102DE000849EFF1F6A9CFF1F6C9EFF1F0C9CFF1F91
:102DF000589EFF1FEC9BFF1FB09CFF1F7C9FFF1F77
:102E00006C9CFF1F9C9CFF1F049CFF1FD49DFF1FF9
:102E10006A9EFF1FE89BFF1FABAAAA2A449CFF1FC4
:102E20008489FF1FB59DFF1F919CFF1F5C89FF1FB9
:102E3000554B564A1B681088554AA342B8BF2346D3
:102E4000994200F38482534C12888342A8BF034600
:102E50002360002A7FF457AF9942C8BF134640F35E
:102E60007D82401AB0F5804FAABF9B03C3EB83332A
:102E7000013093FBF0F0FDF72DFCC0F3C6100DF010
:102E8000D5F8454B044618880DF0D0F8434907465D
:102E900020460DF01FF9014638460DF01BF921467A
:102EA0000DF010F84FF07E5104460DF0B1FA0028F5
:102EB00041F031803A4920460DF0C8FA002840F030
:102EC000548620460DF0F2FAC0B2DFF8F48088F89C
:102ED00000001CE7334B34681988A14274DD324B83
:102EE0001B78002B70D1DFF8DC9099F800007F2868
:102EF00040F3FA85A3F155337F3803F1004383FB98
:102F00000032C317C3EB620303EB4303A0EB830060
:102F10007330264B01931B88C0B289F80000002B48
:102F200040F0EB87224B00931B78002B00F0998434
:102F3000204C2378002B00F094841F4FDFF87C8016
:102F40004FF0000A0AE003F17300C0B205F042FF3F
:102F500023780AF1010A534540F3838457F8043F6C
:102F600099F800001844A0F17F0388FB0321DA17C9
:102F7000C2EB610202EB42027F28A3EB8203E2DC98
:102F8000FDF780FBE1E700BFD49DFF1F6A9EFF1F96
:102F9000049CFF1FE89BFF1F749EFF1FCDCCCC3D00
:102FA0000000FE42B09CFF1F149CFF1F449CFF1FAB
:102FB000549EFF1F8489FF1F5C89FF1FABAAAA2AAA
:102FC000919CFF1F069EFF1FB84F38687F2840F373
:102FD000CC81B74B7F3883FB0032C317C3EB62034E
:102FE00003EB4303A0EB83007330DFF8249399F8DD
:102FF00000A0824500F01F82AE4B1B88002B43D1FE
:10300000AD4AAE4812680088914205DC8242D4BFC6
:10301000C1EB0203C1EB0003411AB1F5804FA6BF1B
:103020009B030131C3EB833393FBF1F0FDF752FBBC
:10303000C0F3C6100CF0FAFFA14B044618880CF040
:10304000F5FFA049804620460DF044F80146404671
:103050000DF040F821460CF035FF4FF07E5104464C
:103060000DF0D6F9002840F0C286974920460DF0B1
:10307000EDF9002840F0768520460DF017FAC0B231
:10308000DFF8908288F80000BAF17F0F40F3B28336
:103090008748AAF17F0A80FB0A304FEAEA73C3EB44
:1030A000600000EB4000AAEB80007330874B009378
:1030B0001B78C0B289F80000002B40F01283844BCB
:1030C00003931B78002B40F0F584824B02931B780E
:1030D000002B40F03487804B0193029B1B78FBB19F
:1030E0007E4B1B88012B00F00086022B00F05987D5
:1030F000032B01F0EB80042B01F0EB82052B01F098
:103100000784062B01F06085072B01F0D185082B81
:1031100002F02A80092B02F02F810A2B02F0828212
:10312000009B1B78002B00F05F84019B6A4C198880
:10313000002900F0B58438687F2840F3CF825C4BCB
:103140007F3883FB0032C317C3EB620303EB4303F7
:10315000A0EB830073303860002940F06484009B4A
:103160001B78002B00F072815D4C2378002B00F05F
:103170006D81DFF8A4A1DFF89C814FF0000B0CE01B
:1031800003F17300C0B298F8001005F0FBFD23783E
:103190000BF1010B5B4540F359813B685AF8040F72
:1031A000434A1844A0F17F0382FB0321DA17C2EBE4
:1031B000610202EB42027F28A3EB8203E0DCFDF711
:1031C00061FADFE7474B1960474B1B68A92202FBF6
:1031D00003F3002BBCBF03F57F533F339B13543BDA
:1031E000194481F30C01282009F0A6FFFFF70BBB5F
:1031F000384C3E483549364A237003700B7029E439
:1032000093424FF0000B80F2B3800123CDF800B061
:10321000CDF814B00493FFF76EBB354B1B78002B31
:103220007FF4C1AB039B334A243B83F34703D9B2FA
:103230005B20136005F07EFD99F80040032C30D12F
:10324000DFF8D88098F80030002B42F022812A4F16
:103250003B78002B42F01081254C2378002B42F064
:10326000FE80264B1B78002B42F0EC80244A138012
:10327000244B1B78002B42F018810E4B7F221A80C2
:1032800098F800306BB93B785BB923784BB91E4A8C
:103290007F210720138005F04DFD7F210B2005F0D5
:1032A00049FD1A4B1F68FFF77EBB00BF849EFF1FBE
:1032B000ABAAAA2A049CFF1FE89BFF1F6A9EFF1F60
:1032C000749EFF1FCDCCCC3D0000FE42549EFF1FDC
:1032D000E59BFF1FB29CFF1F449CFF1FCE9DFF1F5D
:1032E0008489FF1F0C9CFF1FBC89FF1F109EFF1FBE
:1032F000929EFF1F289CFF1F919EFF1FC39DFF1FD3
:10330000A29CFF1F939EFF1F049EFF1FF89BFF1FA1
:10331000069EFF1F919CFF1F5C89FF1F8F9EFF1F52
:10332000B04A1078002840F04383AF4A1268D2F1C7
:103330007F0248BF033203EBA202531CAB4A236057
:103340009942B8BF1160FFF63FAF19463CE7A84B62
:1033500012881960002A7FF4D6AC0B469842D4BF7D
:10336000C1EB0003C1EB03037BE5FDF78BF93CE602
:103370000123CDF810B0CDF800B00593FFF7BBBA2C
:1033800001232B609B4EFFF7F9B99B4B6A201988EC
:1033900005F054FE3B782370FFF7F0B9029B1B78D1
:1033A000FBB1964B1B88012B00F01884022B00F018
:1033B0007686032B01F00080042B01F0AF81052BF2
:1033C00001F02A82062B01F01484072B01F0C0853E
:1033D000082B01F07D86092B01F0EF870A2B02F004
:1033E000B281019B1B88002B00F02683009B1B7879
:1033F0003BB9039B1B7823B9029B1B78002B00F081
:1034000054877F4B1B78002B00F035817D490B786A
:10341000082B00F230817C483A6800687B4C01330D
:10342000DBB25F1E101A44F827000B70784B34682B
:10343000198889F800208C426E4E7FF79FA9326868
:10344000744B0892089A1A60FFF798B9039B1B788F
:10345000002BA3D03B68A3F10C007F2840F3278307
:103460006D488B3B80FB0320DA17C2EB600000EB5A
:103470004000A3EB800303F17300DFF8AC81C0B21E
:1034800098F8001005F07EFC009B1B78002B85D07F
:103490005C4C2378002B81D0DFF890A14FF0000B1B
:1034A0000CE003F17300C0B298F8001005F06AFC5C
:1034B00023780BF1010B5B457FF770AF3B685AF83F
:1034C000040F554A1844A0F18B0382FB0321DA173D
:1034D000C2EB61020C3802EB42027F28A3EB8203AD
:1034E000DFDCFDF7CFF8DEE7454B1B78002B40F023
:1034F000A9823B68494A1278002A45D0A3F10C0002
:103500007F2840F3EE82444A8B3B82FB0321DA178B
:10351000C2EB610202EB4202A3EB820303F17300F0
:10352000C0B298F8001005F02DFC009B1B7853B337
:10353000344C23783BB3DFF8F490DFF8DCA04FF095
:10354000000B0BE003F17300C0B298F8001005F017
:1035500019FC23780BF1010B5B4514DD3B6859F82E
:10356000040F1844A0F18B038AFB0321DA17C2EB86
:1035700061020C3802EB42027F28A3EB8203E1DCFC
:10358000FDF780F8E0E73B68254A1278FAB11B4A5C
:103590001288012A00F02E84022A00F00186032AF4
:1035A00000F08387042A01F0E080052A01F01882E8
:1035B000062A01F02A83072A01F01984082A01F05B
:1035C0005786092A01F09B860A2A02F08880019A10
:1035D0001288002A00F04882124903220B702A60E8
:1035E000FFF7CCB8589EFF1FEC9BFF1F0C9CFF1FE2
:1035F000E89BFF1F7C9FFF1F389CFF1FCE9DFF1F76
:10360000109EFF1F8489FF1F089CFF1F6089FF1FFA
:10361000B09CFF1F249FFF1FABAAAA2AE59BFF1F98
:10362000B29CFF1F069EFF1F919CFF1F5C89FF1F1E
:10363000B04F3B78002B3FF41DAAAF4C207802F02E
:10364000CDFEAE4B1B78002B00F0748223887E2BBE
:1036500000F27082AA4A0133108899B221800028B2
:1036600000F07882C9B2C0B2A64C05F063FB3B788B
:103670002370FFF783B83A68D8E6DBB218461370B8
:1036800005F036FBA04BA1491A46A14B1846002372
:103690000B703B7013700370FFF7FEB80123FFF748
:1036A0003DB980249B499C4B9C4A09881B88126821
:1036B0000B44B2EB630FBFF676A98E4B1B78002B41
:1036C00040F0DF81B8F80030954AA3423FF46BA97F
:1036D000944B148001221A70FFF765B9FCF7D2FFF2
:1036E00039E5914B01931B88002B42F00B81884BED
:1036F00003938E4B02938E4C23786BB3DFF840829A
:10370000DFF830A24FF0000B09E003F17300C0B204
:1037100005F060FB23780BF1010B5B451CDD58F8CD
:10372000043F99F800001844A0F17F038AFB0321AD
:10373000DA17C2EB610202EB42027F28A3EB82039D
:10374000E3DCFCF79FFFE2E7784B029305F042FBD6
:10375000009B1B78002BCED1039B1B78002B3FF4E2
:10376000BCAC99F80030A3F10C007F2840F3B6817F
:1037700070488B3B80FB0320DA17C2EB600000EB44
:103780004000A3EB800303F17300C0B205F022FBFD
:10379000009B1B78002B00F09681654C2378002B52
:1037A00001F04B82DFF89881DFF888A14FF0000B21
:1037B0000AE003F17300C0B205F00CFB23780BF1B3
:1037C000010B5B457FF789AC58F8043F99F800007E
:1037D0001844A0F18B038AFB0321DA17C2EB6102C4
:1037E0000C3802EB42027F28A3EB8203E1DCFCF7FA
:1037F00049FFE0E75046FCF745FF57E4FCF742FF7E
:10380000FFF798BA002008704B49087840B13E494C
:1038100000910978002900F0AB81009F00213970E8
:103820004649097800297FF4FAA8002C40F0CC80A2
:10383000002840F0C9802F4C334F94F800E0344CFE
:1038400003943A4C0294324C30492070374C009724
:10385000087038702070BEF1000F7FF4F2A8FFF7F7
:10386000F9B82B4B1B78002B6CD099F80030A3F1E2
:103870000C007F2840F37B832E4A8B3B82FB032185
:10388000DA17C2EB610202EB4202A3EB820303F1FF
:103890007300C0B205F09EFA009B1B78002B51D03C
:1038A000234C2378002B4DD0254FDFF888804FF034
:1038B000000A09E003F17300C0B205F08BFA237827
:1038C0000AF1010A53453DDD57F8043F99F800001D
:1038D0001844A0F18B0388FB0321DA17C2EB6102C5
:1038E0000C3802EB42027F28A3EB8203E2DCFCF7F8
:1038F000C9FEE1E7069CFF1F389CFF1F949EFF1F37
:10390000809CFF1F029CFF1F549EFF1F109EFF1FE5
:10391000E59BFF1FC49DFF1FC09DFF1F3C9CFF1F19
:10392000DC9DFF1F079CFF1F449CFF1FB29CFF1FD5
:103930008489FF1FABAAAA2A939EFF1F8F9EFF1F99
:103940005C89FF1F924B1B78FBB1924B1B88012BAC
:1039500000F03886022B00F03287032B01F0AB8099
:10396000042B01F05D81052B01F09783062B01F0FC
:103970003084072B01F0BC85082B01F07B86092BD6
:1039800001F088870A2B01F06587019B1B88002BBB
:1039900000F0BC82804B1B78002B40F0B2827F4B42
:1039A0007F4A198834680020012310602B6042E5AB
:1039B0000130C0B2022886BF002111701070194674
:1039C00002E40398002101707649097800293FF448
:1039D00041A86F4902910978002900F016870298E2
:1039E00000210170FFF736B8039B1B78002B7FF492
:1039F0009CAB029B1B78002B7FF497AB019B198833
:103A0000FFF799BB243B002BB8F8000040F3478434
:103A100098423EF4A0AF9BB26348A8F8003001235F
:103A20000370FEF798BFDFF88481C0B298F80010E9
:103A300005F0A8F9FFF793BB5C4B3878197805F0CF
:103A4000A1F9D3E47F21402005F074F95849594A7F
:103A50003B680B60002111704CE5C0B298F8001073
:103A600005F090F9FFF76DB9D8B298F8001005F09D
:103A700089F93B68B0E5504BDFF85CE11978FEF757
:103A80006ABF4B2C40F34A821834802CB8F80030BF
:103A90004A4AA8BF8024A3427FF41AAEFEF783BF30
:103AA00099F8000005F096F92188FFF744BBFCF770
:103AB000E9FDE2E4424B01931B88002B7FF444AE06
:103AC000334B02934DE6029B1B78002B7FF408AB2F
:103AD000039B1B78002B7FF428AB8FE7FCF7D2FD0C
:103AE00053E6FCF7CFFD1BE5FCF7CCFDFFF711BA61
:103AF0000132D2B2022A40F23D82002202701946FF
:103B0000FFF762BB2F4C207802F068FC2E4B1B782D
:103B10001BB123887E2B41F23B802C4B1B7823B1B9
:103B20002388284A002B41F05880294C3B78237089
:103B3000FEF724BE254B1B78002BF6D02388214AA4
:103B4000002BF2D02349013B088899B2118000284C
:103B50007FF488ADC8B21E4C05F060F93B78237045
:103B6000FEF70CBE7F20FFF78BBA7F20FFF7ADB9C1
:103B7000074F094902974FF0000C81F800C0009FE1
:103B800002994FF0010E87F800E081F800C047E687
:103B9000B29CFF1FCE9DFF1F109EFF1FB09CFF1FFA
:103BA000E89BFF1F069CFF1F079CFF1F919CFF1FA8
:103BB000089CFF1F8489FF1F739EFF1FDC9DFF1F52
:103BC000449CFF1F389CFF1F949EFF1F939EFF1F66
:103BD000029CFF1F809CFF1F5D9CFF1FDFF8B0A3AE
:103BE0003868BAF80030E54AE54CC31A82FB031E78
:103BF000D917C1EB6E0101EB4101A3EB810303EB8C
:103C0000430354F8233018447F2840F3C9847F3895
:103C100082FB0032C317C3EB620303EB4303A0EB49
:103C200083007330DFF86C83DFF86CB398F8001012
:103C3000C0B205F0A7F8BBF80030022B7FF6D1AB7D
:103C40003968BAF80030CD4ACB1A82FB030ED81778
:103C5000C0EB6E0000EB4000A3EB800303EB4303DB
:103C600004EB8303586808447F2840F320877F389B
:103C700082FB0032C317C3EB620202EB4202A0EBED
:103C800082007330C0B298F8001005F07BF8BBF8E2
:103C90000030032B7FF6A5AB3968BAF80030B74A7D
:103CA000CB1A82FB030ED817C0EB6E0000EB40006E
:103CB000A3EB800303EB430304EB8304A0680844F5
:103CC0007F2840F36B817F3882FB0032C317C3EB40
:103CD000620202EB4202A0EB8200733098F80010FF
:103CE000C0B205F04FF8FFF77CBBDFF8A4A299F84B
:103CF0000000BAF80030A14AA14CC31A82FB031E8F
:103D0000D917C1EB6E0101EB4101A3EB810303EB7A
:103D1000430354F8233018447F2840F33D847F3810
:103D200082FB0032C317C3EB620303EB4303A0EB38
:103D300083007330DFF860B2C0B205F04BF8BBF817
:103D40000030022B7FF6ECA999F80010BAF8003089
:103D50008A4ACB1A82FB030ED817C0EB6E0000EB29
:103D60004000A3EB800303EB430304EB8303586899
:103D700008447F2840F397867F3882FB0032C317C0
:103D8000C3EB620202EB4202A0EB82007330C0B2CE
:103D900005F020F8BBF80030032B7FF6C1A999F895
:103DA0000010BAF80030754ACB1A82FB030ED81700
:103DB000C0EB6E0000EB4000A3EB800303EB43037A
:103DC00004EB8304A06808447F2840F3CA807F384E
:103DD00082FB0032C317C3EB620202EB4202A0EB8C
:103DE00082007330C0B204F0F5FFFFF799B90120EB
:103DF000FFF746B9DFF898A16049BAF80020604C97
:103E00009A1A81FB020ED017C0EB6E0000EB400047
:103E1000A2EB800202EB420254F8220018447F28F1
:103E200040F3C283A0F17F0381FB0321DA17C2EBC9
:103E3000610000EB4000A3EB80007330DFF858B165
:103E400098F80010C0B204F09DFFBBF80030022BC0
:103E500050D93968BAF80030484ACB1A82FB030EB1
:103E6000D817C0EB6E0000EB4000A3EB800303EB20
:103E7000430304EB8303586808447F2840F37E869D
:103E80007F3882FB0032C317C3EB620202EB4202AF
:103E9000A0EB82007330C0B298F8001004F072FFFB
:103EA000BBF80030032B25D93868BAF80030334A04
:103EB000C31A82FB031ED917C1EB6E0101EB41014E
:103EC000A3EB810303EB430304EB8304A3681844CF
:103ED0007F2849DD7F3882FB0032C317C3EB6202C3
:103EE00002EB4202A0EB82007330C0B298F80010DF
:103EF00004F048FF3B68FFF76ABB04F06BFFFFF775
:103F000011B80021402004F015FF48E599F80000A1
:103F100004F060FF3EE50120FEF7D7BF243C002CF3
:103F2000B8F8003040F35685A3423EF43CADA4B24D
:103F3000144BA8F8004001221A70FEF734BD124B52
:103F400001931B88002B7FF401ACFFF7C6B80F4923
:103F50008342A8BF03460B60FEF7D5BE1446FFF7A9
:103F6000ACBBFCF78FFB3DE7FCF78CFBBDE7FCF738
:103F700089FB8EE402701946FFF726B9ABAAAA2A7C
:103F8000E4180100079CFF1F449CFF1FE89BFF1FD4
:103F90000C9EFF1F919CFF1F1A9CFF1FFCF772FBDA
:103FA0009CE6DFF81CA399F80000BAF80030C24A7A
:103FB000C24CC31A82FB031ED917C1EB6E0101EB81
:103FC0004101A3EB810303EB430354F8233018446E
:103FD0007F2840F3C7837F3882FB0032C317C3EBCF
:103FE000620303EB4303A0EB83007330DFF8D4B22A
:103FF000C0B204F0EFFEBBF80030022B7FF690A8B1
:1040000099F80010BAF80030AB4ACB1A82FB030EC5
:10401000D817C0EB6E0000EB4000A3EB800303EB6E
:10402000430304EB8303586808447F2840F3018668
:104030007F3882FB0032C317C3EB620303EB4303F9
:10404000A0EB83007330C0B204F0C4FEBBF80030B4
:10405000032B7FF665A899F80010BAF80030964A4D
:10406000CB1A82FB030ED817C0EB6E0000EB4000AA
:10407000A3EB800303EB430304EB8304A068084431
:104080007F287FF76EAF7F3882FB0032C317C3EB08
:10409000620303EB4303A0EB83007330A2E6DFF877
:1040A00020A23868BAF80030834A844CC31A82FBD5
:1040B000031ED917C1EB6E0101EB4101A3EB810394
:1040C00003EB430354F8233018447F2840F37183F3
:1040D0007F3882FB0032C317C3EB620303EB430359
:1040E000A0EB83007330DFF8E081DFF8D8B198F8F7
:1040F0000010C0B204F046FEBBF80030022B7FF681
:1041000070A93968BAF800306B4ACB1A82FB030EEB
:10411000D817C0EB6E0000EB4000A3EB800303EB6D
:10412000430304EB8303586808447F2840F37485F5
:104130007F3882FB0032C317C3EB620303EB4303F8
:10414000A0EB83007330C0B298F8001004F01AFEA0
:10415000BBF80030032B7FF644A93868BAF800306A
:10416000554AC31A82FB031ED917C1EB6E0101EB3E
:104170004101A3EB810303EB430304EB8304A36836
:1041800018447F287FF70AAF7F3882FB0032C317BD
:10419000C3EB620303EB4303A0EB830073309DE5A5
:1041A000DFF81CA14449BAF80020444C9A1A81FB5C
:1041B000020ED017C0EB6E0000EB4000A2EB8002B5
:1041C00002EB420254F8220018447F2840F3F482A4
:1041D000A0F17F0381FB0321DA17C2EB610000EB42
:1041E0004000A3EB80007330DFF8D8B098F80010DF
:1041F000C0B204F0C7FDBBF80030022B7FF67AAEE8
:104200003968BAF800302C4ACB1A82FB030ED81753
:10421000C0EB6E0000EB4000A3EB800303EB430315
:1042200004EB8303586808447F2840F3EA847F380E
:1042300082FB0032C317C3EB620303EB4303A0EB23
:1042400083007330C0B298F8001004F09BFDBBF8F7
:104250000030032B7FF64EAE3868BAF80030164AAD
:10426000C31A82FB031ED917C1EB6E0101EB41019A
:10427000A3EB810303EB430304EB8304A36818441B
:104280007F287FF771AE7F3882FB0032C317C3EB04
:10429000620303EB4303A0EB8300733025E60128A0
:1042A0003EF459AB0123FFF7B7BB99F8000004F0C7
:1042B00091FDFFF7A6B800BFABAAAA2AC01B010058
:1042C0000C9EFF1F1A9CFF1F919CFF1FDFF8E8A2A6
:1042D00099F80000BAF80030B54AB64CC31A82FB10
:1042E000031ED917C1EB6E0101EB4101A3EB810362
:1042F00003EB430354F8233018447F2840F3DD8157
:104300007F3882FB0032C317C3EB620202EB42022A
:10431000A0EB82007330DFF8A4B2C0B204F05AFD03
:10432000BBF80030022B7EF6FBAE99F80000BAF81D
:1043300000309F4AC31A82FB0321DA17C2EB6102E5
:1043400002EB4202A3EB820303EB430304EB830380
:104350005B6818447F2840F327847F380C2290FB49
:10436000F2F302FB13007330C0B204F033FDBBF86C
:104370000030032B7EF6D4AE99F80000BAF8003076
:104380008B4AC31A82FB0321DA17C2EB610202EBEC
:104390004202A3EB820303EB430304EB8304A36811
:1043A00018447F287FF7DDAD7F380C2290FBF2F3B5
:1043B00002FB1300733015E5DFF8FCA13868BAF88A
:1043C00000307B4A7B4CC31A82FB031ED917C1EB1A
:1043D0006E0101EB4101A3EB810303EB430354F8AE
:1043E000233018447F2840F365817F3882FB0032F8
:1043F000C317C3EB620202EB4202A0EB82007330F0
:10440000DFF8BC81DFF8B4B198F80010C0B204F056
:10441000B9FCBBF80030022B7EF6E3AF3868BAF87F
:104420000030634AC31A82FB0321DA17C2EB610230
:1044300002EB4202A3EB820303EB430304EB83038F
:104440005B6818447F2840F3A0837F380C2290FBE0
:10445000F2F302FB13007330C0B298F8001004F0BE
:1044600091FCBBF80030032B7EF6BBAF3868BAF87E
:1044700000304F4AC31A82FB0321DA17C2EB6102F4
:1044800002EB4202A3EB820303EB430304EB83043E
:10449000A36818447F287FF781AD7F380C2290FBFA
:1044A000F2F302FB1300733018E4DFF80CA140496B
:1044B000BAF800203F4C9A1A81FB020ED017C0EBCD
:1044C0006E0000EB4000A2EB800202EB420254F8C7
:1044D000220018447F2840F3F380A0F17F0381FB82
:1044E0000321DA17C2EB610101EB4101A3EB81006B
:1044F0007330DFF8C8B098F80010C0B204F042FC86
:10450000BBF80030022B7FF6F5AC3868BAF8003003
:10451000274AC31A82FB0321DA17C2EB610202EBBE
:104520004202A3EB820303EB430304EB83035B68C8
:1045300018447F2840F345837F380C2290FBF2F328
:1045400002FB13007330C0B298F8001004F01AFC9C
:10455000BBF80030032B7FF6CDAC3868BAF80030DA
:10456000134AC31A82FB0321DA17C2EB610202EB82
:104570004202A3EB820303EB430304EB8304A3682F
:1045800018447F287FF7F0AC7F380C2290FBF2F3C1
:1045900002FB13007330A8E4FCF774F8FFF7CABB02
:1045A000FCF770F8FFF73EBBFCF76CF846E400BF81
:1045B000ABAAAA2A501C01000C9EFF1F1A9CFF1FC9
:1045C000919CFF1FDFF83CA399F80000BAF8003077
:1045D000C44AC54CC31A82FB0317D917C1EB670144
:1045E00001EB4101A3EB810303EB430354F82330B8
:1045F00018447F286ADD7F3882FB0032C317C3EB83
:10460000620202EB4202A0EB82007330DFF8F8B2E4
:10461000C0B204F0DFFBBBF80030022B7FF6B5A977
:1046200099F80000BAF80030AE4AC31A82FB0321A1
:10463000DA17C2EB610202EB4202A3EB820303EB47
:10464000430304EB83035B6818447F2840F3B6827E
:104650007F380C2290FBF2F302FB13007330C0B2E0
:1046600004F0B8FBBBF80030032B7FF68EA999F855
:104670000000BAF800309B4AC31A82FB0321DA1704
:10468000C2EB610202EB4202A3EB820303EB4303A2
:1046900004EB8304A36818447F2814DD7F380C22C0
:1046A00090FBF2F302FB13007330C0B204F092FBF4
:1046B000FFF76BB9FBF7E6FFA2E6FBF7E3FF2AE69D
:1046C000FBF7E0FF15E7FBF7DDFFEEE7FBF7DAFFAF
:1046D0009CE7DFF830A299F80000BAF80030814A70
:1046E000824CC31A82FB031ED917C1EB6E0101EB8A
:1046F0004101A3EB810303EB430354F82330184437
:104700007F28DADD7F3882FB0032C317C3EB6203F8
:1047100003EB4303A0EB83007330FCE5DFF8E4A177
:104720003868BAF800306F4A704CC31A82FB031E17
:10473000D917C1EB6E0101EB4101A3EB810303EB40
:10474000430354F8233018447F28B3DD7F3882FBBD
:104750000032C317C3EB620303EB4303A0EB8300F8
:1047600073304DE6FBF78EFF40E4DFF898A15D491A
:10477000BAF800205D4C9A1A81FB020ED017C0EBEC
:104780006E0000EB4000A2EB800202EB420254F804
:10479000220018447F2893DDA0F17F0381FB0321D1
:1047A000DA17C2EB610000EB4000A3EB800073302E
:1047B0009FE6FBF767FF96E4FBF764FF14E5DFF87D
:1047C00044A199F80000BAF80030464A484CC31A90
:1047D00082FB0317D917C1EB670101EB4101A3EB82
:1047E000810303EB430354F8233018447F287FF7F9
:1047F0006DAF7F3882FB0032C317C3EB620303EB5C
:104800004303A0EB8300733000E73A4800903A4836
:104810003A490390FEF715B9DFF8E8A03868BAF80E
:104820000030304A364CC31A82FB0321DA17C2EB40
:10483000610202EB4202A3EB820303EB430354F851
:10484000233018447F2840F3B6817F380C2290FB38
:10485000F2F302FB13007330DFF8B080DFF8A8B08A
:1048600098F80010C0B204F08DFABBF80030022BAB
:104870001AD93868BAF800300C22C11A91FBF2F349
:1048800002FB131302FB03435B6818447F2840F3C9
:1048900067847F3890FBF2F302FB13007330C0B2E1
:1048A00098F8001004F06EFABBF80030032B7EF687
:1048B00098ADBAF8003038680C22C11A91FBF2F3B7
:1048C00002FB131302FB0344A36818447F287FF7FD
:1048D00065AB7F3890FBF2F302FB13007330FFF7F8
:1048E000FDB900BFABAAAA2AE4180100D41D01003B
:1048F000C01B0100549EFF1FE59BFF1F109EFF1F62
:10490000801A01000C9EFF1F1A9CFF1F919CFF1F25
:10491000DFF894A399F80000BAF80030D84AD94CCF
:10492000C31A82FB0321DA17C2EB610202EB4202D7
:10493000A3EB820303EB430354F8233018447F288E
:1049400040F320817F380C2290FBF2F302FB13002E
:104950007330DFF858B3C0B204F03CFABBF8003053
:10496000022B19D999F80000BAF800300C22C11AAC
:1049700091FBF2F302FB131302FB03435B68184441
:104980007F2840F322847F3890FBF2F302FB130070
:104990007330C0B204F01EFABBF80030032B7EF671
:1049A000BFABBAF8003099F800000C22C11A91FB95
:1049B000F2F302FB131302FB0344A36818447F289D
:1049C0007FF7CFAA7F3890FBF2F302FB130073301E
:1049D000FFF708BA012B3DF4E6AF0124FFF7A8BAB0
:1049E000DFF8C4A2A649BAF80020A64C9A1A81FBA7
:1049F0000210D117C1EB600101EB4101A2EB810272
:104A000002EB420254F8220018447F2840F3D08081
:104A1000A0F17F030C2093FBF0F200FB1230733007
:104A2000DFF888B298F80010C0B204F0ABF9BBF818
:104A30000030022B1AD93868BAF800300C22C11A9B
:104A400091FBF2F302FB131302FB03435B68184470
:104A50007F2840F382837F3890FBF2F302FB130040
:104A60007330C0B298F8001004F08CF9BBF8003035
:104A7000032B7FF63FAABAF8003038680C22C11A1F
:104A800091FBF2F302FB131302FB0344A3681844E7
:104A90007F287FF769AA7F3890FBF2F302FB1300AF
:104AA0007330FFF722BAFBF7EDFDFFF770B9FBF7A4
:104AB000E9FDFFF7E7B8DFF8F0A199F80000BAF8D0
:104AC00000306F4A704CC31A82FB0321DA17C2EB25
:104AD000610202EB4202A3EB820303EB430354F8AF
:104AE000233018447F2846DD7F380C2290FBF2F3F8
:104AF00002FB13007330DFF8B4B1C0B204F06AF9FE
:104B0000BBF80030022B19D999F80000BAF8003030
:104B10000C22C11A91FBF2F302FB131302FB0343B5
:104B20005B6818447F2840F3A7807F3890FBF2F33E
:104B300002FB13007330C0B204F04CF9BBF8003034
:104B4000032B7EF622AFBAF8003099F800000C2251
:104B5000C11A91FBF2F302FB131302FB0344A36897
:104B600018447F287FF7AFAD7F3890FBF2F302FB4C
:104B70001300733099E5FBF785FDBCE7FBF782FD79
:104B8000FFF789B9FBF77EFDE3E6FBF77BFD63E406
:104B900001339BB22380D9B205203C4C04F0CAF803
:104BA0003B782370FDF7EABDFBF76CFDFFF7DCBB3C
:104BB000FBF768FD34E7FBF765FD4DE6FBF762FDAB
:104BC0004DE5FBF75FFDBEE4DFF8DCA099F80000DF
:104BD000BAF800302A4A2E4CA2E6013B9BB2D9B269
:104BE00005202A4C138004F0A5F83B782370FDF7CC
:104BF000C5BDDFF8B4A03868BAF80030204A244CAC
:104C000011E6FBF73FFDFFF71DBBDFF89CA01C4939
:104C1000BAF800201E4CE9E6FBF734FDFFF793BA23
:104C2000DFF884A099F80000BAF80030144A194C53
:104C300049E7FBF727FDFFF706BA029B1B78002B1D
:104C40007EF44EAAFEF771BA134B1B78002B00F0CE
:104C5000DE82124B1B78002B7DF4A5AE104B1B7827
:104C6000002B3DF4A0AEB8F800300E490A33A8F886
:104C700000300A70FDF797BEFBF704FD5BE700BF4D
:104C8000ABAAAA2A801A0100501C0100029CFF1F37
:104C9000441D0100D41D0100C39DFF1F919EFF1FF5
:104CA000929EFF1F079CFF1F0C9EFF1F1A9CFF1F59
:104CB000A14C2388002B40F05483DFF890B29F4929
:104CC0009F4A098899F80000B2F800E0DFF878827E
:104CD000C1EB000C0C229CFBF2F102FB11C14FF066
:104CE000900C0CFB0EFE02FB01E16FF00B0E58F86E
:104CF000011008440EFB03007F2840F3EC84A0F170
:104D00007F0393FBF2F002FB10307330C0B204F06B
:104D100061F8BBF8002023881344022B22DD874A68
:104D2000874B118899F80000B3F800C0DFF818E24B
:104D3000411A0C2291FBF2F302FB1311902303FBA7
:104D40000CF302FB013373445B6818447F2840F383
:104D500050857F3890FBF2F302FB13007330C0B232
:104D600004F038F8BBF8002023881344032B22DD1D
:104D7000724A734B118899F80000B3F800C0DFF84D
:104D8000C8E1411A0C2291FBF2F302FB13119023AC
:104D900003FB0CF302FB013373449B6818447F2828
:104DA00040F338857F3890FBF2F302FB1300733039
:104DB000C0B204F00FF8BBF8002023881344042B82
:104DC0007EF7AEA95F4B1B88012B7EF4A9A999F849
:104DD0000020A2F10C007F287FF7C3A88B3A0C209B
:104DE00092FBF0F300FB13207330FEF7FBBF524C35
:104DF0002288002A00F018835249DFF850B1098850
:104E0000BBF800000331884227DD4C484C4900883C
:104E1000B1F800E0DFF830C1181A0C2190FBF1F96D
:104E200001FB19004FF0900909FB0EFE01FB00E0A9
:104E30006FF00B0E5CF8000003440EFB02307F287D
:104E400040F311847F3890FBF1F301FB13007330C2
:104E5000C0B298F8001003F095FFBBF8002023883B
:104E60001344022B23DD354B354A38681B88B2F8D2
:104E700000C0DFF8D4E0C31A0C2193FBF1F201FB70
:104E80001232902303FB0CF301FB023373445B6883
:104E900018447F2840F3A5847F3890FBF1F301FB91
:104EA00013007330C0B298F8001003F06BFFBBF82A
:104EB000002023881344032B23DD204B204A38682D
:104EC0001B88B2F800C0DFF880E0C31A0C2193FB06
:104ED000F1F201FB1232902303FB0CF301FB0233CE
:104EE00073449B6818447F2840F37F847F3890FB8D
:104EF000F1F301FB13007330C0B298F8001003F017
:104F000041FFBBF8002023881344042B7EF7F2AF47
:104F10000C4B1B88012B7EF4EDAF3A68A2F10C001C
:104F20007F287FF721A88B3A0C2092FBF0F300FB3F
:104F300013207330FEF7D9BF949CFF1F0C9EFF1FF8
:104F4000B69DFF1F369CFF1FE01501001A9CFF1F36
:104F5000B84C2388002B40F06A82DFF810B3B649C2
:104F6000B64A0988D7F80080B2F800E0B448C1EB2F
:104F7000080C0C229CFBF2F102FB11C14FF0900CCB
:104F80000CFB0EFE02FB01E16FF00B0E405880445B
:104F90000EFB03807F2840F36A83A0F17F0393FB1D
:104FA000F2F002FB10307330A64BC0B2197803F058
:104FB000E9FEBBF8002023881344022B23DD9E4A20
:104FC0009E4B11883868B3F800C0DFF874E2411ACC
:104FD0000C2291FBF2F302FB1311902303FB0CF361
:104FE00002FB013373445B6818447F2840F30B8451
:104FF0007F3890FBF2F302FB13007330914BC0B289
:10500000197803F0BFFEBBF8002023881344032B5C
:1050100023DD894A894B11883868B3F800C0DFF86E
:1050200020E2411A0C2291FBF2F302FB13119023B0
:1050300003FB0CF302FB013373449B6818447F2885
:1050400040F3DE837F3890FBF2F302FB13007330F2
:105050007C4BC0B2197803F095FEBBF80020238882
:105060001344042B7EF7BDA9774B1B88012B7EF4DC
:10507000B8A93A68A2F10C007F2840F3B2808B3ABD
:105080000C2092FBF0F300FB132073306D4BC0B289
:10509000197803F077FEFEF7A4B9DFF89CA199F820
:1050A0000000BAF80030694CC11A0C2291FBF2F3EF
:1050B00002FB131302FB03F3E35818447F287FF726
:1050C0005AAD7F3890FBF2F302FB1300733012E508
:1050D0005F4B1A88182A13D03B681344A3F11800B9
:1050E0007F2840F37B830C20973B93FBF0F200FB7F
:1050F000123303F17300534BC0B2197803F042FE30
:10510000544B55491A78022A94BF013200221A7072
:105110001A7831F81200182810D10424022A02F15A
:105120000100C2B288BF002231F81200182804D151
:10513000013CF3D11A70FEF754B91A703B6803446E
:10514000A3F118007F284CDD0C20973B93FBF0F275
:1051500000FB123303F1730098E7FBF793FA80E446
:10516000FBF790FAFFF79BBB394B1B88182B12D02B
:1051700099F800201344A3F118007F2840F33D83E1
:105180000C20973B93FBF0F200FB123303F173000A
:10519000C0B203F01FFE2F4A2F4B127833F81230A3
:1051A000182B3DF4BDAF99F800201344A3F118006B
:1051B0007F287EF7D6AE0C20973B93FBF0F200FBE6
:1051C000123303F17300FEF70DBEFBF75BFAFFF736
:1051D000E0BBDFF864A099F80000BAF800301F4C7B
:1051E00062E7FBF74FFA51E71D4B1B78002B7DF46C
:1051F000DAAB1C4B1B78002B3DF4D5ABB8F8003074
:105200001949013BA8F800300A70FDF7CCBB144BDC
:105210001B78002B7EF401A8124B1B78002B3DF469
:10522000C2ABB8F8003010490133A8F800300A705A
:10523000FDF7B9BB949CFF1F0C9EFF1FB69DFF1F7F
:10524000E0150100919CFF1F369CFF1F801A010092
:10525000269CFF1F929CFF1F249EFF1F441D0100E0
:10526000919EFF1F929EFF1F079CFF1F1A9CFF1F0E
:10527000944A1288182A12D01344A3F118007F28E8
:1052800040F3CC820C20973B93FBF0F200FB1233EF
:1052900003F17300C0B298F8001003F073FD8A4B5D
:1052A0008A491A78022A94BF013200221A701A78A9
:1052B00031F81200182811D10424022A02F1010049
:1052C000C2B288BF002231F81200182805D1013C73
:1052D000F3D11A703B68FEF77AB91A703B68034441
:1052E000A3F118007F287EF73FAE0C20973B93FB7D
:1052F000F0F200FB123303F17300FEF7F6BD744ABF
:105300001288182A12D01344A3F118007F2840F302
:105310007E820C20973B93FBF0F200FB123303F1EB
:105320007300C0B298F8001003F02CFD664B694979
:105330001A78022A94BF013200221A701A7831F8C2
:1053400012001828CAD10424022A02F1010294BFD3
:10535000D2B2002231F812001828BED1013CF3D19C
:10536000B7E75D4ADFF884B11288BBF8001003325A
:1053700091427FF7CEACA2E4554B1B88182B12D07C
:1053800099F800201344A3F118007F2840F32382EA
:105390000C20973B93FBF0F200FB123303F17300F8
:1053A000C0B203F017FD484A4A4B127833F8123066
:1053B000182B7FF4F8AEFDF7B3BE454B1A88182AB8
:1053C00013D03B681344A3F118007F2840F3F28107
:1053D0000C20973B93FBF0F200FB123303F17300B8
:1053E0003E4BC0B2197803F0CDFC374B39491A78DF
:1053F000022A94BF013200221A701A7831F8120082
:1054000018287FF49BAE0424022A02F1010294BF03
:10541000D2B2002231F8120018287FF48EAE013C7F
:10542000F2D11A70FDF7DDBFDFF8C0B0EDE42A4A13
:10543000DFF8B8B01288BBF80010033291427FF752
:10544000B8AD8CE5264B01227F2107201A8003F09E
:1054500071FC7F210B2003F06DFCFDF709BF214B90
:1054600004227F2107201A8003F064FC00210B2016
:1054700003F060FCFDF7F5BE1A4B02227F210720E6
:105480001A8003F057FC7F210B2003F053FCFDF73B
:10549000E3BE144B002107201C8003F04BFC7F214E
:1054A0000B2003F047FCFDF7D2BE0F4B00227F21FB
:1054B00007201A8003F03EFC7F210B2003F03AFC0A
:1054C000FDF7DEBE269CFF1F929CFF1F249EFF1F40
:1054D0002E9CFF1F989DFF1F369CFF1F919CFF1F56
:1054E000A29CFF1F049EFF1F049CFF1F1A9CFF1F0E
:1054F000CC4C2388002B40F06381DFF854B3CA49B9
:1055000099F80000C94A09881788DFF824E3411A8E
:105510000C2291FBF2FC02FB1C114FF0900C0CFBD7
:1055200007F702FB01716FF00B075EF801100144F1
:1055300007FB03107F2840F340817F3890FBF2F394
:1055400002FB13007330C0B203F044FCBBF8002030
:1055500023881344022B21DDB34BB44A99F8000091
:105560001B88B2F800E0B24FC31A0C2193FBF1F292
:1055700001FB1232902303FB0EF301FB02333B4489
:105580005B6818447F2840F3B1817F3890FBF1F3CA
:1055900001FB13007330C0B203F01CFCBBF8002009
:1055A00023881344032B21DD9F4BA04A99F8000068
:1055B0001B88B2F800E09E4FC31A0C2193FBF1F256
:1055C00001FB1232902303FB0EF301FB02333B4439
:1055D0009B6818447F2840F386817F3890FBF1F365
:1055E00001FB13007330C0B203F0F4FBBBF80020E2
:1055F00023881344042B7EF7C8A98E4B1B88012BEC
:105600007EF4C3A999F80020A2F10C007F287FF74F
:105610005AA88B3A0C2092FBF0F300FB1320733056
:10562000FFF743B8844B1B88182B12D099F8002041
:105630001344A3F118007F2840F35B810C20973BB3
:1056400093FBF0F200FB123303F17300C0B203F0DE
:10565000C1FB7A4A7A4B127833F81230182B7FF458
:10566000A2ADFDF75DBDFBF70DF8FFF7F1BBFBF752
:1056700009F899E4734B1B88182B12D099F8002075
:105680001344A3F118007F2840F339810C20973B85
:1056900093FBF0F200FB123303F17300C0B203F08E
:1056A00099FB664A684B127833F81230182B3EF497
:1056B0006CA999F800201344A3F118007F287FF704
:1056C00002A80C20973B93FBF0F200FB123303F18E
:1056D0007300FEF7EABFFAF7D5FFFFF717BB564A8C
:1056E0001288182A12D01344A3F118007F2840F31F
:1056F00003810C20973B93FBF0F200FB123303F184
:105700007300C0B298F8001003F03CFB4B4B4C49BF
:105710001A78022A94BF013200221A701A7831F8DE
:10572000120018287FF4DAAD0424022A02F10102E3
:1057300094BFD2B2002231F8120018287FF4CDAD08
:10574000013CF2D1C5E53C4B1A88182A13D03B68BE
:105750001344A3F118007F2840F3C2800C20973B2C
:1057600093FBF0F200FB123303F17300374BC0B22E
:10577000197803F007FB314B31491A78022A94BF9C
:10578000013200221A701A7831F8120018287FF4BA
:10579000D5AC0424022A02F1010294BFD2B2002245
:1057A00031F8120018287FF4C8AC013CF2D11A700D
:1057B000FDF717BEFAF766FF12E6FAF763FFC2E6D7
:1057C0001C4ADFF88CB01288BBF8001003329142FB
:1057D0007FF7BCAE93E6FAF755FFE1E5FAF752FF23
:1057E00089E4FAF74FFFFFF75DBBFAF74BFFFFF7CE
:1057F00083BBFAF747FFFFF7B2BAFAF743FFC7E4F4
:10580000FAF740FF24E4FAF73DFFFFF7F7BBFAF79A
:1058100039FF86E5FAF736FFFFF7CABAFAF732FF23
:1058200038E500BF949CFF1F0C9EFF1FB69DFF1F15
:10583000E0150100369CFF1F309CFF1F929CFF1F4C
:10584000A09DFF1F269CFF1F249EFF1F919CFF1FF2
:105850001A9CFF1F304B1B88182B11D099F8002081
:105860001344A3F118007F2834DD0C20973B93FBF1
:10587000F0F200FB123303F17300C0B203F0AAFA96
:10588000264A274B127833F81230182B7FF411AFC9
:10589000FEF77BB8234B1B88182B11D099F80020FA
:1058A0001344A3F118007F2817DD0C20973B93FBCE
:1058B000F0F200FB123303F17300C0B203F08AFA76
:1058C000164A194B127833F81230182B7FF4F1AEC8
:1058D000FEF75BB8FAF7D6FECFE7FAF7D3FEECE7B0
:1058E000FAF7D0FE42E7FAF7CDFE7CE6FAF7CAFEF9
:1058F00051E6FAF7C7FEA9E6FAF7C4FE01E7FAF7A0
:10590000C1FECBE6094B0393094B0293FDF71EBF83
:1059100023601946FDF758BC309CFF1F929CFF1F67
:10592000A09DFF1F2E9CFF1F989DFF1FE59BFF1F43
:10593000B29CFF1F38B507F015F90E4805F04CF87A
:105940000D4805F049F80D4805F046F800234FF0E2
:105950007E5201210A48FAF789FD0A4B0A4A0B498F
:10596000802400251C7118461D60BDE838400AF0EF
:10597000BDBD00BF189CFF1F4C9CFF1FA89CFF1FB4
:10598000E09DFF1F5C9EFF1F1C89FF1F2906000072
:1059900043682A20198803F051BB00BF10B50446A4
:1059A00022206368198803F049FBE36824201988E2
:1059B000BDE8104003F042BB10B504460A206368FE
:1059C000198803F03BFBE3680C201988BDE8104000
:1059D00003F034BB10B5044606206368198803F051
:1059E0002DFBE36808201988BDE8104003F026BBB2
:1059F00010B5044602206368198803F01FFBE368B2
:105A000004201988BDE8104003F018BB70B50E4C97
:105A100084B01225042201230646039002932046F7
:105A20008DE824001423102106F0DAF90622092358
:105A3000029303960195204600921423102106F04C
:105A4000CFF904B070BD00BFC09EFF1F2DE9F0412B
:105A5000224D82B0012602B284B2009228460196FD
:105A60007823192106F002F904F10C0212B28DE834
:105A700044002846A7197823192104F1020806F0EA
:105A8000F5F83FB20FFA88F819233A462846194626
:105A90000196CDF8008006F0E9F878233A462846CA
:105AA0001946CDF80080019604F10A070B3406F080
:105AB000DDF83FB224B278233A46284619468DE8ED
:105AC000500006F0D3F8192300943A460196284670
:105AD000194606F0CBF802B0BDE8F081C09EFF1F6A
:105AE0002DE9F0411E4682B01446002A6AD0099B77
:105AF0004D4A00EBC305012C6F8929896868A7EB23
:105B0000010382FB03E21A444FEAE373C3EBA213DF
:105B100002887BD0042C38D112FA83F3994203DC3B
:105B20009F423946A8BF1946089A0180B6F900304D
:105B3000BDF920803D48971D4FF0000E3FB2194639
:105B400042460097CDF804E006F090F829896A896A
:105B50006B68521A1B885C2AA3EB010359DD03EB27
:105B600043030132C3EB431393FBF2F303F11B0234
:105B700013B20120328019464246019000972B480B
:105B800006F074F82A4B00221A702A4B022CB3F943
:105B9000001045D0082C31D100221A8091422DD01E
:105BA000089AB6F9003021480632012412B2009258
:105BB00019460194BDF9202006F058F8204602B09D
:105BC000BDE8F0811C4D1D4A2B681268CB1A934228
:105BD0000F4617D9164A338811781448012918BF7F
:105BE00001241470089A06321BB212B28DE8140018
:105BF0001946BDF9202006F039F82F60012002B0C7
:105C0000BDE8F081204602B0BDE8F0819BB2D31A16
:105C100084E75C2101FB03F393FBF2F21B32A7E75D
:105C20004A1C12B21A80B9E7C94216B2C09EFF1FC1
:105C3000399FFF1FA29EFF1F249FFF1FFC2D010005
:105C400030B583B000230C4605B2009326225B23B7
:105C50001C210C4805F05AFD29460123262209483B
:105C600005F064F8002C24B205DB2146012326222E
:105C7000044805F05BF8044A044B15801C8003B00F
:105C800030BD00BFC09EFF1F668AFF1F688AFF1FCE
:105C90002DE9F041AA4C237882B01BB1A94B4FF6F5
:105CA000FF721A80A84BB3F90030CBB9A74AA54BB5
:105CB0001068B3F9002080F30C005B2303FB00F0B5
:105CC00000131C30824269D04FF0FF31FFF7B8FF5C
:105CD0009F4805F07FFD0023237002B0BDE8F081EE
:105CE000012B40D0022B78D0032B5DD0042BF2D1B6
:105CF000252200258DE8240076231C219448954E0A
:105D0000954FDFF8888205F0B1FF17E0B0F5AF7F5F
:105D1000A8BF4FF4AF70323802FB00F088FB0031AF
:105D2000C017C0EB61111C3109B201231D442522AB
:105D3000874804F0FBFF0C2D00F08C80E9B2874807
:105D400004F0B2FE56F8043BC3F5967300FB03F073
:105D500087FB0013C017C0EB631031284FF05B02C4
:105D6000D4DC1C21E1E77E4B1A68B2F52F7F32DBD1
:105D700041F25C239342A8BF1346A3F52F735B2225
:105D8000784802FB03F380FB0320DB17C3EBA02062
:105D90001C306C4BB3F90030834295D1724BB3F990
:105DA0000030013390D196E7704B1B68B3F5FA7F52
:105DB00011DBB3F57A6FA8BF4FF47A63A3F5FA72DB
:105DC0006B485B2303FB02F380FB0320DB17C3EB71
:105DD00020201C30DDE71C20DBE7664B1B68B3F599
:105DE000FA7F33DBB3F57A6FA8BF4FF47A63A3F57C
:105DF000FA725F485B2303FB02F380FB0320DB178F
:105E0000C3EB20201C305C4B1B68B3F5FA7F1FDB13
:105E1000B3F57A6FA8BF4FF47A63A3F5FA725449C9
:105E20005B2303FB02F381FB0321DB17C3EB21217F
:105E30001C31444BB3F9003083427FF447AF4A4BE7
:105E4000B3F900308B427FF441AF44E71C20DAE71E
:105E50001C21EEE7262200258DE8240076231C2154
:105E60003B48464E3C4FDFF8248105F0FFFE16E02C
:105E7000B0F5AF7FA8BF4FF4AF70323802FB00F02F
:105E800088FB0031C017C0EB61111C3109B201233E
:105E90001D4426222E4804F049FF0C2D14D0E9B2EF
:105EA000374804F001FE56F8043BC3F5967300FB37
:105EB00003F087FB0013C017C0EB631031284FF0CD
:105EC0005B02D5DC1C21E2E7272200258DE82400B7
:105ED00076231C211E482B4E1F4FDFF8B08005F0A3
:105EE000C5FE17E0B0F5AF7FA8BF4FF4AF703238F2
:105EF00002FB00F088FB0031C017C0EB61111C31C0
:105F000009B201231D442722114804F00FFF062D7A
:105F10003FF4DEAEE9B21C4804F0C6FD56F8043B7F
:105F2000C3F5967300FB03F087FB0013C017C0EBAB
:105F3000631031284FF05B02D4DC1C21E1E700BF85
:105F4000989EFF1F668AFF1F9E9EFF1F189EFF1FC1
:105F5000C09EFF1F1C8AFF1FB5814E1B4C9CFF1F5C
:105F6000F49BFF1FD3058541688AFF1F3C9CFF1FE0
:105F7000011FB812489CFF1F889EFF1F2C89FF1F1E
:105F8000A89CFF1F4C8AFF1F189CFF1F4B48371B04
:105F90002DE9F04FDFF8EC82B74CB8F900604D788E
:105FA00054F8264087B08246039305B10D78DFF898
:105FB000FCB2002A34D19BF800308BBBAF4EB6F94F
:105FC0000000002800F0CE80012800F0248101208C
:105FD00032232A46019000935146A94B2046FFF7F1
:105FE0007FFD00250746B6F90030022B40F3F48010
:105FF00000233380B8F90030A24A002BC0F2F880A9
:10600000042BC4BF00231380039B002B40F0F680B9
:10601000002D0CBF38464FF0FF3007B0BDE8F08FC1
:10602000964EE368226898480493002705923780CB
:106030008BF8007005F0C2FA1120FFF707FD4FF052
:10604000010919232821CDF8049000912422194632
:106050008D4805F00BFE782328212422CDF80490EA
:1060600000918948194605F001FE4946864806F028
:1060700093F902221921844806F08AF9DDF8149078
:1060800048460AF0FDFF494602467F4806F01AFBE3
:106090007D4806F02DFB394614227B4806F078F93E
:1060A00003227A49784806F00DFB774806F020FB7A
:1060B00039462322744806F06BF90322744972486A
:1060C00006F000FB704806F013FB049B002B72D116
:1060D0000123704A18461370FFF798FC20896389E2
:1060E0006768191A5C293A885BDC131A5C2202FB88
:1060F00003F292FBF1F31B33674A634813800127D5
:106100001BB21A2219468DE88400142205F0AEFD58
:10611000049BDBB1218A638AE768581A5C283A88B5
:106120006FDD521A02EB4202C2EB4212431C92FB99
:10613000F3F31B33524A54481380012738221BB211
:106140008DE884001946322205F090FD534A544BE5
:10615000B6F90000012111704FF6FF721A80002875
:106160007FF432AFDFF848914E4AD9F80030126818
:10617000C3EB0A0393424CD9464B1A78012A18BF45
:10618000012018700127FFF741FCC9F800A0012D7C
:106190004ED0042D59D0022D60D0082D64D000259A
:1061A00021E7121A02EB4202C2EB42124B1C92FB95
:1061B000F3F31B33A0E72F20FFF748FC39463222C8
:1061C000314806F0E5F8032237492F4806F07AFAFD
:1061D0002D4806F08DFA7BE77FF40CAFE368002BC7
:1061E0003FF406AFB8F90030264A002BBFF608AFDF
:1061F00004231380039B002B3FF40AAFFFF748FDF5
:1062000006E7511A5C2202FB01F292FBF0F31B330A
:1062100090E70746BBE7002714238DE888002A464D
:1062200051461D4B2046FFF75BFC3D460746DAE62C
:10623000B8F800308BF800500133A8F800306369DB
:1062400083B1002520469847CDE6B8F800300122FA
:10625000013BA8F800308BF80020F0E701233380E1
:106260000025C7E61D46BEE66369002232804FF076
:10627000FF35002BE6D1BDE66C8AFF1FA29EFF1FF3
:106280009C9EFF1F9E9EFF1FC09EFF1F241F01009C
:10629000281F0100399FFF1F9A9EFF1F989EFF1F16
:1062A000668AFF1FFC2D01002C1F0100A09EFF1F0E
:1062B000249FFF1F01210D2007F0CEB800210D20E3
:1062C00007F0CAB801460D2007F0C6B808B50D2082
:1062D00007F0C8F8B0FA80F149090D20BDE8084080
:1062E00007F0BAB810B5002144080D2007F0B4F843
:1062F000204607F0EDF80D20012107F0ADF820460B
:10630000BDE8104007F0E4B82D4A2E4B10881B68FA
:10631000984210B549DA2C4A1288141A9A42A8BF3A
:106320001A46B4F5157F36DA121A40F2532303FBEE
:1063300002F393FBF4F105310A2006F0FDFE234B36
:106340001978C9B3224B23491B6840F2271283F303
:10635000070302FB03F381FB03211944DB17C3EBA3
:10636000A1110531092006F0E7FE1B4B1968F1B1B8
:1063700081F3070140F22712164802FB01F380FB6C
:1063800003211944DB17C3EBA11105311620BDE829
:10639000104006F0D1BE131A4FF41572611C02FBB7
:1063A00003F393FBF1F10531C6E70021C4E71620A2
:1063B000BDE8104006F0C0BE092006F0BDFED4E7DF
:1063C000B09CFF1FE89BFF1F6A9EFF1F6A9CFF1F78
:1063D000EC9BFF1F090402812C9EFF1F7F2838B50C
:1063E000A8BF7F200F4C4FF4167202FB00F284FB13
:1063F00002311144D2170546C2EBA1110A2006F062
:106400009BFE7F3D4FF4967303FB05F384FB032152
:106410001944DB17A3EBA1110920BDE8384006F0B1
:106420008BBE00BF09040281C368B3F9003030B5E8
:1064300083EAE374A4EBE374002BA0B218DB01231E
:1064400000E0134603EB830252009442F9DA0A4D4E
:1064500090FBF3F285FB03E403FB1200DB17303201
:10646000D3EBA40380B201F8012BF1D10B7030BD46
:106470002D230B700131E2E76766666638B5094D7A
:106480008224204602F0F4FD35F8021B00B2884257
:10649000204601D002F0D2FD0234A4B28A2CF0D101
:1064A00038BD00BFA09DFF1F024B8020198802F05D
:1064B000C5BD00BF309CFF1F38B5094D782420466C
:1064C00002F0D6FD35F8021B00B28842204601D00A
:1064D00002F0B4FD0234A4B2802CF0D138BD00BF6C
:1064E000989DFF1F024B7620198802F0A7BD00BFC0
:1064F0002E9CFF1F38B5094D4624204602F0B8FDFA
:1065000035F8021B00B28842204601D002F096FD09
:106510000234A4B24E2CF0D138BD00BF249EFF1F20
:10652000024B4420198802F089BD00BF269CFF1F42
:10653000024B4E20198802F081BD00BF449CFF1F12
:10654000024B9A20198802F079BD00BF949CFF1F6E
:10655000024B9820198802F071BD00BF369CFF1FC6
:10656000024B8C20198802F069BD00BFB69DFF1F49
:10657000024B9C20198802F061BD00BF1A9CFF1FCE
:10658000024BA020198802F059BD00BF8C9EFF1F4E
:10659000024B9620198802F051BD00BF0C9EFF1FD0
:1065A000024B8A20198802F049BD00BFCE9DFF1F13
:1065B00008B5034B1020198802F040FD012008BDEA
:1065C000CC9DFF1F024B1020198802F037BD00BF81
:1065D000CC9DFF1F024B2C20198802F02FBD00BF5D
:1065E000169CFF1F024B1E20198802F027BD00BF1A
:1065F000349CFF1FC3680E20198802F01FBD00BF26
:10660000024B2820198802F019BD00BF209EFF1FF1
:10661000024B6420198802F011BD00BF1C9EFF1FB1
:10662000024B5A20198802F009BD00BFFC9BFF1FD6
:10663000024B1620198802F001BD00BF049CFF1F09
:10664000024B2E20198802F0F9BC00BF9C9CFF1F52
:10665000024B3020198802F0F1BC00BF749EFF1F6E
:10666000024B9E20198802F0E9BC00BFC089FF1FC1
:10667000024B1820198802F0E1BC00BFB49CFF1F38
:10668000024B1A20198802F0D9BC00BF4E9CFF1F94
:10669000024B1C20198802F0D1BC00BF469CFF1F92
:1066A000024B6620198802F0C9BC00BF529EFF1F32
:1066B000024B7220198802F0C1BC00BF709EFF1F00
:1066C000024B2020198802F0B9BC00BF509EFF1F6A
:1066D000024B3220198802F0B1BC00BF469EFF1F5A
:1066E000024B6820198802F0A9BC00BF809CFF1FE4
:1066F000024B6C20198802F0A1BC00BFF09BFF1F69
:10670000024B6E20198802F099BC00BF969EFF1FB5
:10671000024B5220198802F091BC00BF5E89FF1F16
:10672000024B5020198802F089BC00BF148AFF1F59
:10673000024B5420198802F081BC00BF168AFF1F4B
:10674000024B5C20198802F079BC00BF648AFF1FED
:10675000024B5E20198802F071BC00BF5C89FF1FEC
:10676000024B6020198802F069BC00BFBC9DFF1F6E
:10677000024B5620198802F061BC00BF8E9CFF1F9F
:10678000244B1B880B2B43D8DFE803F00B10151AA2
:106790001F24292E33383D06084604221E490AF0DC
:1067A0002DBD084604221D490AF028BD08460422D2
:1067B0001B490AF023BD084604221A490AF01EBDEF
:1067C0000846042218490AF019BD08460422174950
:1067D0000AF014BD0846042215490AF00FBD084608
:1067E000042214490AF00ABD0846042212490AF09C
:1067F00005BD0846042211490AF000BD08460422DE
:106800000F490AF0FBBC084604220E490AF0F6BC08
:10681000704700BF0C9EFF1FD42A0100A82801006A
:106820005C2701004428010060270100E02B0100E3
:106830006427010068270100E02901006C2701009E
:10684000E02A010070270100064B074A10B41C889B
:10685000064B0846002C14BF11461946042210BCF2
:106860000AF0CCBC649CFF1F74270100782701004C
:10687000064B074A10B41C88064B0846002C14BF70
:1068800011461946042210BC0AF0B8BC9E9CFF1F9A
:106890007427010078270100064B074A10B41C88B2
:1068A000064B0846002C14BF11461946042210BCA2
:1068B0000AF0A4BCBE9DFF1F7427010078270100C9
:1068C000064B074A10B41C88064B0846002C14BF20
:1068D00011461946042210BC0AF090BC0E9EFF1F00
:1068E0007427010078270100064B074A10B41C8862
:1068F000064B0846002C14BF11461946042210BC52
:106900000AF07CBCA29CFF1F7427010078270100BD
:106910001B4B1B880A2B0AD8DFE803F00A0E12165D
:106920001A1E22262A2E0600164B18680860704789
:10693000154B186808607047144B1868086070475A
:10694000134B186808607047124B1868086070474E
:10695000114B186808607047104B18680860704742
:106960000F4B1868086070470E4B18680860704736
:106970000D4B1868086070470C4B1868086070472A
:10698000CE9DFF1FA0270100782701007C27010072
:106990008027010084270100882701008C2701003F
:1069A0009027010094270100982701009C270100EF
:1069B000F0B52B4E2B4FDFF8C4E005460FCE87B065
:1069C0006C460FC496E803003B68274A274F44F8FB
:1069D000040B40F6CC308342C8BF3A46BEF8006094
:1069E0002180012E11889278ADF80D108DF80F20BE
:1069F0002AD032D340F6CA02022E18BF00229A4291
:106A000026DCA3F698031A491A4AC3EB031381FB49
:106A100003011944DB17C3EB6123243382FB0321F9
:106A2000DA17C2EBA10202EB8201A3EB4103303380
:106A300030328DF813308DF8112069462846162221
:106A40000AF0DCFB07B0F0BD40F698029A42D8DDB0
:106A5000094B1868CDF81100EFE740F6FC02CEE7CD
:106A6000B4270100309EFF1FA8270100A4270100C2
:106A70003B773B9867666666AC270100A89DFF1FC1
:106A8000F8B5174C174E2278174D33782F888E465D
:106A9000003218BF012201467046FFF779FA002341
:106AA00098423370237015DB14BF012000202B881F
:106AB0009F420ED040F23A72A3F5AF730B490C4CD3
:106AC00002FB03F381FB0312DB17A3EB62133233E8
:106AD0002360F8BD0749012218460A702270E6E7D4
:106AE000108BFF1FB19EFF1F649EFF1FB5814E1BC1
:106AF000048AFF1F389FFF1F014B187802F036BA37
:106B0000209FFF1F014B187802F04ABAB490FF1F74
:106B1000134BB3F9003030B583EAE374A4EBE374AC
:106B2000002BA0B218DB012300E0134603EB830225
:106B300052009442F9DA0B4D90FBF3F285FB03E42B
:106B400003FB1200DB173032D3EBA40380B201F851
:106B5000012BF1D10B7030BD2D230B700131E2E719
:106B6000B490FF1F67666666144BB3F9003070B5CA
:106B700083EAE375A5EBE375002BACB21ADB0123C6
:106B800000E0034603EB830040008542F9DA0C4E37
:106B900094FBF3F086FB03E503FB1044DB17303076
:106BA000D3EBA503A4B201F8010BF1D105480B709A
:106BB000106070BD2D230B700131E0E7FC9BFF1FBF
:106BC00067666666CC270100134BB3F9003030B519
:106BD00083EAE374A4EBE374002BA0B218DB012377
:106BE00000E0134603EB830252009442F9DA0B4DA6
:106BF00090FBF3F285FB03E403FB1200DB1730325A
:106C0000D3EBA40380B201F8012BF1D10B7030BD9E
:106C10002D230B700131E2E7C089FF1F67666666AE
:106C2000134BB3F9003030B583EAE374A4EBE3749B
:106C3000002BA0B218DB012300E0134603EB830214
:106C400052009442F9DA0B4D90FBF3F285FB03E41A
:106C500003FB1200DB173032D3EBA40380B201F840
:106C6000012BF1D10B7030BD2D230B700131E2E708
:106C70005E89FF1F67666666134BB3F9003030B557
:106C800083EAE374A4EBE374002BA0B218DB0123C6
:106C900000E0134603EB830252009442F9DA0B4DF5
:106CA00090FBF3F285FB03E403FB1200DB173032A9
:106CB000D3EBA40380B201F8012BF1D10B7030BDEE
:106CC0002D230B700131E2E7148AFF1F67666666A9
:106CD000134BB3F9003030B583EAE374A4EBE374EB
:106CE000002BA0B218DB012300E0134603EB830264
:106CF00052009442F9DA0B4D90FBF3F285FB03E46A
:106D000003FB1200DB173032D3EBA40380B201F88F
:106D1000012BF1D10B7030BD2D230B700131E2E757
:106D2000168AFF1F67666666134BB3F9003030B5ED
:106D300083EAE374A4EBE374002BA0B218DB012315
:106D400000E0134603EB830252009442F9DA0B4D44
:106D500090FBF3F285FB03E403FB1200DB173032F8
:106D6000D3EBA40380B201F8012BF1D10B7030BD3D
:106D70002D230B700131E2E7648AFF1F67666666A8
:106D8000134BB3F9003030B583EAE374A4EBE3743A
:106D9000002BA0B218DB012300E0134603EB8302B3
:106DA00052009442F9DA0B4D90FBF3F285FB03E4B9
:106DB00003FB1200DB173032D3EBA40380B201F8DF
:106DC000012BF1D10B7030BD2D230B700131E2E7A7
:106DD0005C89FF1F6766666608B5702002F048F997
:106DE000044B1988884204D07020BDE8084002F0A6
:106DF00025B908BDA89DFF1F08B5742002F038F919
:106E0000044B1988884204D07420BDE8084002F081
:106E100015B908BD3C9EFF1F054B1B880846042280
:106E200013B904490AF0EAB903490AF0E7B900BF07
:106E3000449CFF1FD4270100D02701000E4B1B8864
:106E4000032B17D8DFE803F0110C070208460422D1
:106E50000A490AF0D3B90846042209490AF0CEB912
:106E60000846042207490AF0C9B90846042206491F
:106E70000AF0C4B9704700BFB69DFF1FE4270100A8
:106E8000E0270100DC270100D827010010B40A4BDD
:106E90000A4C0A4693E8030083B0238802AC04E955
:106EA000030004EB8303104653F8081C052203B0CB
:106EB00010BC0AF0A3B900BFB41F01001C9EFF1F45
:106EC00030B40A4B0A4D0C4693E8070084B02B8877
:106ED00004AD05E9070005EB8303204653F80C1CBD
:106EE000042204B030BC0AF089B900BFBC1F010005
:106EF000A89DFF1FF0B40C4D0C4F0E460FCD8CB06B
:106F000001AC0FC40FCD0FC495E807003B8884E89F
:106F100007000CAA02EB8303304653F82C1C042212
:106F20000CB0F0BC0AF06AB9C81F0100049EFF1F34
:106F3000F0B40A4D0A4F0E460FCD86B001AC0FC417
:106F40002A683B88226006AA02EB8303304653F886
:106F5000141C042206B0F0BC0AF050B9F41F010062
:106F6000B49CFF1FF0B40A4D0A4F0E460FCD86B0F9
:106F700001AC0FC42A683B88226006AA02EB830397
:106F8000304653F8141C0C2206B0F0BC0AF036B997
:106F900008200100469CFF1FF0B40A4D0A4F0E4620
:106FA0000FCD86B001AC0FC42A683B88226006AAC8
:106FB00002EB8303304653F8141C042206B0F0BCE5
:106FC0000AF01CB91C2001003C9EFF1F164B1B88B9
:106FD0000BB31BB283EAE370A0EBE370002B30B578
:106FE00084B21DDB012300E0134603EB8302520051
:106FF0009042F9DA0D4894FBF3F280FB03E503FBC2
:107000001244DB173032D3EBA503A4B201F8012BF5
:10701000F1D10B7030BD0846042205490AF0EEB8E4
:107020002D230B700131DDE7809CFF1F67666666CC
:10703000E8270100F0B40A4D0A4F0E460FCD86B086
:1070400001AC0FC42A683B88226006AA02EB8303C6
:10705000304653F8141C042206B0F0BC0AF0CEB837
:1070600030200100F09BFF1F054B1B881BB9054B0F
:107070001868086070470846042203490AF0BEB841
:10708000949CFF1F7827010074270100164B1B8872
:107090000BB31BB230B583EAE374A4EBE374002BAB
:1070A000A0B21CDB012300E0134603EB8302520075
:1070B0009442F9DA0D4D90FBF3F285FB03E403FBF8
:1070C0001200DB173032D3EBA40380B201F8012B9E
:1070D000F1D10B7030BD064B1868086070472D2346
:1070E0000B700131DEE700BF349CFF1F67666666E8
:1070F00078270100164B1B880BB31BB230B583EA0F
:10710000E374A4EBE374002BA0B21CDB012300E0CA
:10711000134603EB830252009442F9DA0D4D90FBC3
:10712000F3F285FB03E403FB1200DB173032D3EBF1
:10713000A40380B201F8012BF1D10B7030BD064BD6
:107140001868086070472D230B700131DEE700BF1F
:10715000129EFF1F6766666678270100164B1B8824
:107160000BB31BB230B583EAE374A4EBE374002BDA
:10717000A0B21CDB012300E0134603EB83025200A4
:107180009442F9DA0D4D90FBF3F285FB03E403FB27
:107190001200DB173032D3EBA40380B201F8012BCD
:1071A000F1D10B7030BD064B1868086070472D2375
:1071B0000B700131DEE700BF049CFF1F6766666647
:1071C000EC270100174B1B881BB31BB270B583EA79
:1071D000E375A5EBE375002BACB21EDB012300E0E9
:1071E000034603EB830040008542F9DA0E4E94FB20
:1071F000F3F086FB03E503FB1044DB173030D3EBE1
:10720000A503A4B201F8010BF1D108480B7010607E
:1072100070BD074B1868086070472D230B70013153
:10722000DCE700BF9C9CFF1F67666666F0270100D5
:1072300078270100164B1B880BB31BB230B583EACD
:10724000E374A4EBE374002BA0B21CDB012300E089
:10725000134603EB830252009442F9DA0D4D90FB82
:10726000F3F285FB03E403FB1200DB173032D3EBB0
:10727000A40380B201F8012BF1D10B7030BD064B95
:107280001868086070472D230B700131DEE700BFDE
:10729000749EFF1F6766666678270100164B1B8881
:1072A0000BB31BB230B583EAE374A4EBE374002B99
:1072B000A0B21CDB012300E0134603EB8302520063
:1072C0009442F9DA0D4D90FBF3F285FB03E403FBE6
:1072D0001200DB173032D3EBA40380B201F8012B8C
:1072E000F1D10B7030BD064B1868086070472D2334
:1072F0000B700131DEE700BF529EFF1F67666666B6
:1073000078270100164B1B880BB31BB230B583EAFC
:10731000E374A4EBE374002BA0B21CDB012300E0B8
:10732000134603EB830252009442F9DA0D4D90FBB1
:10733000F3F285FB03E403FB1200DB173032D3EBDF
:10734000A40380B201F8012BF1D10B7030BD064BC4
:107350001868086070472D230B700131DEE700BF0D
:10736000709EFF1F6766666678270100174B1B88B3
:107370001BB31BB270B583EAE375A5EBE375002B75
:10738000ACB21EDB012300E0034603EB83004000A8
:107390008542F9DA0E4E94FBF3F086FB03E503FB1E
:1073A0001044DB173030D3EBA503A4B201F8010B76
:1073B000F1D108480B70106070BD074B1868086069
:1073C00070472D230B700131DCE700BF509EFF1F7B
:1073D00067666666F027010078270100074B1B8867
:1073E000022B06D0012B0CBF054B064B186808601A
:1073F0007047054B18680860704700BFBC9DFF1FB1
:10740000F8270100FC270100F4270100054B1B8829
:107410001BB1054B186808607047044B186808607A
:10742000704700BF8E9CFF1F042801000028010048
:10743000184B1A8852B3184A128830B50A80B3F92B
:107440000030002B83EAE374A4EBE374BCBF2D236C
:107450008B70A0B2ACBF02310331012300E01346B0
:1074600003EB830252009442F9DA0C4D90FBF3F2E5
:1074700085FB03E403FB1200DB173032D3EBA403DC
:1074800080B201F8012BF1D10B7030BD044B1868AC
:10749000086070474E9CFF1F0828010067666666FB
:1074A0007827010070B53C4D2B780646002B35D16E
:1074B0001C4673780BB9204670BDFAF75DFC374A5D
:1074C000374B3848127831781B78007802EB430349
:1074D0004A1E03EB80030E2AEDD801A050F822F0DB
:1074E000497500006B750000B77400004975000015
:1074F000B7740000B7740000B7740000377500005F
:10750000B7740000B7740000B7740000B7740000CF
:10751000B7740000B774000033750000AE21224834
:1075200003F0FCFD204804F049F800232B700124EF
:10753000BFE706F0DFFAAF211B4803F0EFFD1B4A5F
:10754000012313702B70B6E783B919480388042907
:107550004FF6FF7103F1FF320CBF01230B461344BA
:1075600003F07F03013303800FE073B1013B114A45
:1075700032F813304BB10E4E0F481049104A338089
:107580000123002606700B701370084A02210123A4
:1075900011702B70204670BD108BFF1F559EFF1F72
:1075A000569EFF1F579EFF1FC09EFF1F389FFF1F45
:1075B000DC9DFF1F889DFF1F789CFF1F079CFF1FFE
:1075C0003B9FFF1F10B5064B064C1A882046012131
:1075D00001F022FD21884220BDE8104001F02EBDBF
:1075E000649CFF1F249CFF1F10B5064B064C1A8895
:1075F0002046022101F010FD21884220BDE8104004
:1076000001F01CBD9E9CFF1F249CFF1F10B5064B64
:10761000064C1A882046042101F0FEFC21884220F5
:10762000BDE8104001F00ABDBE9DFF1F249CFF1F56
:1076300010B5064B064C1A882046002101F0ECFCE0
:1076400021884220BDE8104001F0F8BC0E9EFF1FCB
:10765000249CFF1F08B5122001F00AFD054B198874
:10766000884206D0122001F0E9FCBDE8084001F094
:10767000FDBB08BD049EFF1F08B5582001F0F8FCB3
:10768000054B1988884206D0582001F0D7FCBDE888
:10769000084001F0EBBB08BD129EFF1F08B5142087
:1076A00001F0E6FC054B1988884206D0142001F051
:1076B000C5FCBDE8084001F0D9BB08BDA29CFF1F76
:1076C000F0B480EAE075A5EBE0750028ACB21FDBF2
:1076D0001DBF2B230B704E1C0E46012300E01346EA
:1076E00003EB830252009542F9DA0B4F94FBF3F25D
:1076F00087FB030503FB1244DB173032D3EBA503F2
:10770000A4B206F8012BF1D133700846F0BC7047E3
:107710002D230B704E1CE0E767666666084B1888E1
:1077200028B10D2807D00D3800B2FFF7C9BF054AB0
:10773000106808607047044A10680860704700BF0E
:10774000969EFF1F782701000C280100174B188810
:107750000C2813D0192815D01A2817D01B2819D097
:107760001C281BD01D281DD01E2803D00C3800B2A9
:10777000FFF7A6BF0E4A1068086070470D4A1068F0
:10778000086070470C4A1068086070470B4A106820
:10779000086070470A4A106808607047094A106814
:1077A00008607047084A106808607047469EFF1FCF
:1077B00028280100102801001428010018280100C1
:1077C0001C2801002028010024280100034B1888F0
:1077D000A0EB8000400000B2FFF772BF209FFF1FA8
:1077E000024B1888033800B2FFF76ABF209EFF1FC4
:1077F000024B18880C3800B2FFF762BF009CFF1FD5
:10780000024B1888183800B2FFF75ABF309CFF1F90
:10781000024B1888183800B2FFF752BF2E9CFF1F8A
:10782000024B1888183800B2FFF74ABF269CFF1F8A
:10783000C3681888183800B2FFF742BF054B1B8891
:107840001BB9054B186808607047084604220349B5
:1078500009F0D4BC8C9EFF1F78270100742701001B
:10786000054B1B881BB9054B186808607047084614
:107870000422034909F0C2BC369CFF1F782701008F
:107880007427010030B5134C85B001252B463C22EE
:1078900002212046009503F0B7FC204603F08EFE3F
:1078A00000224021802320460191009311460A4B7B
:1078B000029504F031FB204603F08CFF074808498D
:1078C000084A0023036083800B608B8013609380E1
:1078D00005B030BDC09EFF1FE0220100A49EFF1F27
:1078E000B89EFF1F289FFF1F10B500EBC00000F1DE
:1078F0000F02D2B293B284B09C1E981C3D23039118
:107900008DE819003921024804F06AFA04B010BD6C
:10791000C09EFF1F014B01221A707047B19EFF1FCE
:10792000F0B5664B664C674F674E684D85B00422D4
:107930008DE80C0002932046654B4022802103F025
:107940006BFA2046634A6449644C08F0CFFD644BEF
:1079500064489F61644FDF61644FB761644FF761B2
:10796000644FAF61644FEF61644FA761644FE7619B
:10797000644F87616449654FC761654F8F61654A90
:10798000654FCF61654F9761654B664FD761664F15
:107990009F61664E664FDF61664FB761664D674F08
:1079A000F761674F674CAF61674FEF61674F68489A
:1079B000A761684FE761684F68498761684FC76191
:1079C000684F694A8F61694FCF61694F694B976111
:1079D000694FD761694F6A4E9F616A4FDF616A4F95
:1079E0006A4DB7616A4FF7616A4FAF616A4C6B4F7E
:1079F000EF616B4FA7616B486B4FE7616B4F87611E
:107A00006B496C4FC7616C4F8F616C4A6C4FCF6193
:107A10006C4F97616C4B6D4FD7616D4F9F616D4E91
:107A20006D4FDF616D4FB7616D4D6E4FF7616E4FFA
:107A3000AF616E4C6E4FEF616E4FA7616E486F4F36
:107A4000E7616F4F87616F496F4FC7616F4F704A32
:107A50008F61704FCF61704F704B9761704FD761DE
:107A6000704F714E9F61714FDF61714F714DB76102
:107A7000714FF761714F724CAF61724F7248734929
:107A8000EF61734F734DA761E561734F734D744C94
:107A9000DFF8F0E1734A744B8761744EC561744F2F
:107AA0008C61744D744CC1F81CE074487449976142
:107AB000D5619C61D861B16005B0F0BD40420F0056
:107AC000C09EFF1FF1770000108FFF1F808EFF1FE9
:107AD000D090FF1F1C89FF1F71AE0000788CFF1F24
:107AE000988DFF1F348FFF1FF5650000E1770000C0
:107AF0000166000049680000C5750000716800005B
:107B0000E975000099680000748DFF1F0D76000074
:107B10008D6E0000E48CFF1F11660000C16800003C
:107B2000508DFF1F31760000CD7700002C8DFF1F98
:107B3000F96A0000116B0000EC8EFF1F056B00005E
:107B4000C16E00000C8CFF1FD96D0000F56E0000A7
:107B5000A08FFF1F55760000F5700000C08CFF1F3E
:107B600079760000696B0000C88BFF1F216600005A
:107B7000E96800000C90FF1F9D7600005D71000019
:107B80009C8CFF1F31660000C5710000BC8DFF1F7B
:107B90004166000035720000548CFF1F51660000E2
:107BA000C96B0000388BFF1F61660000316F000059
:107BB000088DFF1F7166000031740000C88EFF1F22
:107BC00081660000656F00009090FF1F91660000C5
:107BD0009D7200005C8EFF1FA1660000057300000F
:107BE0005C8BFF1FB1660000996F0000C48FFF1F00
:107BF000F96D00006D730000A48EFF1FC1660000C8
:107C00004D770000808BFF1FD1660000CD6F000014
:107C1000148BFF1FE166000035700000808AFF1F93
:107C2000F16600001D7700006090FF1F01670000F3
:107C3000216C0000308CFF1F11670000796C000080
:107C4000EC8AFF1F21670000A48BFF1F588FFF1FC6
:107C5000D16C000031670000296D00004167000011
:107C6000816D0000C88AFF1FA48AFF1F8490FF1F38
:107C7000DD730000616700000D7400007167000093
:107C80000D82000051670000F0B5461C83B00D4620
:107C90000127032336B22AB2044631468DE8880014
:107CA0002448ADB204F032F80C23AA1C12B200939F
:107CB0000197052321B21F4804F028F81E4A1F4BE4
:107CC00012881B68BA422AD023D3022A10D11C4C36
:107CD000A3F6CA0384FB03241C44DB17C3EB241460
:107CE0000A2CA8BF0A2424EAE474A2B223B202E058
:107CF00000231A461C460D35AA1A01200093019054
:107D000012B2314603230B4803F07EFF204603B036
:107D1000F0BD0C4CA3F6FC0384FB0324DDE7084C08
:107D2000A3F6980384FB03241C44DB17C3EBE40491
:107D3000D6E700BFC09EFF1FA89DFF1F309EFF1FFC
:107D4000898888881F85EB512DE9F0438FB283B075
:107D5000DFF84C80BD1D461D2DB204B236B24FF087
:107D600001090AB22346314640460095CDF80490F9
:107D700003F07CFF2A463346214640468DE8200228
:107D800003F074FF07F10C020095334612B221464E
:107D9000CDF80490404603F069FF03B0BDE8F083DE
:107DA000C09EFF1F2DE9F043804685B0002956D1C3
:107DB0000121304804F0F0FA2F4998F8062098F88D
:107DC000083011F80290994522DA4FEA89064D46AB
:107DD0000C24D8F80C3027489B595F6822B2002148
:107DE00004F0D6FA384609F04BF9394602462148E4
:107DF00004F068FC1F4804F07BFC98F8083001355B
:107E00000934AB42A4B206F1040601DD422CE0D1F4
:107E1000B9F1000F13D109F1060999450CDA3C2399
:107E200001213B22039102930093019239233F22C7
:107E30003A21104803F0D4FF05B0BDE8F0830F23CA
:107E400001213B22039102930093019239230C22DA
:107E50003A21084803F0C4FF98F80830DBE7002116
:107E60003423009301913F230C22024803F0CCFEFF
:107E70009EE700BFC09EFF1FB89EFF1F10B5104CAD
:107E80000121204604F08EFA2046012104F084FAF4
:107E900020463422552104F07BFA2046022209496B
:107EA00004F010FC20460522074904F00BFC204694
:107EB00004F01EFC2046BDE8104003F08BBC00BF60
:107EC000C09EFF1F2C2801003028010070B50D4610
:107ED000064609F0D5F800EB40008400002D36D0AE
:107EE000284609F0CDF800EB4000400023185B1055
:107EF00003F16001091A282209B21748C3F160048E
:107F000004F046FA0121144804F046FA284609F024
:107F1000B7F829460246104804F0D4FB0E4804F096
:107F2000E7FB02210C4804F037FA21B221220A486B
:107F300004F02EFA304609F0A3F83146024606480E
:107F400004F0C0FB0448BDE8704004F0D1BB6410ED
:107F5000C4F16004E5E700BFC09EFF1F184B70B579
:107F6000B3F9003083EAE374A4EBE374002B82B02E
:107F7000A1B21EDB68466D46012300E0134603EB09
:107F8000830252009442F9DA0E4E91FBF3F286FB23
:107F900003E403FB1211DB173032D3EBA40389B2E5
:107FA00005F8012BF1D119462B70FFF78FFF02B0B6
:107FB00070BD2D238DF800300DF101056846DBE71B
:107FC000CC9DFF1F6766666610B50D4B1B5C51F8B4
:107FD0002340237884B013B1012004B010BD04AA5B
:107FE00001A942F8103D2046A3699847A38A9B0740
:107FF000F2D401A80099FFF769FF012004B010BD79
:10800000A49EFF1F2DE9F04F2F4DDFF8CCB0DFF815
:10801000C4A0DFF8C8900FCD91B003AC0FC40FCD52
:108020000FC40FCD0FC42B6823600025A8462F4630
:108030002E4600E09846BAF8003024495BF8232029
:1080400028461123F8F730FB00EBC00400EB840056
:1080500089FB00340444C017C0EB6434C4F13C0015
:10806000C6F13C0207F14101012600B208F14103CB
:1080700000901BB2019612B209B2154803F0F6FD4A
:1080800008EB060305F211153C2B2646ADB2474618
:10809000D0D134226B210E4804F07AF900210C482B
:1080A00004F07AF90B4B1B8810AA02EB830353F8F8
:1080B000344C204608F0E4FF02460548214611B042
:1080C000BDE8F04F04F0FEBA44200100BC190100E5
:1080D000C09EFF1F169CFF1F201801000900028090
:1080E00010B5424C424882B003F068FA2378C3B915
:1080F00006213F4804F050F92378012B37D90A2292
:10810000022B11463A486BD004F042F93949032258
:10811000374804F0D7FA364802B0BDE8104004F002
:10812000E7BA354B1A7801210523002A35D1019190
:10813000009311462E4803F0E9FD304B1A78002ACF
:1081400036D0052301220192009300220A212848FB
:1081500003F05AFD2A4B1A78002A35D10121052354
:10816000019100931421224803F0D0FDC0E7254C73
:108170002388092B32D9632B8CBF0A211F210A22A5
:108180001B4804F005F92188194804F001FB184840
:1081900002B0BDE8104004F0ABBA00220191009398
:1081A0001146134803F030FD144B1A78002AC8D149
:1081B00005230121019100930A210D4803F0A6FD3A
:1081C0000F4B1A78002AC9D001220523019200938F
:1081D00000221421064803F017FD89E73021CEE77D
:1081E00004F0D6F80322084992E700BF3B9FFF1F27
:1081F000C09EFF1F3C280100559EFF1F569EFF1F7B
:10820000579EFF1FDC9DFF1F38280100F8B56D4DFC
:10821000287840B96C4B1B6899425CD36B4A0123A8
:1082200013702B70F8BD0C4600266948664F03F0AA
:10823000C5F904F6AC53324665483B6031212E70D7
:1082400004F0A6F801216248624D04F0ABF8314613
:108250005F4804F0A1F805225F495D4804F032FA56
:108260005B4804F045FA0C221021594804F090F8BC
:108270000B225A49564804F025FA05225849544819
:1082800004F020FA524804F033FA564B50481C6868
:10829000A4F69803C3EB031385FB03251D441021AB
:1082A000DB172022C3EB652504F072F840F6CC33CF
:1082B0009C4205F124054FF022014FF004000BDC35
:1082C000FFF7E2FC484B1C88064674B3012C46D0ED
:1082D000022C41D00120F8BDFFF736FD09224349A9
:1082E0003B4804F0EFF92A221021394804F050F8F5
:1082F0003F4C374884FB0534EB17C3EBA4042146FD
:1083000004F046FA01223B49314804F0DBF904EB62
:108310008401A5EB41012E4804F03AFA01223649C6
:108320002B4804F0CFF90120F8BD34491022284829
:1083300004F0C8F9264804F0DBF92A221021244869
:1083400004F026F83146224804F022FA07222C498C
:108350001F4804F0B7F9CBE70C222A49E7E70C22C3
:1083600029491B4804F0AEF9194804F0C1F92A2242
:108370001021174804F00CF8314615481C4E04F043
:1083800007FA07221E49124804F09CF986FB0536BD
:10839000EB17C3EBA60631460D4804F0F9F9224667
:1083A00014490B4804F08EF906EB8601A5EB410158
:1083B000074804F0EDF922460F49054804F082F918
:1083C0002046F8BD108BFF1F3C9FFF1F389FFF1FEB
:1083D000C09EFF1F3B773B984028010048280100C2
:1083E00030280100309EFF1FA89DFF1F5428010068
:1083F00067666666882F0100F82E0100602801007C
:10840000742801008C2801007C2801002DE9F0412E
:10841000754C2278002A05460F4614BF4FF001081C
:108420004FF000084ED1714E3368CB1AB3F5FA6F96
:1084300004D86B78A3B94046BDE8F0816C4B6D4819
:108440006D49DFF8D0E11A700123037009882370A9
:1084500026208EF8002000F0F1FD6B78002BEAD08A
:108460003760F9F789FC654A654B664912782878C8
:108470001B78097802EB4303421E03EB81030E2AAB
:10848000D9D801A151F822F0798500004585000076
:1084900037840000798500003784000037840000AD
:1084A000378400002D85000037840000DF84000041
:1084B00037840000378400003784000037840000D0
:1084C000DB840000AF215048484E02F027FEFFF742
:1084D00007FE002337602370ABE705F00BFB4A482B
:1084E00003F06CF80221484803F056FF0F222321C5
:1084F000454803F04DFF05224449434804F0E2F8A3
:10850000414804F0F5F81E2223213F4803F040FFC4
:1085100005223F493C4804F0D5F83B4804F0E8F810
:10852000394803F057F900F0ADFC84E7394D2B785A
:10853000012B50D9304B2620198800F07FFD0023F5
:108540002B7078E7002B3FF476AF013B324A32F8CC
:108550001330002B3FF46FAF274C304825492D4A8C
:1085600023804FF001080023037081F8008082F817
:108570000080FFF7B5FD5EE793B1013B264A32F874
:10858000131019B31C4B254D1A4C224A1980002692
:10859000012326202E702370137000F04FFD15E08C
:1085A000154C1E4922880B7004284FF6FF7002F10B
:1085B000FF310CBF012202460A440E4E154D02F057
:1085C0007F0201320121228031702B70FFF788FD7C
:1085D0004FF001082FE70649064A012300200870E2
:1085E00013702370A6E700BF108BFF1F349FFF1F7F
:1085F000389FFF1F079CFF1FDC9DFF1F559EFF1F1D
:10860000569EFF1F579EFF1FC09EFF1F9C28010004
:10861000A42801003B9FFF1F889DFF1F789CFF1F20
:108620002DE9F04F05468BB00F46AD4801211646A7
:1086300003F0B8FEAA8812F0010440F0B080DFF821
:10864000CC8298F80030002B7DD1AB79A54AD15C63
:10865000A1B9DFF8BCA279781AF8039041B3397850
:108660000139072900F2B780DFE811F0F100540169
:10867000B5006C01B500B500B500E9007C78002CB0
:1086800000F0CA800139EC68387854F82170FC6831
:10869000411EB4F80080072900F2A780DFE811F03E
:1086A00074015901A5006C01A500A500A5009F005B
:1086B000DFF854A2DAF80020B21AB2F5967F75D925
:1086C000894A107801281ABF012010701170874A5A
:1086D00018BF0146D05CC0EB0900C0B2FFF704F937
:1086E0000124CAF80060AB889B0770D57B78002B0B
:1086F0006DD0F9F741FB7E4B7E4A7F481B7812789C
:1087000039780078022515FB02330A2903EB800330
:1087100000F04E810C295AD1002B58D003F11900DA
:10872000764E774A013B0021400080B226F81310B4
:108730000123157088F8003000F080FC714B032293
:1087400020461A702FE0664802F038FF0121644885
:1087500003F022FE62482246214603F019FEAB8850
:10876000580725D42C68204608F08AFC214602468A
:108770005B4803F0A7FF5A4803F0BAFF0922012320
:108780008DE80C0000217F23554803F06FFA00218B
:108790002846FFF707FB002388F8003055E7AB6851
:1087A0003146384698470BB0BDE8F08F0846FAE7E7
:1087B0002B6804A8984704A808F062FC04A90246A4
:1087C000474803F07FFF464803F092FFD6E7204674
:1087D0000BB0BDE8F08F00240AF8039083E7002176
:1087E000D1543846FB699847FC68A4F800800027FC
:1087F00025223C238DE8840041211822384803F0CB
:1088000003FAE968A879FFF7DFFB374A3E4B177098
:108810001E600BB0BDE8F08F3B490A68B21AB2F592
:10882000967FD4D9304F0E603E78012E00F0B48090
:10883000E968184601233B70FFF7C6FBB3E7304AEF
:10884000E9791170012288F800200024C4E72A7A0F
:10885000013A4A45BFDD09F10104E4B2A145BAD0AD
:10886000224E16F803B0CBEB0900C0B20021FFF78F
:108870003BF82B7A052BD9461BD9CBEB0402042AF3
:1088800040F3AE80A4F1040BBBF1000FC0F2B08046
:10889000063B5B45A8BF5B465FFA83F9AA7913489C
:1088A000B15C994205D000F8029001212846FFF7FB
:1088B00079FAC9EB0400C0B201210B4EFFF714F89E
:1088C00000213423019100930548317040230B228D
:1088D0003F21A14603F098F90124AB797CE700BF62
:1088E000C09EFF1F289FFF1F399FFF1FB89EFF1FBD
:1088F000559EFF1F569EFF1F579EFF1F889DFF1FFF
:10890000389FFF1F3B9FFF1F249FFF1F108BFF1FE0
:10891000A49EFF1F0FFA89F1E868604C50F82160AF
:108920002168049134785E4904980860002C71D065
:10893000012C7FF450AF5B4A317A88F80040117007
:10894000002449E7B9F1000F50D009F1FF34E4B237
:1089500084E7B98A01F0040189B200293FF440AFED
:108960003B6A03929847039A00283FF43DAFAB79E6
:10897000FC680021D15438E77B8A43453CD908F193
:1089800001081FFA88F830E73B8A43453BD208F1DB
:10899000FF381FFA88F828E725238DE81800424899
:1089A0003C703C231822412103F02EF93046FAE6B0
:1089B000002B3FF40CAF3D4A3D4E1188394A03F17C
:1089C0001900013B400080B226F81310012388F8FB
:1089D0000030157000F032FB364B20461D70E2E689
:1089E000002A3FF755AF04F1FF3B4DE74C46F3E655
:1089F0004FF000094B4651E7BB8ADA077FF5F5AE29
:108A0000B7F81080F1E6BB8AD9077FF5EEAEB7F86C
:108A10001280EAE62849C85CC0EB090009F1010EA2
:108A2000C0B201214FF0340B02F803E0FEF75CFF07
:108A3000B6681D48019440230B223F210124CDF844
:108A400000B003F0E1F840230B223F211648CDF897
:108A500000B0019403F05AF92146134803F09CFC3E
:108A6000304608F00DFBA0EB800000F15F0109B279
:108A70000F220D4803F08CFC304608F001FB314614
:108A80000246094803F01EFE074803F031FEE9687C
:108A9000A879FFF799FAAB799EE600BF7C9FFF1F8C
:108AA000249FFF1F389FFF1FC09EFF1FDC9DFF1FDD
:108AB000889DFF1F3B9FFF1FB89EFF1F2DE9F047BA
:108AC000DFF808926D4B99F800601B68DFF800A290
:108AD00082B0003601934FF0030018BF0126019FBA
:108AE0009AF8008004F0BEFC0546042004F0BAFCAD
:108AF0000446052004F0B6FC800040EA4404062049
:108B000004F0B0FC2C4364B25D4944EAC0000A782A
:108B100080F00F03DBB29A425A4A3CD01760002221
:108B200059480B7003788DF800808DF8012053B3FD
:108B3000564A12684EF66021BA1A8A4219D8022B98
:108B400059D0012B5FD0062B48D0032B63D0042BC8
:108B500069D0052B77D0072B7DD0082B00F08380C0
:108B6000092B68D016B14A4802F034FE02B0BDE8C5
:108B7000F087484A484C002301212370037013609A
:108B8000938089F800103A4669464448FFF748FD4B
:108B90003043C6B2E6E71268BA1A1E2A6BD99AF8B1
:108BA0000020934222D0394C3D488AF80030012BF6
:108BB000276082EA030207609846B1D0042BAFD148
:108BC00037480068381AB0F5C87FA9D9354C2068F5
:108BD000381A3228A4D927601A46A1E73A466946CE
:108BE0003148FFF71DFD3043C6B2BBE7012B4FF004
:108BF0000002E3D1E4E73A4669462C48FFF710FD4E
:108C00003043C6B2AEE73A4669462948FFF708FD49
:108C10003043C6B2A6E73A4669462648FFF700FD4C
:108C20003043C6B29EE73A4669462348FFF7F8FC50
:108C30003043C6B296E73A4669462048FFF7F0FC53
:108C40003043C6B28EE73A4669461D48FFF7E8FC56
:108C50003043C6B286E73A4669461A48FFF7E0FC59
:108C60003043C6B27EE73A4669461748FFF7D8FC5C
:108C70003043C6B276E7002252E700BF7C9FFF1F59
:108C8000409FFF1FAC9EFF1F389FFF1F309FFF1F9D
:108C9000C09EFF1F289FFF1F3A9FFF1FB0220100A9
:108CA000449FFF1FB49EFF1FE02601000822010021
:108CB0000C21010084200100482E0100FC2001004D
:108CC00064210100EC2101008490FF1F108BFF1F25
:108CD000B09EFF1F28B11028044BA8BF10201860B9
:108CE0007047024B01201860704700BF489FFF1F6C
:108CF00038B50F4D2B78013B01381B02C4B203F489
:108D00007063200443F4404343F00C0300F4FE007E
:108D1000184305F00FFD2868013860F03F00C0B22D
:108D200004F036FD2046BDE8384004F031BD00BFF8
:108D3000489FFF1F70B5124D2B78013B1B0203F4B7
:108D40007063064643F430430806320400F0FE40E8
:108D500043F00B03034302F4FE0018430C4605F0F6
:108D6000E9FC2868013860F04F00C0B204F010FD43
:108D7000304604F00DFD2046BDE8704004F008BD0B
:108D8000489FFF1F70B5124D2B78013B1B0203F467
:108D90007063064643F410430806320400F0FE40B8
:108DA00043F00903034302F4FE0018430C4605F0A8
:108DB000C1FC2868013860F06F00C0B204F0E8FC24
:108DC000304604F0E5FC2046BDE8704004F0E0BC0D
:108DD000489FFF1F38B5104D2B78013B1B0203F451
:108DE0007063044643F41043000443F0090300F4A5
:108DF000FE00184305F09EFC2868013860F06F0003
:108E0000C0B204F0C5FC204604F0C2FC0020BDE85E
:108E1000384004F0BDBC00BF489FFF1F38B50E4D61
:108E20002B78013B1B0203F47063044643F4504368
:108E3000000443F00D0300F4FE00184305F07AFC33
:108E40002868013860F02F00C0B204F0A1FC204671
:108E5000BDE8384004F09CBC489FFF1F08B50020C7
:108E600005F032FD0028FAD108BD00BF08B5642125
:108E70000720FFF75FFF7F210B20BDE80840FFF7C9
:108E800059BF00BF10B500217B20FFF753FF00241E
:108E9000E0B2FFF79FFF0134022004F019FB802CA1
:108EA000F6D110BD10B504464FF4406004F020FC2C
:108EB00004F078FC2CB1102C044BA8BF10241C60CB
:108EC00010BD024B01241C6010BD00BF489FFF1F56
:108ED00010B5044641F0E00004F05AFC04F07F00B5
:108EE00004F056FCC4F3C610BDE8104004F050BCBA
:108EF00038B5134D2B78044641F6FF72A0F50050AB
:108F0000824203F1FF33A8BF02461B0202F5005262
:108F100003F47063100443F4604343F00E0300F461
:108F2000FE005204184302F0FE42104305F002FC1A
:108F3000296801392046C9B2BDE83840FFF7C8BFEB
:108F4000489FFF1F38B504460D46F02004F020FC72
:108F500035B1254414F8010B04F01AFCAC42F9D1E8
:108F6000F720BDE8384004F013BC00BF00B50B4B40
:108F700083B00246998818680090032AADF804105F
:108F800002D903B05DF804FB684606218DF8052080
:108F9000FFF7D8FF03B05DF804FB00BFB82E010057
:108FA00000B50B4B024683B0186899880090131FD8
:108FB0004C2BADF8041002D903B05DF804FB6846F1
:108FC00006218DF80520FFF7BDFF03B05DF804FB17
:108FD000C02E0100030203F4FE43C0F3C610184381
:108FE000704700BF03784078DB0103F47E5300F044
:108FF0007F001843704700BF82B002AA114642F8B2
:10900000040D002012F8013B03F07F03914243EA74
:109010000020F7D102B07047003210B403884FF03F
:10902000010404FA01F418BF012202FA01F123EA53
:1090300004020A43028010BC704700BF70B5CEB274
:109040000C46054603F0D6FD864203D0314628463D
:1090500003F0EAFD0135284603F0CCFD240A8442E2
:1090600005D021462846BDE8704003F0DDBD70BD47
:1090700038B5054603F0BEFD4FF0000460F3070469
:10908000681C03F0B7FD60F30F24A0B238BD00BF29
:10909000F8B504460020FFF7EBFF002C00F01B851D
:1090A0004FF4AF610220FFF7C9FF4FF47A6104204B
:1090B000FFF7C4FF4FF496610620FFF7BFFF4FF4A0
:1090C000FA610820FFF7BAFF4FF4FA610A20FFF7B0
:1090D000B5FF40F6B8310C20FFF7B0FF4FF42F6119
:1090E0002220FFF7ABFF40F6AC512420FFF7A6FF8C
:1090F0007D212A20FFF7A2FF0C210E20FFF79EFF03
:1091000001211020FFF79AFF02211220FFF796FF9E
:1091100000211420FFF792FF00211620FFF78EFF99
:1091200002211820FFF78AFF01211A20FFF786FF8E
:1091300001211C20FFF782FF04211E20FFF77EFF84
:1091400014212020FFF77AFF01212620FFF776FF68
:1091500003212820FFF772FF04212C20FFF76EFF68
:1091600014212E20FFF76AFF00213020FFF766FF51
:109170000C213220FFF762FF00213420FFF75EFF51
:1091800000213620FFF75AFF00213820FFF756FF55
:1091900000213A20FFF752FF00213C20FFF74EFF4D
:1091A00000213E20FFF74AFF00214020FFF746FF45
:1091B00000214220FFF742FF1F214420FFF73EFF1E
:1091C00013214620FFF73AFF0E214820FFF736FF14
:1091D00011214A20FFF732FF0A214C20FFF72EFF12
:1091E00000214E20FFF72AFF06215020FFF726FF1F
:1091F00002215220FFF722FF0C215420FFF71EFF0F
:1092000000215620FFF71AFF00215820FFF716FF14
:1092100001215A20FFF712FF08215C20FFF70EFF03
:109220000A215E20FFF70AFF00216020FFF706FFFA
:1092300004216220FFF702FF01216420FFF7FEFEF8
:1092400000216620FFF7FAFE0B216820FFF7F6FEEB
:109250007F216A20FFF7F2FE00216C20FFF7EEFE6F
:1092600000216E20FFF7EAFE00217020FFF7E6FEE6
:1092700000217220FFF7E2FE00217420FFF7DEFEDE
:109280001F217620FFF7DAFE13217820FFF7D6FEA4
:109290000E217A20FFF7D2FE11217C20FFF7CEFEAF
:1092A0000A217E20FFF7CAFE1F218020FFF7C6FE9D
:1092B00013218220FFF7C2FE0E218420FFF7BEFE9D
:1092C00011218620FFF7BAFE0A218820FFF7B6FE9B
:1092D00000218A20FFF7B2FE00218C20FFF7AEFEAE
:1092E00000219620FFF7AAFE00219820FFF7A6FE96
:1092F00000219A20FFF7A2FE05219C20FFF79EFE89
:1093000006219E20FFF79AFE0021A020FFF796FE7F
:1093100027210020FFF792FE0220FFF7A9FEB0F5FB
:10932000805F034680F04785D24A04201380FFF710
:109330009FFEB0F5805F034680F03485CE4A06205C
:109340001380FFF795FEA0F52F739BB2B3F57A6FEC
:10935000024606D940F628210620FFF76FFE40F6A8
:109360002822C64B08201A80FFF782FEA0F52F7333
:109370009BB2B3F57A6F024606D940F6E441082065
:10938000FFF75CFE40F6E442BD4B0A201A80FFF76F
:109390006FFEA0F5FA739BB240F6AC518B420246C9
:1093A00006D94FF4FA610A20FFF748FE4FF4FA623B
:1093B000B44B0C201A80FFF75BFEA0F5FA739BB24A
:1093C00040F6AC518B42024606D940F6B8310C202B
:1093D000FFF734FE40F6B832AB4B0E201A80FFF791
:1093E00047FE1828034600F2D684A84A10201380AE
:1093F000FFF73EFE431E9BB20F2B024604D901210C
:109400001020FFF71BFE0122A14B12201A80FFF74C
:109410002FFE0A28034600F2B7849E4A14201380C8
:10942000FFF726FE0128034604D900211420FFF788
:1094300005FE0023984A16201380FFF719FE7F28A7
:10944000034600F29A84954A18201380FFF710FE15
:109450000428034600F28A84914A1A201380FFF7F9
:1094600007FE0C28034600F27A848E4A1C201380E3
:10947000FFF7FEFD0428034600F26A848A4A1E2094
:109480001380FFF7F5FD0928034600F25A84874A46
:1094900020201380FFF7ECFD4628034600F24A84A3
:1094A000834A22201380FFF7E3FDA0F5FA739BB2F5
:1094B00040F6AC518B42024606D94FF42F61222070
:1094C000FFF7BCFD4FF42F627A4B24201A80FFF780
:1094D000CFFDA0F5FA739BB240F6AC54A34202460E
:1094E00004D921462420FFF7A9FD2246724B2620ED
:1094F0001A80FFF7BDFD7F28034600F214846F4AEF
:1095000028201380FFF7B4FD0628034600F20484E8
:109510006B4A2A201380FFF7ABFDA0F132039BB208
:10952000B3F5967F024604D97D212A20FFF786FDF8
:109530007D22644B2C201A80FFF79AFD0C280346ED
:1095400000F2E483604A2E201380FFF791FD1E286D
:10955000034600F2D5835D4A30201380FFF788FD73
:109560000928034600F2C683594A32201380FFF7C8
:109570007FFD1E28034600F2B783564A342013802D
:10958000FFF776FD7F28034600F2A883524C362071
:109590002380FFF76DFD7F28034600F29983382072
:1095A0006380FFF765FD7F28034600F28B833A2036
:1095B000A380FFF75DFD7F28034600F27D833C20FA
:1095C000E380FFF755FD7F28034600F26F833E20BE
:1095D0002381FFF74DFD7F28034600F26183402081
:1095E0006381FFF745FD7F28034600F25383422045
:1095F000A381FFF73DFD394D28804420FFF738FD5A
:109600003028034600F24083354A46201380FFF796
:109610002FFD3028034600F23183324C482023804E
:10962000FFF726FD3028034600F222834A2063809C
:10963000FFF71EFD3028034600F214834C20A38060
:10964000FFF716FD3028034600F206834E20E38024
:10965000FFF70EFD0128034604D900214E20FFF735
:10966000EDFC0023204A50201380FFF701FD431E2C
:109670003CE000BFB09CFF1F6A9EFF1F669CFF1F5F
:10968000449EFF1F149EFF1F2C9CFF1F009CFF1F6A
:10969000CC9DFF1F049EFF1FA29CFF1F049CFF1F69
:1096A000B49CFF1F4E9CFF1F469CFF1F349CFF1F56
:1096B000509EFF1FC49DFF1FC09DFF1FDC9DFF1F0D
:1096C000209EFF1F649EFF1F169CFF1F9C9CFF1F78
:1096D000749EFF1F469EFF1F889DFF1F249CFF1F37
:1096E000269CFF1F249EFF1F449CFF1F9BB20B2B39
:1096F000024604D906215020FFF7A0FC0622CE4BDB
:1097000052201A80FFF7B4FC0428034600F29E8220
:10971000CA4A54201380FFF7ABFC431E9BB21D2B9B
:10972000024604D90C215420FFF788FC0C22C44BBC
:1097300056201A80FFF79CFC0128034604D900211B
:109740005620FFF77BFC0023BE4A58201380FFF70A
:109750008FFC7F28034600F27382BB4A5A20138095
:10976000FFF786FC431E9BB2092B024604D9012158
:109770005A20FFF763FC0122B44B5C201A80FFF7EC
:1097800077FC431E9BB2102B024604D908215C20B3
:10979000FFF754FC0822AE4B5E201A80FFF768FCEE
:1097A000431E9BB21D2B024604D90A215E20FFF7FF
:1097B00045FC0A22A74B60201A80FFF759FC0228BB
:1097C000034600F23782A44A64201380FFF750FC5E
:1097D0000128034604D901216420FFF72FFC01234F
:1097E0009E4A62201380FFF743FCC31E9BB2012BED
:1097F000024604D904216220FFF720FC0422984B82
:1098000066201A80FFF734FC7F28034600F20C82A2
:10981000944A68201380FFF72BFC7F28034600F250
:10982000FD81914A6A201380FFF722FC7F280346BE
:1098300000F2EE818D4A6C201380FFF719FC04289A
:10984000034600F2DF818A4A6E201380FFF710FC86
:109850001928034600F2D081864A70201380FFF752
:1098600007FC0228034600F2C181834A722013805C
:10987000FFF7FEFB0628034600F2B2817F4A742000
:109880001380FFF7F5FB0428034600F2A3817C4A0E
:109890008A201380FFF7ECFB0A28034600F294812C
:1098A000784A8C201380FFF7E3FB0428034600F27C
:1098B0008581754A98201380FFF7DAFB012803465B
:1098C00004D900219820FFF7B9FB00236F4A9A20A2
:1098D0001380FFF7CDFB0128034604D900219A200D
:1098E000FFF7ACFB00236A4A96201380FFF7C0FB0A
:1098F0000B28034600F25C81664A9C201380FFF728
:10990000B7FB831E9BB2032B024604D905219C2082
:10991000FFF794FB0522604B76201A80FFF7A8FB27
:109920003028034600F23E815C4A78201380FFF71E
:109930009FFB3028034600F22F81594C7A20238068
:10994000FFF796FB3028034600F220817C206380DD
:10995000FFF78EFB3028034600F212817E20A380A1
:10996000FFF786FB3028034600F204818020E38065
:10997000FFF77EFB3028034600F2F680494A82203A
:109980001380FFF775FB3028034600F2E780464C52
:1099900084202380FFF76CFB3028034600F2D88038
:1099A00086206380FFF764FB3028034600F2CA80FC
:1099B0008820A380FFF75CFB3028034600F2BC80C0
:1099C000A020E380FFF754FB0128034604D90021BF
:1099D000A020FFF733FB0023344A9E201380FFF7BB
:1099E00047FBC31E9BB20C2B04D99E200621FFF718
:1099F00025FB06202B88DFF8D4E02D4F2D4A2E4D75
:109A00002E4E2F4C2F4903F0010CAEF800C0C3F3CB
:109A1000400EA7F800E0C3F380071780C3F3C00728
:109A2000294A2F70C3F30017C3F34015C3F3801303
:109A3000378025804CE000BF148AFF1F5E89FF1F1E
:109A4000168AFF1F8E9CFF1F129EFF1FFC9BFF1F8D
:109A5000648AFF1F5C89FF1FBC9DFF1F1C9EFF1FA8
:109A6000549CFF1F529EFF1F809CFF1F389CFF1FAE
:109A7000F09BFF1F969EFF1FA89DFF1F709EFF1F5C
:109A80003C9EFF1FCE9DFF1FB69DFF1F369CFF1FF4
:109A9000949CFF1F0C9EFF1F1A9CFF1F2E9CFF1FF4
:109AA000989DFF1F309CFF1FA09DFF1F8C9EFF1FD6
:109AB000649CFF1F9E9CFF1FAC9DFF1FBE9DFF1F50
:109AC0001E9EFF1FD29DFF1FC089FF1F0E9EFF1FFE
:109AD0000B801080F8BD4FF6FF7398423FF4E0AA68
:109AE00027283FF419AC17287FF6DAAA19287FF641
:109AF00043AB1B287FF660AB1C283FF475AB1E28D8
:109B00007FF67AAB1F283FF47FAB20283FF498AB59
:109B100021283FF4A1AB22283FF4A6AB23283FF431
:109B2000AFAB24283FF4E0AB25283FF4E5AB262873
:109B30007FF4EEABFFF7E4BB0A218820FFF77EFA43
:109B40000A233DE711218620FFF778FA11232FE73A
:109B50000E218420FFF772FA0E2321E713218220C1
:109B6000FFF76CFA132312E71F218020FFF766FA34
:109B70001F2303E70A217E20FFF760FA0A23F5E698
:109B800011217C20FFF75AFA1123E7E60E217A20F3
:109B9000FFF754FA0E23D9E613217820FFF74EFA87
:109BA0001323CAE61F217620FFF748FA1F23BBE6DE
:109BB00000219620FFF742FA00239DE600218C2029
:109BC000FFF73CFA002374E600218A20FFF736FAFB
:109BD000002365E600217420FFF730FA002356E6E3
:109BE00000217220FFF72AFA002347E600217020A7
:109BF000FFF724FA002338E600216E20FFF71EFA53
:109C0000002329E600216C20FFF718FA00231AE64A
:109C10007F216A20FFF712FA7F230BE60B216820D1
:109C2000FFF70CFA0B23FCE500216620FFF706FA8C
:109C30000023EDE500216020FFF700FA0023C2E5D4
:109C400000215820FFF7FAF9002386E5022152206F
:109C5000FFF7F4F902235BE50A214C20FFF7EEF948
:109C60000A23F3E411214A20FFF7E8F91123E5E480
:109C70000E214820FFF7E2F90E23D7E413214620F6
:109C8000FFF7DCF91323C8E41F214420FFF7D6F9BE
:109C90001F23B9E400214020FFF7D0F90023A6E4F8
:109CA00000213E20FFF7CAF9002398E400213C2060
:109CB000FFF7C4F900238AE400213A20FFF7BEF938
:109CC00000237CE400213820FFF7B8F900236EE47C
:109CD00000213620FFF7B2F9002360E40021342090
:109CE000FFF7ACF9002351E40C213220FFF7A6F96D
:109CF0000C2342E400213020FFF7A0F9002333E4D5
:109D000014212E20FFF79AF9142324E404212C2097
:109D1000FFF794F9042315E403212820FFF78EF9B7
:109D20000323FFF7F5BB01212620FFF787F9012365
:109D3000FFF7E5BB14212020FFF780F91423FFF77C
:109D4000AFBB04211E20FFF779F90423FFF79FBB67
:109D500001211C20FFF772F90123FFF78FBB0121BE
:109D60001A20FFF76BF90123FFF77FBB02211820B0
:109D7000FFF764F90223FFF76FBB00211620FFF7FE
:109D80005DF90023FFF75FBB02211220FFF756F9B0
:109D90000223FFF742BB0C210E20FFF74FF90C23E3
:109DA000FFF723BB4FF47A610420FFF747F94FF424
:109DB0007A63FFF7C3BA4FF4AF610220FFF73EF9B1
:109DC0004FF4AF63FFF7B0BAF8B5B32006F0C8FBA5
:109DD000204B214A054603CB1368C5F803001A0C33
:109DE000A220C5F807102B80AA70FFF7F3F82E46C3
:109DF000002426F80B0FA0B2FFF73AF9FFF7EAF8B4
:109E00000234A22C26F8020FF5D16C1E05F1AE0625
:109E10004FF0FF3014F8013F082758400F4B40F334
:109E200000017A1E0B4012F0FF0783EA5000F5D1C3
:109E3000B442EFD1C043FFF7DFF83A46C5F8AF00B0
:109E4000B321284604F0C4FC2846BDE8F84006F0DB
:109E50008FBB00BFCC2E0100C82E01002083B8EDBF
:109E6000F0B50E4B0E4C054693E8070085B024680C
:109E70002E88AD7801AB83E80700270C1846002236
:109E80000B21ADF804408DF80670ADF80C608DF82C
:109E90000E5004F09DFC05B0F0BD00BFD82E0100AF
:109EA000C82E0100F0B5124B124D1E68124F0FCD97
:109EB00087B06C460FC495E8030044F8040B38687B
:109EC0003B79CDF80D00320C272021808DF802203F
:109ED0008DF81130ADF80060FFF77CF80022ADF886
:109EE0000B001221684604F073FC07B0F0BD00BF00
:109EF000C82E0100E42E010030280100002004F0EB
:109F0000E3BC00BF02F02EBE70B5124C82B000253B
:109F100040230646294620460093019580232022AF
:109F200001F072FE20222946204602F031FA204636
:109F3000012102F037FA304607F0A2F83146024616
:109F4000204602F0BFFB204602B0BDE8704001F0A1
:109F500041BC00BFC09EFF1FF0B5B22983B075D9C8
:109F60000546441E00F1AE064FF0FF3014F8012FF5
:109F700008275040404A40F300017B1E0A4013F07E
:109F8000FF0782EA5000F5D1B442EFD1C043FFF79A
:109F900033F80146D5F8AF000190019A914202D002
:109FA000B2F17F2F0BD105F10B00FFF71BF8A228B0
:109FB0000BD03248FFF7A8FF002003B0F0BD3048B7
:109FC000FFF7A2FF384603B0F0BD05F10D00FFF723
:109FD00009F8272840D1002440F6AC5613E00428A5
:109FE0001AD0062821D008281FD00A2828D00C28EB
:109FF00022D1A1F5FA7292B2B24201D8FFF71EF84F
:10A000000234A22C0ED004F10D002844FEF7EAFF22
:10A01000022C0146A0B2E2D1B1F5805FEED302344A
:10A02000A22CF0D1012003B0F0BDA1F52F7292B2A5
:10A03000B2F57A6FE4D8E1E7222801D0242811D1C3
:10A04000A1F5FA7292B2B242DAD8D7E70D48FFF71B
:10A050005BFF002003B0F0BD0B48FFF755FF002069
:10A0600003B0F0BD2A28C9D1A1F1320292B2B2F5F3
:10A07000967FC5D8C2E700BF2083B8ED282F010026
:10A08000142F0100FC2E01003C2F010003290CD9E4
:10A0900070B5461C82B005460C46304603222A495C
:10A0A00007F05CF810B102B070BD70470B2C05D9F9
:10A0B00005222649281D07F051F840B12448FFF732
:10A0C00023FF244802B0BDE87040FFF7C9BE05F188
:10A0D0000901032201A807F091F801A803221E49F3
:10A0E00007F03CF8D8B103221C4901A807F036F864
:10A0F00008B301A803221A4907F030F8B0B919488B
:10A10000FFF702FFA11E89B23046FFF725FF0028A6
:10A11000C9D0154802B0BDE87040FFF7F5BE13483E
:10A12000FFF7F2FEFFF750FE1148F3E71148FFF783
:10A13000EBFE1148C6E71148FFF7E6FE02B0BDE8A6
:10A140007040FFF7AFBE00BFC82E0100542F0100C2
:10A150005C2F0100702F0100742F01009C2F010063
:10A16000B42F0100B82F0100CC2F0100782F01007F
:10A170008C2F0100E02F0100F42F0100A02F01001F
:10A180002DE9F043174D2B6883B081460F4690466A
:10A19000F3B1154E34880A1992B21846114632802E
:10A1A00006F05CFD28603A464946204402F06CFD0A
:10A1B000B8F1000F09D031882868FFF767FF2868D9
:10A1C00006F0D6F900232B60338003B0BDE8F0839E
:10A1D000054E01930846318006F0C2F9019B2860C4
:10A1E0001C46E0E7509FFF1F4C9FFF1F10B51F4C00
:10A1F0004FF4FA70FCF776F8204601F0DFF9002200
:10A200001146204602F0C4F82046012102F0CAF8A7
:10A210002046002102F0C0F80B221549204602F02A
:10A2200051FA204602F064FA0F221249204602F049
:10A2300049FA204602F05CFA0F490722204602F054
:10A2400041FA204602F054FA204601F0C3FA0B4BC3
:10A250000B4A1A604FF4FA70FCF744F8FFF722FE3D
:10A260000848BDE81040FFF74FBE00BFC09EFF1F6B
:10A27000F82F0100043001001430010008A1FF1F75
:10A2800081A100001C3001000020704790F83920A7
:10A2900090F83800101A704790F8383090F839204C
:10A2A0009A4205D95A1C034480F83820187E70471A
:10A2B0004FF0FF30704700BF90F8383090F83920E9
:10A2C0009A4286BF1B18187E4FF0FF30704700BFC0
:10A2D000704700BF38B50546B0F85E0090B195F8FC
:10A2E0005D301446C3F1210294420CD805F13B00C5
:10A2F0001844224602F0C8FC95F85D30234485F8E6
:10A300005D30204638BD012014462871EEE700BFBD
:10A31000B0F85E306BB190F85D30202B07D8C218D2
:10A32000013380F85D30012082F83B107047012333
:10A3300003710020704700BF0023426980F8383065
:10A3400080F8393080F85C3080F85D3080F85E301D
:10A3500080F85F3006CA30B40D68046943662A434A
:10A3600083660A60A370426990F8613016491468E8
:10A3700013441D7A5B7B01EBC5051B026D6803F47A
:10A38000E06343F064032B6090F8623013449D7CDB
:10A39000DB7D01EBC5011B02496803F4E06343F078
:10A3A00064030B6021685368194205D003692722B2
:10A3B0005A70036904229A71036920225A71036951
:10A3C00080229A7030BC7047503B010043690CCB2F
:10A3D00012681A420CD0094B99420AD9084B99428B
:10A3E000036994BF1A220D225A70036904229A71DC
:10A3F0007047036927225A70F7E700BF7F1A0600EB
:10A400003F420F0010B50269D378DBB2D90604468B
:10A410003DD510215806D17038D503F0040303F060
:10A42000FF02002B51D03D49626E00230B7084F86F
:10A430005D30002A5BD0904794F85D30002B56D0F9
:10A440002369D0229A70236994F83B201A712369FA
:10A45000012284F85C200222DA7010BD304B84F8AF
:10A4600060009C424AD02F4B9C4252D094F8391045
:10A4700013791F29DBB207D82848007820B160186B
:10A48000013184F8391003760223D37010BD5906C8
:10A49000C3D4917801F0100101F0FF000029DDD054
:10A4A00013F001031ED194F85C1094F85D0088420B
:10A4B00081BF4B1C091984F85C3091F83B30137153
:10A4C0002369D0229A702269DEE7236984F8392053
:10A4D000C0229A702369114A197901211170022250
:10A4E000DA7010BDC023937022691379CCE7012282
:10A4F000002384F85D2084F83B30A1E7626994F87A
:10A500006130094913440322187A02F043FD22699D
:10A51000ACE7626994F861300449F3E7549FFF1F88
:10A52000D090FF1F3C91FF1F8DA5000099A5000052
:10A530000369DB7803F0200373B190F860300133D6
:10A54000DBB2012B80F860301AD9426990F8613093
:10A550001344187A02F09ABD70B5426903F0FF0502
:10A5600090F8613013440446187A02F08FFDA36E10
:10A570005BB184F8385094F83900BDE87040184752
:10A5800090F85F30002BE0D0704770BD0148FFF7B6
:10A59000CFBF00BFD090FF1F0148FFF7C9BF00BF6A
:10A5A0003C91FF1F2DE9F047374FDFF8E0903B6803
:10A5B000026982B006460093DDF800800021A025E4
:10A5C000D3789B065BD53B680193019BC8EB0303E3
:10A5D0000F2BF5D949B1102BF2D0002090703369C0
:10A5E00080229A7002B0BDE8F087726996F86130F7
:10A5F00013440521187A02F043FF726996F861301E
:10A600001344012193F812A0504602F039FF0924A7
:10A610000021504602F020FF2B46013BFDD10121D5
:10A62000504602F019FF2B46013BFDD1013CEFD112
:10A63000706996F8611001444FF4A0720C7A4B7B5C
:10A6400009EBC4011B02496803F4E06343F06403AF
:10A650000B6096F862300344997CDB7D09EBC10105
:10A660001B02496803F4E06343F064030B60013AA2
:10A67000FDD13269D3789B064FF00101A3D40120AC
:10A6800002B0BDE8F08700BF7C9FFF1F503B010078
:10A69000F0B503691222DA700269937803F020039F
:10A6A00085B004460D46002B5ED0B42393703C4920
:10A6B00022690B680093009E05E00B680193019BE3
:10A6C0009B1B042B42D8D37803F0200303F0FF0038
:10A6D000002BF2D094F85D30002B31D04FF0000EFB
:10A6E0004FF0020C04EB0E0393F83B3013710B6830
:10A6F0000393039F206907E09B060DD50B68029327
:10A70000029BDB1B052B28D8C378DBB203F00202C7
:10A7100002F0FF06002AEFD080F803C02669F37824
:10A72000DBB2DF0632462DD49F062BD5DB0731D4B2
:10A730000EF1010E94F85D305FFA8EFE7345D1D8AC
:10A7400000201DBB002384F85E3004E09070236974
:10A7500080229A70042005B0F0BD867023698022A3
:10A7600004209A7005B0F0BD03F0FF06FFF71AFF52
:10A7700010B9042005B0F0BD236984F85F60B022F1
:10A780009A7094E78023B3700420DAE72669802367
:10A79000B370D7E7BEF1000F0CBF02200320F6E72D
:10A7A0007C9FFF1F2DE9F04106690025122780F8E4
:10A7B000385080F83950F770D0F810C09CF802E09B
:10A7C0000EF0200E88B00446884615461E46BEF19F
:10A7D000000F49D0B4238CF80230784B21691A68F5
:10A7E0000092DDF800E006E01A6801920198CEEBD5
:10A7F0000000042830D8C87800F0200000F0FF07DF
:10A800000028F1D04FEA480242F00102D2B20A71A8
:10A810001A680292DDF808E0206906E01A680392DF
:10A820000399CEEB010105292AD8C17801F0020174
:10A8300001F0FF070029F1D04FF0020C80F803C0AF
:10A840002269D17811F0110722D12DBB002E0CBF47
:10A85000A0238023937003E08F70236980229A7075
:10A86000384608B0BDE8F0810EF0FF07FFF79AFE0A
:10A870000028F5D0236984F85F70B0229A70ACE7A5
:10A8800087702369802238469A7008B0BDE8F0814D
:10A89000802393700027E3E7012D75D0A0219170EC
:10A8A00021690A79BE4667464FF0A80C1A680492DF
:10A8B000049805E01A680592059A121A052A4AD8E2
:10A8C000CA7802F0020202F0FF08002AF2D0CF702C
:10A8D0002169CA78D2B212F0100F08465AD19206F6
:10A8E00058D5013DEDB2012D49D0BEF11F0F3BD926
:10A8F0000A79012DDAD11A680692069D05E01A68D8
:10A900000792079A521B052A46D8C27802F0020223
:10A9100002F0FF01002AF2D00223C3702269D3782B
:10A92000DBB2D9063AD49B0634D5B023BEF11F0F53
:10A9300093703FD8226904EB0E0312791A760EF158
:10A94000010E5FFA8EFE16B1236980229A7084F898
:10A9500039E0774684E781F80280236980229A7083
:10A96000774684F839E07BE704EB0E0291F8048027
:10A9700082F818800EF1010E5FFA8EFEB9E781F8B9
:10A9800002C021690846B0E7A82191702069BE463F
:10A990000279B0E7774663E78170DEE71021A023F4
:10A9A000D170013BFDD12269937803F0F70377461C
:10A9B000937055E723691B79C5E700BF7C9FFF1F94
:10A9C0000148FFF71FBD00BFD090FF1F0148FFF7F0
:10A9D00019BD00BF3C91FF1F704700BF38B5144C34
:10A9E000037801225B000546204684F83B3084F85A
:10A9F0005E2084F85D20FFF78BFC20460021FFF7E6
:10AA000047FE0B4C2978012320461A46FFF7CAFE61
:10AA10000128F6D194F8383094F839209A4205D9B3
:10AA2000E218013384F83830107E38BDFF2038BD7D
:10AA3000D090FF1F38B51B4C037801225B00054600
:10AA4000204684F83B3084F85E2084F85D20FFF7D0
:10AA50005FFC20460021FFF71BFE124C29782046A0
:10AA600001230222FFF79EFE0228F6D194F8382037
:10AA700094F839108A420FD2531CDBB2A0189942C5
:10AA800084F83830007E0AD9234402321B7E84F8D1
:10AA9000382040EA032038BD4FF6FF7038BD40F43F
:10AAA0007F4038BDD090FF1F0C2901D9002070478E
:10AAB0000231490001F0FE01FFF7BCBF70B50C4C3C
:10AAC0000378164601255B00204684F83B3084F865
:10AAD0005E5084F85D50FFF71BFC31462046FFF7BF
:10AAE00017FC29462046BDE87040FFF7D1BD00BFE6
:10AAF000D090FF1FF8B505460F4616464124214663
:10AB00003A462846FFF7DAFF611C0234C9B23246E2
:10AB10002846E4B2FFF7D2FF592CF0D1F8BD00BFB0
:10AB200038B504460D463548FFF706FC6322802100
:10AB300020462570FFF7C2FF012002F0C9FC204625
:10AB400000225E21FFF7BAFF20465D21FFF746FF96
:10AB5000242801D0002038BD204606220C21FFF712
:10AB6000C9FF204601222B21FFF7A8FF2046012222
:10AB70002C21FFF7A3FF20460E222D21FFF79EFF79
:10AB8000204600222E21FFF799FF204601222F2187
:10AB9000FFF794FF204605223021FFF78FFF204664
:10ABA00001223121FFF78AFF204600223221FFF7E0
:10ABB00085FF204600223321FFF780FF2046002238
:10ABC0003421FFF77BFF204600223521FFF776FF77
:10ABD000204600225B21FFF771FF204610225C21F6
:10ABE000FFF76CFF204620225D21FFF767FF20461C
:10ABF0008F225E21FFF762FF012038BDD090FF1F3A
:10AC000010B4047F4160022CC26002D010BC01F07D
:10AC1000D7BB836810BC184790E80C00F0B41C68E0
:10AC200059682568164F174E29432160164D17495C
:10AC30001760D66015611160417A154A5C180A31B7
:10AC400094F8244053F8215002EBC40149680D6088
:10AC5000017A5C1803EB8101247ECD6902EBC4010B
:10AC600049680D60817A581803EB810390F8300031
:10AC7000596B02EBC002F0BC53681960704700BF0B
:10AC800001401F00011000380110007800001F80F3
:10AC9000503B0100704700BFF0B50C1EBDF81460BA
:10ACA00034DBB0F906701919B942C4BF3B1B1BB2A3
:10ACB000002BA6461CDD002A1146B8BFD11D02F0AC
:10ACC0000705CC10826A012007FB04E1A840012E91
:10ACD0000A44C0B21ED00CD3022E09D1013B12FA95
:10ACE00083F3013A12F8011F41409A421170F9D1E1
:10ACF000F0BDC043013B12FA83F3C0B2013A12F82F
:10AD0000011F014093421170F9D1F0BD23441BB2E1
:10AD10000024C6E7013B12FA83F3013A12F8011F3F
:10AD200001439A421170F9D1F0BD00BFF8B50D1E74
:10AD30000EDB14461F46064601F03AFBA84207DD2B
:10AD4000002C05DB304601F037FBA04201DCF8BDEA
:10AD5000F8BD304601F02AFB022853D003284BD01F
:10AD6000012806D16540F3886C406540013B5D1BBE
:10AD70002DB2012F03D02AD3022F14D0F8BD002CFE
:10AD80002246B6F90630B06AB8BFE21D42F3CF02E0
:10AD900002FB035504F00704435D012101FA04F4AA
:10ADA0001C434455F8BD002C2246B6F90630B06A63
:10ADB000B8BFE21D42F3CF0202FB035504F00704C3
:10ADC000435D012101FA04F45C404455F8BD002CB8
:10ADD0002246B6F90630B06AB8BFE21D42F3CF0290
:10ADE00002FB035504F00704435D012101FA04F45A
:10ADF00023EA04044455F8BD3389013B591B254619
:10AE00000CB2B6E7F18832890139013A4D1B141BA7
:10AE10002DB224B2ADE700BF2DE9F041079E9DF9A8
:10AE20001880089D04461F4600F0C0FF0D4B0E48D9
:10AE30000E4984F83380FF22002F08BF1F4684F894
:10AE40002F20002384F8302084F8312084F8322029
:10AE50002060A665E565676261652362A36220469E
:10AE6000BDE8F081D090FF1FA8300100011001382B
:10AE700010B50446806A034B236008B105F078FBE7
:10AE8000204610BDA8300100F8B5436ADBB190F848
:10AE90002C200125AA4083F83B2083F85E5083F8DC
:10AEA0005D500446406A03680E461B6800219847BF
:10AEB000606A036831461B6898472946606ABDE8A6
:10AEC000F840FFF7E5BBC26BC56C1368046A23EA60
:10AED000050313604CB122684FF00043D362516305
:10AEE000D36A002BFCDA936BF8BD836B466B0825A5
:10AEF000802410E03768426C3A4332601F68826CED
:10AF00003A431A601A68876C013D22EA07024FEA49
:10AF100054041A6007D02142ECD13268476C22EA0F
:10AF200007023260EAE7F8BD70B50446406A0D4694
:10AF300000282BD0A16DFFF749FA002D20460CBF49
:10AF4000A621A721FFF7A0FF606A20B1E16DBDE84F
:10AF50007040FFF73BBA216C226D0868236A0243F8
:10AF60000A6093B1DA7A82B1D00703D5224A99698F
:10AF70001160DA7A910703D5204AD9691160DA7A2B
:10AF8000520702D51E4A1B6A136070BD236A002B4C
:10AF90002BD0D97A626DE1B172B6D97ACE0706D5D7
:10AFA0001848D9680668314099610160D97A8807E4
:10AFB00006D51548196906683140D9610160D97A0A
:10AFC0004E0705D51148596906683140196201607C
:10AFD00062B61B68D968914207D00D4818600D49C8
:10AFE000DA6042F0804018611960226C216D1368AC
:10AFF00023EA01031360A0E700E100E004E100E0C0
:10B0000008E100E080E100E084E100E088E100E0A8
:10B0100001403F0000003F80436A2DE9F0410546B2
:10B020000E469046002B3ED090F82C100124A140F3
:10B0300083F83B1083F85E4083F85D40406A036804
:10B0400000211B6808F1FF379847FFB2B8F1000FE5
:10B0500023D03744A046013E686A16F8011F0368F2
:10B060001B6898470134B742E4B216D0202CF3D1C4
:10B070000121686AFFF70CFB95F82C206B6A5200DF
:10B0800083F83B2083F85E8083F85D80686A0368FC
:10B0900000211B6898470124DEE7686A0121BDE8AA
:10B0A000F041FFF7F5BAC26BC16C136823EA0103E4
:10B0B00006EB080413604FF00048A6420ED02B6A3E
:10B0C00016F801EB63B11A68C2F82C80C2F834E0BC
:10B0D000D36A002BFCDAA642936BF0D1BDE8F08175
:10B0E000AB6BD5F834C008208021DCF800206F6CF1
:10B0F0001EEA010F14BF3A43BA43CCF800201A6885
:10B10000AF6C3A431A601A68AF6C013822EA070242
:10B110004FEA51011A60E8D1CFE700BF70B504468D
:10B12000406A0D46002828D0A16DFFF74FF9204650
:10B130002946FFF7A9FE606A20B1E16DBDE87040C5
:10B14000FFF744B9216C226D0868236A02430A6044
:10B1500093B1DA7A82B1D00703D5234A9969116095
:10B16000DA7A910703D5214AD9691160DA7A520750
:10B1700002D51F4A1B6A136070BD236A002B2BD0B7
:10B18000D97A626DE1B172B6D97ACE0706D519487F
:10B19000D9680668314099610160D97A880706D577
:10B1A0001548196906683140D9610160D97A4E079E
:10B1B00005D512485969066831401962016062B6C6
:10B1C0001B68D968914207D00D4818600D49DA60B4
:10B1D00042F0804018611960226C216D136823EAE7
:10B1E00001031360A3E700BF00E100E004E100E019
:10B1F00008E100E080E100E084E100E088E100E0B7
:10B2000001403F0000003F802DE9F041044686B038
:10B21000806A9DF830801E460F461546B4F9083006
:10B22000002800F04281DA1D48BF03F10E02B4F994
:10B230000630D21003FB02F2002105F0BDFCB4F988
:10B240000820202A00F39280B4F90610A34B0120B5
:10B25000203A733902EBD27201EBD1714FF0200E1C
:10B26000029073208DE8014042F34F0241F34F01F9
:10B27000204600F051FE606A84F82D70002800F02E
:10B280004D81002D40F08A80B4F90830202B14BF86
:10B290003D253C2584F82C50B8F1000F40F0858006
:10B2A00006B394F93300002818DBC0B2012102F084
:10B2B000E7F8012194F8330002F0CEF8012002F003
:10B2C00007F9002194F8330002F0C6F80A2002F0D2
:10B2D000FFF8012194F8330002F0BEF8606A0028FC
:10B2E00000F08280A16DFFF771F804227C492046AE
:10B2F000FFF792FE217A0139C9B22046FFF7C4FD5B
:10B30000784904222046FFF787FE94F92D30012B5F
:10B3100014BF142110212046FFF7B6FD0422724904
:10B320002046FFF779FEB4F90630802B00F09280BA
:10B33000602B00F0A680D9212046FFF7A5FD94F9E7
:10B340002D30012B14BFF12122212046FFF79CFD57
:10B35000204606226549FFF75FFE606A50B3E16D43
:10B36000FFF734F8012006B0BDE8F081B4F906100B
:10B370005F4B0120403A52394FF0400E029002EBF1
:10B38000D272522001EBD1718DE8014042F34F029D
:10B3900041F34F01204600F0BFFD6CE76DB284F829
:10B3A0002C50B8F1000F3FF47BAFFEF7C5FF002E25
:10B3B00094D076E7216C226D0868236A02430A6004
:10B3C00073B1DA7A62B1D00703D54A4A996911603C
:10B3D000DA7A91077CD4520702D5474A1B6A136078
:10B3E000012006B0BDE8F081236A002B2BD0D97A6A
:10B3F000626DE1B172B6D97ACF0706D53F48D968F8
:10B400000568294099610160D97A8E0706D53C48C4
:10B41000196905682940D9610160D97A4D0705D5B8
:10B4200038485969056829401962016062B61B688D
:10B43000D968914207D0344818603449DA6042F044
:10B44000804018611960226C216D136823EA0103A2
:10B4500013604AE7B4F90830202B00F08680402BB7
:10B460007FF469AF2A4920460322FFF7D5FD94F9FE
:10B470002D30012B14BFCF219F212046FFF704FD63
:10B4800059E7B4F90830102B7FF455AF2149204615
:10B490000322FFF7C1FD94F92D30012B14BFAF211A
:10B4A00010212046FFF7F0FC45E7DA1D48BF03F105
:10B4B0000E02B4F90630D21003FB02F210460592D8
:10B4C00005F04EF8A06200283FF44DAF059AB3E6B0
:10B4D000114AD9691160DA7A7DE700BF00310100B5
:10B4E000E0320100E4320100E8320100EC320100F8
:10B4F000F432010000E100E008E100E080E100E05A
:10B5000084E100E088E100E001403F0000003F806E
:10B51000FC300100B435010004E100E0012194F8A1
:10B520003100244F01F0ACFF94F83200012101F00A
:10B53000A7FF94F9312094F9323057F83220E263B2
:10B5400057F83330206A23640125E56425651A68BD
:10B550002A431A6078B1B8F1000F3FF428AFFFF723
:10B560005BFB002E3FF4BAAE9BE604221249204654
:10B57000FFF752FDDFE6294694F82F0001F080FF27
:10B58000294694F8300001F07BFF94F92F2094F9BC
:10B59000303057F83220626357F833306564A56461
:10B5A0001A68A36322F001021A60002E3FF496AEDF
:10B5B00077E600BF503B0100F8300100B0F90820E9
:10B5C000D31D48BF02F10E03B0F90620806ADB10DC
:10B5D00002FB03F2002105F0EFBA00BFF0B500292D
:10B5E000BDF814502EDBB0F90660B1422ADA002A09
:10B5F00059DBB0F9087014461C44BC42C4BFBB1AE6
:10B600001BB2002B1EDDD2B2D408D0F828E016FB06
:10B61000041112F00702DBB20EEB010421D0C2F1DB
:10B620000807FAB2374F9342BF5C0CD2C3EB020C4F
:10B63000FF2646FA0CF6012D07EA06073FD005D390
:10B64000022D36D0F0BD012D39D030D21EF8016068
:10B6500026EA07070EF801709342F3D3B0F90610FB
:10B660000C449A1AD2B2072A10D9022D36D0002DD6
:10B6700014BFFF26002613462670083BB0F90610BB
:10B68000DBB2072B0C44F7D802F00702002AD9D00E
:10B690001D4B012D9B5C1DD017D3022DD2D12278DA
:10B6A00053402370F0BD13441BB20022A1E7022DCA
:10B6B00025D11EF8016077400EF80170CCE71EF826
:10B6C000016037430EF80170C6E7227822EA0303CF
:10B6D0002370F0BD227813432370F0BD1146237808
:10B6E000DB4323700839B0F90630C9B207291C447E
:10B6F000F5D812F00702A5D0034B9B5CCFE734448A
:10B70000AFE700BF983001008830010070B4C47DFD
:10B71000BDF80C50022C18D0032C1FD0012C0BD0DC
:10B72000002A03DBB0F90840944201DC70BC70478A
:10B73000039570BCFFF7B0BAC4880395013CA41A06
:10B740000A4621B270BCFFF749BF0689C488013E92
:10B75000641AB21AE41A12B221B2E1E7048903951D
:10B76000E41A641A114622B270BCFFF737BF00BF5B
:10B7700070B4C57DBDF80C60022D1AD0032D12D017
:10B78000012D03D0039670BCFFF728BFC488E41ACC
:10B79000A41A0A4621B2002A03DBB0F908409442F9
:10B7A00013DC70BC70470489013C641A114622B254
:10B7B000F1E7C48805890396013CAD1AED1A621AB7
:10B7C00011B22AB270BCFFF709BF039670BCFFF735
:10B7D00063BA00BF2DE9F8430446406A002863D0ED
:10B7E000A16DFEF7F3FD052274492046FFF714FC16
:10B7F000A1790139C9B22046FFF746FBB4F9082008
:10B80000E588A66AD31D48BF02F10E03DB10626A09
:10B8100015FB03F51FFA85F8002A7BD094F82C302D
:10B820000125AB4082F83B3082F85E5082F85D50D3
:10B83000606A036840211B6808F1FF379847BFB270
:10B84000B8F1000F23D03744A846013E606A16F8CD
:10B85000011F03681B6898470135B742EDB216D047
:10B86000202DF3D10121606AFEF712FF94F82C20FD
:10B87000636A520083F83B2083F85E8083F85D8022
:10B88000606A036840211B6898470125DEE70121B3
:10B89000606AFEF7FDFE606A002800F08D80E16DB1
:10B8A000BDE8F843FEF792BD236A002B2BD0D97A6E
:10B8B000626DE1B172B6D97ACE0706D54048D96833
:10B8C0000568294099610160D97A8D0706D53D4800
:10B8D000196905682940D9610160D97A480705D5F9
:10B8E00039485969056829401962016062B61B68C8
:10B8F000D968914207D0354818603549DA6042F07E
:10B90000804018611960226C216D136823EA0103DD
:10B91000136068E7E26BE36C1168276A0B4306EB80
:10B92000080913604FF0004E4E450DD016F801CBBC
:10B930002FB33A68C2F82CE0C2F834C0D36A002BA7
:10B94000FCDA4E45936BF1D1226C236D11680B43E9
:10B95000136097B1FB7A83B1D90703D51D4BBA6940
:10B960001A60FB7A9A0703D51B4BFA691A60FB7AB7
:10B970005B0702D5194B3A6A1A60BDE8F883A36BDE
:10B98000D4F8348008208021D8F80020656C1CEAA7
:10B99000010F14BF2A43AA43C8F800201A68A56CF7
:10B9A0002A431A601A68A56C013822EA05024FEA98
:10B9B00051011A60E8D1B7E7276AC5E79030010066
:10B9C00080E100E084E100E088E100E001403F0028
:10B9D00000003F8000E100E004E100E008E100E059
:10B9E0002DE9F04F85B09946BDF93870BDF83CA0FF
:10B9F000BB1AC1EB090B002BB8BF5B42BBF1000FB8
:10BA0000B8BFCBF1000B5B450D4616460093804650
:10BA100048DC4D453A4633464CDC194613460A4647
:10BA2000C5EB09019B1A89B2002B0CB2B8BF5B426F
:10BA300004EBD474BE42ACBF4FF0FF3201224D453F
:10BA4000039102924FEA640429DC9BB201930DE05A
:10BA5000D8F80070BF69B847019BE41AA3B21CB2C2
:10BA60000135002C2DB211DBA94518DB009B5B458D
:10BA70002A46534631464046EADCD8F80020534671
:10BA80009769294632464046B847E5E7029A164488
:10BA9000039AA94502EB030436B224B2E6DA05B0F4
:10BAA000BDE8F08F4A462B46B94635464D45174608
:10BAB0001E46B2DD304629463E464D46074689467B
:10BAC000AEE700BF10B404682469A44610BC604708
:10BAD00030B40468BDF808500295A46BA44630BC8D
:10BAE000604700BF30B40468BDF808500295E46BAD
:10BAF000A44630BC604700BF70B40468BDF90C6058
:10BB0000BDF8105003960495246CA44670BC6047A1
:10BB1000704700BF10B582B0B0F90C2001910168E8
:10BB2000009200220C6CB0F90A301146A04702B016
:10BB300010BD00BF704700BF01F003010129C175AE
:10BB400006D0032904D0C2880389428183817047CB
:10BB50000289C38842818381704700BF2DE9F0418B
:10BB60000568134E6F6986B0B7420446BDF8308051
:10BB700010D1013B13441BB20093CDF804800B4657
:10BB8000AD6A2046A8472368DB6AB3420AD106B0F3
:10BB9000BDE8F081059304920391B84703A9256895
:10BBA0000EC9E6E7204606B0BDE8F041184700BFE1
:10BBB00011BB00002DE9F0410568124E6F6986B097
:10BBC000B7420446BDF830800FD1013BCDF8048068
:10BBD0000B4400921BB2AD6A2046A8472368DB6A7B
:10BBE000B3420AD106B0BDE8F081059304920391F7
:10BBF000B84703A925680EC9E7E7204606B0BDE8A7
:10BC0000F041184711BB00002DE9F04F0568DFF83F
:10BC100058B06F6985B05F450646BDF93890BDF8EC
:10BC20003CA00C46904615D11F19BC420CDACDF849
:10BC300000A0214601342D6A4B464246304624B2CC
:10BC4000A847BC423568F2DBEB6A5B4507D105B01B
:10BC5000BDE8F08F0393B8473568039BE4E73046AF
:10BC600005B0BDE8F04F184711BB00002DE9F043C7
:10BC700087B099420546BDF93840BDF83C6025D0F3
:10BC8000A24212D00768DFF88080D7F81490C1452F
:10BC900032D18DE850002846BC6AA0472B68DB6A89
:10BCA000434524D107B0BDE8F083994202DD084640
:10BCB0001946034628680E96C46B01335B1A1BB203
:10BCC0002846A44607B0BDE8F0436047A24202DD23
:10BCD000134622461C4628680E96631C846B9B1AEA
:10BCE0001BB22846A44607B0BDE8F043604728468B
:10BCF00007B0BDE8F0431847059304920391C84785
:10BD000003A92F680EC9C4E711BB00002DE9F04F4D
:10BD1000D0F800E0DFF89090DEF814B083B0CB45A7
:10BD20000446BDF93080BDF834A00D4617461E46C6
:10BD300031D1CDF800A0DEF824B0294633463A468A
:10BD40002046D8472368CDF800A008F1FF323A44D6
:10BD5000D3F824B0294612B233462046D847236888
:10BD6000CDF800A02946D3F820B03A4643462046F5
:10BD7000D8472068CDF800A0711E29444346056AC3
:10BD800009B23A462046A8472368DB6A4B4506D1EC
:10BD900003B0BDE8F08FD847D4F800E0C9E72046EB
:10BDA00003B0BDE8F04F184711BB0000F0B4002409
:10BDB00001264FF6FF75094F07600471C475C481F1
:10BDC00004824476C4618675067685824582C18088
:10BDD000028141818281F0BC704700BFC035010003
:10BDE0002DE9F04F85B00668BDF84450BDF93880A4
:10BDF000CDF8008004460195D6F848B00392BDF90D
:10BE00003C60BDF9407089469A46D8472368019541
:10BE1000009742465146D3F8488020463346C047F3
:10BE20002068039B0E930F95856C4B463A4631462E
:10BE30002046AC4605B0BDE8F04F60472DE9F04F15
:10BE400087B01746BDF9404000912546E91D05938E
:10BE500044BF2B4603F10E010268BDF848605369E8
:10BE60000294C91003912B49BDF9444001968B42BD
:10BE7000824645D1002C3CDD029B3C445E1EB6B29E
:10BE80004FF0000923B2049301364D46029B002B6C
:10BE900028DD059B002403EB090806E0EDB22B0624
:10BEA00004F1010411D4A6421CD0A1B211F0070F75
:10BEB00023B24FEA4505F1D1002BB8BF0733DB10A1
:10BEC000013418F803502B06EDD5009BD2F818B0BA
:10BED00019443A4609B2019B5046D847A642DAF8BF
:10BEE0000020E2D1039B01379944049B3FB2BB423F
:10BEF000CCD1D36A074A934206D107B0BDE8F08F90
:10BF00009847DAF80020B5E7504607B0BDE8F04F93
:10BF1000184700BF11BB000070B4BDF90C60BDF93B
:10BF20001050BDF8144003960495059470BCFFF7BB
:10BF300085BF00BF2DE9F04F93B090460591C169D0
:10BF40001090BDF870000790BDF874909DF878A02F
:10BF50000493002900F0CD800A7A0AC98946049921
:10BF60008A1AD2B203EBC203BAF1010FDA780B924C
:10BF700093F905201E8893F802B00F9293F90640BA
:10BF800079D913B2099323B20C93109B1A68A94B69
:10BF90001193194653698B4240F0A6800B9B002BEE
:10BFA00055D01FFA88F300210D93C8462344DDF8CD
:10BFB000409006910E930F460C46BBF1000F3FD008
:10BFC000BDF818100C9B03971FFA8AF0CB1813FBCF
:10BFD00000F304900E9801440D98034409B21BB27B
:10BFE0000A910893002505E00135EBB264009B45FA
:10BFF000E4B222D9039B2B44590703D1731C18F8D0
:10C0000006409EB22306EFD5099BBDF81000E91843
:10C0100011FB00F10598BAF1010F0FFA8AF3014400
:10C020001CD0079801900093D26909B21746484680
:10C03000089AB847D9F80020D6E7039F5F44FFB2BB
:10C04000069B0B9901330693DBB29942B5D8D36AAC
:10C05000119A934243D113B0BDE8F08F0F9B19188A
:10C0600093690A9A29441F4609B2079B4846B84774
:10C07000D9F80020B8E700230C93099385E70A9AC2
:10C080000D9B0132013B52B213F0FF030A920D9354
:10C090006FD1DDF81890079BDDF83C80DDF820A01B
:10C0A0004B4517D0BAF1010F00F0C8800B9A109DD4
:10C0B000CDF804900BEB8B014FEACB030A440093BD
:10C0C0001146DEF81C405346424609B22846A047B6
:10C0D000D5F800E0DEF82C30119A9342BBD01098CE
:10C0E00013B0BDE8F04F1847109D284698472A68BE
:10C0F00054E7109A0598B2F90A308342ABDDB2F9E1
:10C100000C304345A7DD062313FB0A03002BA2DDF9
:10C1100008EBCA03002B9EDD537E2BB9049BAF2B8B
:10C1200002D90133DBB20493109BD3F800E0414BFA
:10C1300011931A46DEF81430934240F08E801FFAB5
:10C1400088F30E9308339BB2BDF8142005930523A2
:10C150000D9300230A93CDF83C800FFA8AF3DDF8A3
:10C160004080CDF818900B921FFA8AFBCDF820A0E2
:10C1700099460A9ABDF810000B9C0E9D052319469E
:10C1800011FB00232C481146C75C039702FB0B42AE
:10C1900014FA81F312B21BB209920C932C462E466C
:10C1A0001CE0089B0999012B2AB24B4640462DD032
:10C1B000079F0197CDF80090DEF81CA0D047D8F873
:10C1C00000E0039B5B0801340393059BA4B25D442C
:10C1D0005E44A342ADB2B6B23FF451AF039BD80761
:10C1E000DFD4079B069A9342EBD0089B012B16D015
:10C1F000069B0193CDF80090DEF81CA009994B46F0
:10C2000032B24046D047D8F800E0DAE7DEF818A0AE
:10C21000079B0C9922B2D047D8F800E0D1E7DEF8AE
:10C2200018A00C991346404622B2D047D8F800E037
:10C23000C7E700BF11BB0000103601000B99109D2D
:10C24000CDF800900531DEF8204009B242460823BF
:10C250002846A047D5F800E03CE7109C20469847C8
:10C26000D4F800E06BE700BFF0B5C36985B00446C1
:10C270002BB30A2968D00D294AD01A7A914247D3A4
:10C28000587A884244D35D688A1A05EBC205AA78B9
:10C29000002A50D0E87800284DD0207E00283AD0DF
:10C2A00095F905E0B4F90E00A67DB4F90A70724460
:10C2B00006FB0202BA4262DCB4F9102030E00A291F
:10C2C00056D00D2924D0027E002A4BD0B0F90E00A2
:10C2D000A57DB4F90A60062212FB0502B2423EDDDA
:10C2E000228AE38102EBC50212B218462282A78A93
:10C2F000668A02950B468DE8C00001462046FFF78E
:10C3000019FEA37DE28903EB430302EB4303E381C0
:10C31000012005B0F0BDA67DB4F90E00B4F91020DF
:10C32000B4F814E0678A02960B468DE88040014617
:10C330002046FFF7FFFD2979E389A27D012001FB5B
:10C340000233E38105B0F0BD0022C2819A7A817D7B
:10C35000038A01FB02330382012005B0F0BDB4F96A
:10C360001020C4E7857DB4F91020B0F90E00BEE7B7
:10C37000028A817DC38102EBC1030382C8E70020EA
:10C38000E0819B7A228A03FB062212B22282C7E74F
:10C39000C1810282704700BF002908BF0121817559
:10C3A000704700BF81824182704700BFC07D7047E7
:10C3B000B0F90A00704700BFB0F90C00704700BF29
:10C3C00010B4EFF3108272B6437F33B9017F0129B5
:10C3D00007D003290FD00123437702B962B610BCFE
:10C3E0007047124C2168A1B1114943610B68836108
:10C3F00008605861EFE70F4C216881B10E49436135
:10C400000B688361086058610C4B4FF080511960D4
:10C41000E1E7074B4161816120601860DBE7064B73
:10C420004161816120601860EEE700BF689FFF1FD7
:10C43000649FFF1F589FFF1F5C9FFF1F04ED00E0DC
:10C4400070B5EFF3108272B60C4C206880B10C4EC0
:10C4500000254369236073B19D6102B962B64577D7
:10C4600083689847EFF3108272B620680028F0D1F5
:10C4700002B962B670BD3360EFE700BF589FFF1F7F
:10C480005C9FFF1FFFF7DCBF184A30B41468002C14
:10C4900027D0036821688B420ED2CB1A002184601A
:10C4A000C1602360E06010600223037530BC7047F8
:10C4B00011688B42144608D3A2685B1A0360002AF5
:10C4C000F6D18260C460A060EEE7D268C26084608A
:10C4D000E060C568CB1A0222A8602360027530BCF8
:10C4E00070478460C4601060DEE700BF609FFF1F7C
:10C4F000F8B5224E34682CB32368002B3AD1204F74
:10C500001D4604E03468ECB12368002B32D1A368E7
:10C5100003B1DD6020693360036825751B68BB4289
:10C5200021D1037F4560022BC46020D0FFF748FF74
:10C530006368002BE6D023602046FFF7A5FF346830
:10C54000002CE1D1EFF3108372B60E4A002110687F
:10C55000116003B962B628B18468FFF795FF2046E1
:10C560000028F9D1F8BD224600219847E0E783680A
:10C570009847DDE7013B2360E4E700BF609FFF1FB2
:10C5800001AC0000709FFF1F024A13680133136063
:10C59000FFF7AEBF7C9FFF1F704700BF0368F0B47A
:10C5A000FBB1002501249D60DC601B4C1A601C441B
:10C5B000241104F144056A11032692009E60174F6E
:10C5C0000679174B47F8241002F1604202F56142E8
:10C5D00005F01F05012000FA05F5E6541560F0BCD2
:10C5E0007047104C236843F40003236000BF0E4BD8
:10C5F0000E4DA4F58734A4F59E7401261E602346D3
:10C6000004609C68002CD0D01033AB420360F8D19A
:10C61000002303601846E2E7008FFCBFA891FF1FCC
:10C6200044E400E03C80044000700340407103405B
:10C630000168A9B10B4BF0B40B441B110A4E0B4F10
:10C640000B4D46F8237003F1440202F01F0401234E
:10C650005211A340002445F822308C600460F0BCE5
:10C66000704700BF008FFCBFA891FF1F99C5000055
:10C6700080E100E0024A034B012111601B6818476A
:10C680000C710340A891FF1F024A034B0121116066
:10C690005B6818471C710340A891FF1F024A034BB7
:10C6A000012111609B6818472C710340A891FF1F5E
:10C6B000024A034B01211160DB6818473C710340BB
:10C6C000A891FF1FF8B50E4671B17AB1074614461E
:10C6D00000253B6816F8011B1B6838469847013C4B
:10C6E0000544F6D12846F8BD0846F8BD1046F8BD09
:10C6F00000B5064A036812885B6883B001A9ADF8EB
:10C7000004200222984703B05DF804FB103B0100AF
:10C71000F0B507468BB0002A33D0012A08BF0A22A1
:10C7200051B3212400E0F4B2B1FBF2F502FB151184
:10C73000C8B2092900F1300198BFC8B20AA988BF60
:10C740003730214488BFC0B201F8240C661E294648
:10C75000002DE8D133B1013CE4B20AAB23442D22D1
:10C7600003F8242C3B6801AA11195B683846C4F110
:10C77000220298470BB0F0BD30228DF825202124ED
:10C78000E8E70368C9B21B6898470BB0F0BD00BF6B
:10C790000029BABF49422D2300230A22FFF7B8BF60
:10C7A000374A384913681B06FCD40B6813F0800322
:10C7B000F8D172B634490A78002A5FD0334A344837
:10C7C000F0B4344C176806682568D4680C303E44D1
:10C7D000143200681268304F35442C44204402441F
:10C7E000C2F34E022D4E2E482E4D2F4C42F40042E5
:10C7F0003A60376806682D682C4A24680C303E443D
:10C80000006812682A4F35442C4420440244C2F385
:10C810004E02284E2848294D294C42F400423A60E5
:10C82000376806682D68274A24680C303E44006843
:10C830001268254F35442C4420440244C2F34E0272
:10C84000224E2348234D244C42F400423A6037687C
:10C8500006682D68214A24680C303E44006812683E
:10C8600035442C4420440244C2F34E021C4842F496
:10C87000004202600B7062B6F0BC704762B670474F
:10C8800024B0034024B00B40759FFF1F38B0034015
:10C890003CB0034040B003402CB0034058B00340CC
:10C8A0005CB0034060B0034064B003406CB0034030
:10C8B00030B0034038B00B403CB00B4040B00B40B0
:10C8C00044B00B404CB00B402CB00B4058B00B4068
:10C8D0005CB00B4060B00B4064B00B406CB00B40E0
:10C8E00030B00B4030B42948294A2A4B2A4D6024E5
:10C8F000E121047011701B78284C082B30D00A2BD2
:10C900002748284937D00C2B0CBF35223D22122353
:10C910002A60236002600B60234B24491B78244A61
:10C92000BBB101230B601360224B23491B78234AC0
:10C93000012B26D9042B0FD9082B1ED9102B94BFFD
:10C94000862387230B6013601D4B01221A7030BCB5
:10C9500070470B601360E7E784230B601360F3E715
:10C9600000F58E200F490830012213232A6023602E
:10C9700002600B60D0E73922F7E785230B60136074
:10C98000E2E780230B601360DEE700BF0040074052
:10C9900001400740B891FF1F08B003400CB00340AE
:10C9A00008B00B400CB00B40789FFF1F20B0034035
:10C9B00020B00B40B991FF1F24B0034024B00B40BE
:10C9C000759FFF1F0C2830B417D91023984228BF39
:10C9D00018461C46104A114D1178181A8C422870BE
:10C9E00018D00F4913700B7823B10E490E4A00235B
:10C9F0000B60136030BCFFF775BF0A2802D90C2307
:10CA00001C46E7E7082802D90A231C46E2E7082368
:10CA10001C46DFE730BC7047B891FF1F749FFF1FB3
:10CA2000759FFF1F24B0034024B00B4028282FD847
:10CA3000334B2DE9F0411E5CFF2E2BD0314B1B7880
:10CA4000002B2AD132062CD472B62F4D2F4C2F46F4
:10CA5000012326602B7062B672B623681B060CD4C5
:10CA60003B781BB9F4E72B78002BF1D062B602F0CB
:10CA70009BF972B623681806F5D5254B1B68002272
:10CA80002A7062B6234A107843FA00F0BDE8F081BC
:10CA9000002070470020BDE8F081FFF781FE3206DC
:10CAA000D2D572B61C4DDFF87C801C4C06F04007D6
:10CAB000FFB206F03F06D8F80030DFB123F01003D4
:10CAC000C8F8003001232660134A2B7062B672B694
:10CAD000236819060CD413781BB9ECE72B78002BCC
:10CAE000E9D062B602F060F972B623681B06F5D58C
:10CAF0000B4BC3E743F01003C8F80030E2E700BF78
:10CB0000143B0100759FFF1F779FFF1F00B003407C
:10CB100010B00340749FFF1F769FFF1F00B00B40B3
:10CB200010B00B400CB00B400A4A0B49136843F499
:10CB3000805313600B7843B9084BC0221A70084B1E
:10CB400080F30C0000B218807047044B80221A70EA
:10CB5000F5E700BF2C800440789FFF1F21C00C40E8
:10CB600000C00C40F0B51B4B1B4E596818689A6802
:10CB7000DB6885B06C460FC4337899071DD5174A1A
:10CB8000174C1378174913F0700318BF1370164A27
:10CB9000164B8027177000263320032226706D461F
:10CBA00008701A7072B6043C45F001052046A8478B
:10CBB00062B6237813F0700309D10D4B064901E0EA
:10CBC000013B02D00A78D207FAD505B0F0BD237038
:10CBD00005B0F0BD403B01000100024000000240F2
:10CBE000040002400B000240070002400A0002401D
:10CBF000410D0300B0F5006F0AD210B5094B1B7848
:10CC0000DB07044606D504F1A0500078C0B210BD81
:10CC100000207047FFF7A6FF04F1A0500078C0B2D3
:10CC200010BD00BF01000240B0F5006F17D238B54B
:10CC30000F4B1B78DA070D46044611D504F1A050BE
:10CC40000378AB420AD00B4A137813F0700318BF75
:10CC50001370074A05701378DB07FCD538BD7047A1
:10CC6000FFF780FF04F1A0500378AB42EBD1F5E76A
:10CC7000010002400000024008B5F4F7ADFEF5F7F0
:10CC800057FD02F091F8FAE7844641EA000313F0F9
:10CC900003036DD1403A41D351F8043B40F8043BC3
:10CCA00051F8043B40F8043B51F8043B40F8043B86
:10CCB00051F8043B40F8043B51F8043B40F8043B76
:10CCC00051F8043B40F8043B51F8043B40F8043B66
:10CCD00051F8043B40F8043B51F8043B40F8043B56
:10CCE00051F8043B40F8043B51F8043B40F8043B46
:10CCF00051F8043B40F8043B51F8043B40F8043B36
:10CD000051F8043B40F8043B51F8043B40F8043B25
:10CD100051F8043B40F8043B403ABDD2303211D3C5
:10CD200051F8043B40F8043B51F8043B40F8043B05
:10CD300051F8043B40F8043B51F8043B40F8043BF5
:10CD4000103AEDD20C3205D351F8043B40F8043BC5
:10CD5000043AF9D2043208D0D2071CBF11F8013BC3
:10CD600000F8013B01D30B8803806046704700BF89
:10CD7000082A13D38B078DD010F003038AD0C3F198
:10CD80000403D21ADB071CBF11F8013B00F8013B7A
:10CD900080D331F8023B20F8023B7BE7043AD9D339
:10CDA000013A11F8013B00F8013BF9D20B7803700E
:10CDB0004B7843708B7883706046704708B5104C91
:10CDC00008E0236859050DD423681A050FD4236899
:10CDD000DB0411D423685803F3D500F08DFE2368DB
:10CDE0005905F1D502F044F823681A05EFD502F091
:10CDF000D5F82368DB04EDD500F0F0FCEAE700BFCE
:10CE00003480044008B5FFF7D9FF00BF014B102262
:10CE10001A80704700200540704700BF094908B5D7
:10CE20000B6830B16A461844A2F58052904202D293
:10CE30000860184608BD03F065FB0C2303604FF043
:10CE4000FF3008BDBC91FF1FFEE700BFEFF313806A
:10CE500070B9EFF310836BB9EFF305825AB94FF451
:10CE60008070EFF311832BB1984228BF18467047AA
:10CE70004FF0FF3070470F2A01D81846F1E7014BF9
:10CE8000D05CEEE7F0E300E0F0B44D1E2E46002447
:10CE900000E00134B0FBF2F302FB1300092800F1BB
:10CEA00030078ABF3730F8B2C0B206F8010F184613
:10CEB000002BEED10A1953704CB1107815F8016FA0
:10CEC00028700133E01A834202F80169F5DB084655
:10CED000F0BC7047704700BF10B40F4B53F83020C0
:10CEE00092F880422CB1012369B182F8803010BCE5
:10CEF000704703EBC0035B681A6841B922F0020275
:10CF00001A6010BC704782F8003110BC704742F0C4
:10CF100003021A6010BC7047503B01001C4A02EB30
:10CF2000C00301295B6811D004291BD052F83000DE
:10CF3000002280F8802229B1022920D0032922D0A2
:10CF40001A6070474FF480721A60704752F83000D0
:10CF50004FF4A27280F880121A601A6822F0200240
:10CF60001A60704752F830104FF4A272012081F815
:10CF700080021A601A6842F020021A60704740F27C
:10CF800003121A6070474FF481721A60704700BF35
:10CF9000503B0100212848D8F8B5042A44D8DFE8DE
:10CFA00002F0484B4E0345004FF410262B4B03EB89
:10CFB000C0030D465C68216811F4E06148D0284B3D
:10CFC000284A2949C3F89C2104F140422748C3F864
:10CFD000A411A2F59221264FC3F8A0017C2925486F
:10CFE000C3F8A871C3F8AC012CD9A2F594237C2B0B
:10CFF0002AD9A2F596237C2B28D9A2F598237C2B3D
:10D0000029D9A2F59A227C2A27D81B4872B6236810
:10D0100023F4702343F08072C4F384011643236029
:10D0200040F82150266062B6F8BD70474FF43026B4
:10D03000BCE74FF40026B9E74FF44026B6E74FF4BB
:10D040002026B3E70D48E1E70D48DFE70D48DDE7AF
:10D05000FFF764FFB3E70C48D8E7F8BD503B010089
:10D060000082FF1FF188FF1F9988FF1FC588FF1FDF
:10D070006D88FF1F4188FF1F9892FF1FC091FF1FFF
:10D08000F891FF1F4892FF1F7892FF1F1A4B03EB86
:10D09000C00010B4426802F14043A3F592217C29FC
:10D0A00023D9A3F594217C290DD9A3F596217C29B8
:10D0B0001FD9A3F598217C2919D9A3F59A237C2B94
:10D0C00011D80E4C00E00E4C72B613680D4823F0D8
:10D0D0008773C2F3840123F4803343F080731360B9
:10D0E00044F8210062B610BC7047074CECE7074CCF
:10D0F000EAE7074CE8E700BF503B01009892FF1FAA
:10D10000F891FF1FD5CE0000C091FF1F7892FF1F3E
:10D110004892FF1F30B4054B054D064C00221021EC
:10D120001A602A602060196030BC704714D0034038
:10D1300004D0034000D00340282838B52ED0002961
:10D1400004464FDD5F4B1B78012505FA03F28A4246
:10D1500002D8212837D938BD0338C2B2012A3AD9BA
:10D16000202C4AD0192C48D0574A126802FB0112D1
:10D1700022FA03F31D2800F29B80DFE800F0928B77
:10D18000847D9999766F99999999999999999968BE
:10D19000615A53994C99999999999945494B1B789A
:10D1A0000B2B08D90C2B1CBF0C3B19410846BDE8C2
:10D1B0003840FFF7B9BCC3F10C0399400846BDE8FD
:10D1C0003840FFF7B1BC2946FFF786FE2946BDE887
:10D1D0003840FFF7A3BE3D4A126802FB011222FA53
:10D1E00003F3C7E72128B6D80021FFF775FE2046D4
:10D1F0000121BDE83840FFF791BE354A126802FBB5
:10D20000011222FA03F3B5E73249334A0B604FF4B7
:10D210005173136038BD3149314A0B604FF451737B
:10D22000136038BD2F49304A0B6040F2444313600D
:10D2300038BD2E492E4A0B6040F24443136038BD7E
:10D240002C492D4A0B6040F24443136038BD2B49F2
:10D250002B4A0B6040F24443136038BD29492A4AE7
:10D260000B6040F24443136038BD2849284A0B60E4
:10D2700040F24443136038BD2649274A0B6040F210
:10D280004443136038BD2549254A0B6040F24443AE
:10D29000136038BD2349244A0B604FF45173136067
:10D2A00038BD2249224A0B604FF45173136038BDD8
:10D2B000212C3FF650AF7F29D4BF00210121204609
:10D2C00093E700BFA092FF1F08800340089003402F
:10D2D00008800B4010800B4048A0044018800B4091
:10D2E0004CA004401880034008B004401080034064
:10D2F00004B004404080034018C00440388003401C
:10D3000014C004402880034010B004402080034033
:10D310000CB004403080034010C0044048800340FB
:10D320001CC0044018900340349004401090034007
:10D330003090044038B1102828BF1020044AC3B2EE
:10D34000107813707047024A0123107813707047E9
:10D35000A092FF1F2DE9F8430E4680463249334D17
:10D36000304603F055F847F6122300281ABF1D4631
:10D370004FF002094FF00109002425FA04F002F0F1
:10D3800051FE4FF05E51074602F0A4FE01463046C2
:10D3900003F052F830B90134072CEED1E80902F05D
:10D3A00041FE07463146384602F048FF4FF07C51B7
:10D3B00002F086FD03F07AF84FF6FF729042A8F172
:10D3C000030328BF1046012B29D9B8F1170F17D82E
:10D3D000174B23FA08F303F0010383F0010223B98A
:10D3E000B8F1190F0FD0BDE8F883124B124D134955
:10D3F0001A6044EAC9042A6008601C60BDE8F8832A
:10D40000B8F1200FECD10E4B0E4D0F49002244EA2B
:10D41000C9041A602A6008601C60BDE8F8830B4BE1
:10D420000B4D0C49F2E700BF001BB740006CDC025B
:10D430006006F00000800340048003400880034041
:10D4400000800B4004800B4008800B40009003409C
:10D450000490034008900340212801D8FFF73CBD09
:10D46000704700BF212806D8044B53F8303093F89A
:10D470000002C0B270470020704700BF503B01005F
:10D48000212801D8FFF74ABD704700BF72B60C498A
:10D490000C4B0D4A1B680868126862B6520102D52F
:10D4A000322B88BF01300949C3F5BB334FF47A7280
:10D4B000FF33A1FB031302FB00F000EB9310704756
:10D4C0007C9FFF1F18E000E004ED00E0ABAAAAAAD1
:10D4D0002DE9F843054672B6204F214B214A1B68BF
:10D4E0003C68126862B6520102D5322B88BF013403
:10D4F00095B3C3F5BB331C4EDFF86490DFF864804E
:10D50000FF334FF47A72A6FB031302FB04F404EB1F
:10D51000931472B6D9F800103A68D8F800E062B6F1
:10D52000C1F5BB33FF33A6FB03031EF0806FC4EBD2
:10D5300093134FF47A7002D0322988BF013200FB76
:10D540000233B3F57A7F04D3013D05D004F57A7434
:10D55000DFE701F029FCDCE7BDE8F8837C9FFF1FD3
:10D5600018E000E004ED00E0ABAAAAAAF8B52D4B44
:10D570002D49DFF8D0E0DFF8D0C02C4E2C4D2D4CDB
:10D580002D4A2E4F4FF4000018604FF08070186045
:10D590004FF0007018604FF0806018604FF000602E
:10D5A00018600020086028234BF6FF71CCF80010AB
:10D5B000CEF80030336013602B6023603B60B362B1
:10D5C0009362092245F8242CC4F8D80F05F57F652D
:10D5D000C7F8D41F07F5FF2707F5FA67C6F8F83F25
:10D5E0002B6006F5FF26C4F8D42F05F5FD2504F5BC
:10D5F000FF24386006F2F4761148316005F5FF65C6
:10D6000004F5FD642B6023600260FFF76BF91920BD
:10D61000FFF75EFF00F0B6FF40F21310BDE8F840E0
:10D62000FFF756BF08E100E0048003401480034088
:10D63000248003402C8003401C800340348003403E
:10D6400000800B400C800340088003402DE9F84F18
:10D65000214B1B6807460BB101221A70DFF8889036
:10D660001E4D99F80040DFF884801D4E0134272CB0
:10D670008ABF4FF0000A5FFA84FA5446AB462B7813
:10D68000A34216D1FFF7E2FB40281FDC33791B06CB
:10D69000F5D59BF800300133272B86BF00221346B7
:10D6A000DAB218F80330DBB2F3712A702B78A34298
:10D6B000E8D00C490A4BFFB208F804700120AC22F4
:10D6C000087089F800A0DA70BDE8F88FFF28D6DD71
:10D6D00001F06AFBD3E700BFF49FFF1FF19FFF1F1C
:10D6E00000C00640F09FFF1FF89FFF1F889FFF1F8D
:10D6F0001C4BDFF894C01A681B49F0B542F4805205
:10D700001A4D1A60DFF884E0194F1A4E1A4C0023A4
:10D710008CF800304FF451722B701F2840F21335F3
:10D720008EF800303B70337025600A6012D81946BD
:10D730000124124A124D11701248547000212C27F6
:10D74000402693724FF4003491701174D7702E708C
:10D750000460F0BDC0F34431C0F3471400F01F0370
:10D76000E7E700BF348004400CC00440859FFF1FE2
:10D77000F19FFF1FF09FFF1F08C0044000C006403C
:10D7800031E400E004E100E0849FFF1FF89FFF1FE9
:10D79000034B1B68DB0401D5FFF758BF704700BF80
:10D7A0003480044010B5044C237823B101F0FCFA16
:10D7B0002378002BFAD110BDF09FFF1F054A064BBE
:10D7C00010781B78C0B2DBB2984238BF4030C01A24
:10D7D000704700BF849FFF1F859FFF1F30B42B4BF6
:10D7E0001A7994061FD52A48DA7903782949013332
:10D7F0003F2B0978C8BF00238B42D2B203D0264CFE
:10D80000D9B2E2540170254A116861B1244A1278F4
:10D81000D2B2934236BFC2F140029B1A9B18272B0B
:10D82000C4BF01230B70194AD378DBB2180611D498
:10D830005A060DD5154B1B795B0609D5194B1A49AC
:10D840001B6800220A7003B11A70104B2C22DA7088
:10D8500030BC704711790906EAD5144910480C7894
:10D860000178C9B28C420DD04A1C272A84BF0021FE
:10D870000A460F4D054C98BFD1B2AA5CD2B2E271F4
:10D880000170D5E76C21D170D2E700BF00C006401F
:10D89000849FFF1F859FFF1FB09FFF1F809FFF1F5B
:10D8A000F19FFF1FF49FFF1FF09FFF1FF89FFF1FB7
:10D8B000889FFF1F21282FD8184B195CFF292BD0D8
:10D8C000174B184ADFF870C003EBC000F0B543688F
:10D8D000DFF868E0144F154D154E00241C60DEF88B
:10D8E0000030012043F020038840CEF8003014605F
:10D8F0004FF4A07338602E60C2F800C0013BFDD128
:10D9000013689B05FCD42023013BFDD1094B09B2D0
:10D9100033F8110080B2F0BD00207047603C010078
:10D92000503B0100005004400850044004500440A3
:10D93000000002030051044080014A003880044086
:10D94000431E032B14D872B60A4951F8230068B15C
:10D9500070B4094C058834F81320466841F82360F8
:10D96000521B24F8132062B670BC704762B6704731
:10D970000020704754A0FF1F98A2FF1F0138032802
:10D980000BD872B6074B53F8203043B100205B68C8
:10D990000130002BFBD162B670470020704718465B
:10D9A000F9E700BFA8A0FF1F30B472B62B4A137866
:10D9B0001D0706D52A4B196A002936D0996A002915
:10D9C00041D053781C0706D5254B196C00293ED051
:10D9D000996C002939D09378190705D5204B196E19
:10D9E000002936D0996E89B1D3781B0707D51C4B17
:10D9F000D3F880207AB3D3F8882011213AB162B6E7
:10DA0000184B00221A7030BC00F04ABE0D21154C94
:10DA1000154D227843F8315003EBC1030830013A29
:10DA20005860227062B630BC704704220D4C0F4D16
:10DA3000217843F8325003EBC20308304A1E586085
:10DA4000227062B6EFE70521E1E70921DFE708224E
:10DA5000ECE70C22EAE71022E8E700BF843C010073
:10DA60000080FF1FD1A0FF1FC800400088004000B9
:10DA7000431E032B1DD81B4A400140F0100030B458
:10DA8000104472B6184CE25C032A1BD8DFE802F09F
:10DA90000212151703220D88E25410F0080F14BF6C
:10DAA000C823882343EA054308310360416062B616
:10DAB00030BC704708300222EDE70522EBE7083062
:10DAC0000422E8E7094A52F8230038B1084A52F81C
:10DAD0002300416042F8231062B6E9E742F82310C0
:10DAE000034AF7E70080FF1FE0A0FF1FA8A0FF1F69
:10DAF000B8A0FF1F00BE70472DE9F04FDFF818B344
:10DB0000DFF818A387B044E0AD4F4FEA930807EB66
:10DB1000C809013ED9F8042003F00803F6B2A2F1C7
:10DB2000080003F0FF04002B40F0018157F8383063
:10DB30001B0C99B222F8081C002B00F0EF80A14BBF
:10DB400022F8064C42F8044C53F82620002A00F034
:10DB5000CF819D4D55F8263058609C4C45F82600E5
:10DB600034F81630194424F8161000F079FD002816
:10DB700000F0C281964A974B19F0080F00F1080097
:10DB800018BF1346C9F8040047F8383008238BF84B
:10DB900000309BF80040E4B265071CD58E4B1B7823
:10DBA000B3B18E490A7802F0FF0322B1013BDBB228
:10DBB0000B7003B900BE8A490A7802F0FF032AB14C
:10DBC000013BDBB20B70002B00F0688100F066FEB9
:10DBD00004238BF8003004F0080303F0FF02002B4D
:10DBE00000F0C9809AF80030DBB21E098CD19A0887
:10DBF000DFF8CC9159F8321009EBC200C1F3830170
:10DC0000013940680C2900F28580DFE801F07A7A5A
:10DC10008383838383834683838307000168714DF5
:10DC20004068714F714E6860296088B240F281612E
:10DC30000024674B49F832304FF0010E88423C60B7
:10DC4000C9F81040C9F8184086F800E05C4A00F2B4
:10DC5000E780B0F5D06F80F01B82B0F5817F00F0D7
:10DC6000D98100F26981802800F02A82822840F060
:10DC7000D781A98801F07F01042900F2D1815C4895
:10DC80005C4A890008441470547001788C0740F194
:10DC9000608382F800E0022173E1534F3A682AB3AF
:10DCA000554B524E554819883478057840298E4690
:10DCB00045F0020828BF4FF0400E002C84F001040C
:10DCC0003470CEEB01010CBF8824C82409EBC806D0
:10DCD00089B285F0010544EA0E447260198049F862
:10DCE000384072440570002965D03A603D4B1A886F
:10DCF000B2F5A06F0ED100219A785970404B1A707E
:10DD000008E038493F4C0D68A54200F09880304942
:10DD100049F832103C4A0123137037E72C4A2D4B47
:10DD200019F0080F18BF134647F838302EE700F0F7
:10DD3000B7FC364A364952F82630002B00F0E38013
:10DD400058688C5D42F8260003F10802C9F80420E7
:10DD5000032C05D8DFE804F02C02292602228A557C
:10DD60001A8819F0080F0CBF8823C82343EA02431E
:10DD700047F838300AE7E00700F19380210600F108
:10DD8000D180A20706D5234A234913780220DBB2AB
:10DD900013700870E30602D51F4B10221A7007B0EB
:10DDA000BDE8F08F04228A55DAE705228A55D7E7C5
:10DDB00003228A55D4E7BEF1400F18BF002294E732
:10DDC0000080FF1F54A0FF1F00A0FF1F98A2FF1F8D
:10DDD000C800400088004000DCA0FF1F65A0FF1FB6
:10DDE00050A1FF1FC8A0FF1FFC9FFF1F64A0FF1FC3
:10DDF000C0200740D4A0FF1F10A0FF1FD0A0FF1F0E
:10DE0000982007402109000394200740A8A0FF1F85
:10DE1000E0A0FF1F88200740802007409020074097
:10DE2000B0F5106F00F07C8140F2A38040F6211223
:10DE3000904240F07B82A54A012313706AE74C6848
:10DE4000A3498C427FF463AF0178A9297FF45FAFC7
:10DE5000417845297FF45BAF8178C2297FF457AFC1
:10DE6000C1786B297FF453AF9A489B4E0178347880
:10DE700081F00105002C41F0020105700CBF8820E3
:10DE8000C82084F0010449F8310009EBC10193482E
:10DE90003470002505244D60047038E700F064FFFD
:10DEA00094E68F4B89488B491A614FF0020E80F837
:10DEB00000E08C4F0A708C49196099608B4E8C4D34
:10DEC0008C4C9A610D213970FF213170DFF84CE2E2
:10DED00029702270884D894A8EF800109F270124EE
:10DEE00006F8047C5D600470DA6007B0BDE8F08F6E
:10DEF00043F82600824D30E6824A47F8380013780E
:10DF00000133137042E68B5D032B00F2BA8001A24D
:10DF100052F823F08DDB00008DDB00006DDF000088
:10DF200067DF00006F49724B80220D2008701A7065
:10DF3000A2077FF52FAF26E740F20232904240F071
:10DF4000ED81AA8802F07F02042A69D86D88002D2D
:10DF500066D16449CDF804E0920011440A7842F099
:10DF600002020A70C1E101238B550FE600238B5595
:10DF70000CE6B0F5086F53D16349644A0978117013
:10DF80007146ED888D4280F0E88252480478402D39
:10DF9000AE4644F0020C28BF4FF0400E02EB0E03D9
:10DFA00009EBCC01029301234A604FEA0E48CEEB05
:10DFB000050101930025C82242EA080384F001020A
:10DFC00049F83C3035700270DFF814C1424BDFF87D
:10DFD000048149BBBEF1400F7FF42DAF42F0020C2B
:10DFE00009EBCC03029ADFF8F8E05A608DBB0D0410
:10DFF00045F088059DF804304EF83C500A443370D3
:10E000000470134640297FF416AF0021404A3B605C
:10E01000118010E7AA8802F07F02042A40F28B8167
:10E02000304A0F23137006E74029D7D942F0020285
:10E030000CEBC200029E4660BDB19DF8045035480D
:10E040001D703346403988F8004040334CF83200A8
:10E05000DCE79DF8043033700D04029B047045F03A
:10E06000C8050B444EF83C50CCE79DF804501D7099
:10E07000029B1D4888F80040403940334CF832007C
:10E08000C4E719F0080F0CBF022303238B557DE56D
:10E0900021494A68002AC3D06C88B5F804E003E03F
:10E0A0000C314A68002ABBD00B88A342F8D14B88B8
:10E0B0007345F5D1240A032C0CBF1178098960E758
:10E0C000124A0221147054705BE700BF942007408D
:10E0D00001000400D0A0FF1F64A0FF1F65A0FF1F68
:10E0E0000080FF1FC02007408800400088200740B4
:10E0F000802007409820074014A0FF1F68A0FF1F42
:10E1000000A0FF1FD1A0FF1FDCA0FF1FD4A0FF1F96
:10E1100010A0FF1FC8004000883C01008C20074071
:10E12000B248116AAC7804700C0600F19881D9F8F5
:10E130002820AF49100600F1DB81D9F83020AC4926
:10E14000120600F1D081D9F83820A949130600F150
:10E15000C581D9F84020A649150600F1BA81D9F841
:10E160004820A349140600F1AF81D9F85020A049F6
:10E17000100600F1A481D9F858209D49120600F13B
:10E180009981D9F860209A49130600F18E81D9F857
:10E1900068209749150600F18381D9F870209449C9
:10E1A000140600F17881D9F878209149100600F121
:10E1B0006D81D9F880208E49120600F16181D9F86D
:10E1C00088208B49130600F15581D9F890208849A1
:10E1D000150600F14981D9F898208549140600F107
:10E1E000FF808448844A854901908548854D864C46
:10E1F000049700230596029580460F4616461D4655
:10E200000394306828B1446800F04AFA2046002C94
:10E21000F9D100233360029B38681A46002342F884
:10E22000253028B1446800F03BFA2046002CF9D193
:10E2300000223A60019A98F800301146002241F815
:10E24000042B039A0191023B4FF0000122F81510B4
:10E25000032B07D8DFE803F05D025D024FF00103F6
:10E2600088F800300135042D06F1040607F1040793
:10E2700008F10108C5D1654C654D2278654B049FB6
:10E28000059E0021100729701A7000F192806249E2
:10E2900062780A700021C9F83010C9F838101107E7
:10E2A000DFF84C816ED4A2785C49DFF844810A70B3
:10E2B00000211207C9F85010C9F858104BD4E27861
:10E2C00057494B4C0A7013074FF00001C9F8701002
:10E2D000C9F8781000F1AE8033780193002283F002
:10E2E0000105C9F89020C9F89820002102918846BC
:10E2F0008E460A464B48047844F0020C09EBCC03E6
:10E300000393019B002B039B5A600CBF8822C822F9
:10E3100052E64FF0000388F80030A3E7B0F5A06F95
:10E320007FF47EAE012300250193DEE740F6212233
:10E330009042F7D074E66D88002D7FF471AE3A49B3
:10E34000CDF804E0920011440A7822F002020A702B
:10E35000CBE7022115E600F083F9002800F0EB80FE
:10E360000830324AC8F86400C8F8602000F078F934
:10E37000002800F0DA8008302D4AC9F86C00C9F88E
:10E3800068209CE700F06CF9002800F0E08008307D
:10E39000264AC8F84400C8F8402000F061F9002877
:10E3A00000F0CF800830224AC9F84C00C9F8482054
:10E3B00079E700F055F9002800F0A58008301B4AE5
:10E3C000C9F82400C9F8202000F04AF9002800F01C
:10E3D00094800830164AC9F82C00C9F8282056E75E
:10E3E000D1F89C00083800F05BF9FAE6DCA0FF1FCA
:10E3F0000080FF1FB8A0FF1F54A0FF1FA8A0FF1F91
:10E40000E0A0FF1F00A0FF1F98A2FF1F843C010097
:10E41000D1A0FF1FC4200740C8200740CC200740E0
:10E42000D0200740D0A0FF1FC02007408800400038
:10E43000C800400000F014F9002870D008304F4A9E
:10E44000C4F88400C4F8802000F00AF9002860D0E5
:10E4500008304B4AC9F88C00C9F888203CE7506A5C
:10E46000083800F01DF962E6D1F89400083800F091
:10E4700017F9B0E6D1F88C00083800F011F9A4E6DD
:10E48000D1F88400083800F00BF998E6C86F083816
:10E4900000F006F98DE6486F083800F001F982E6D1
:10E4A000C86E083800F0FCF877E6486E083800F0CF
:10E4B000F7F86CE6C86D083800F0F2F861E6486DD0
:10E4C000083800F0EDF856E6C86C083800F0E8F8B7
:10E4D0004BE6486C083800F0E3F840E6C86B0838B3
:10E4E00000F0DEF835E6486B083800F0D9F82AE687
:10E4F000C86A083800F0D4F81FE62A78C9F828005E
:10E5000001322A70C3E62A78C9F8200001322A7045
:10E510005AE72A78C9F8880001322A70DCE62A789E
:10E52000C4F8800001322A708EE72A78C9F86800A2
:10E5300001322A70C3E62A78C8F8600001322A70D6
:10E5400014E72A78C9F8480001322A70ABE62A7825
:10E55000C8F8400001322A701FE740298E4628BFC4
:10E560004FF0400E02EB0E0302930123CEEB0101AC
:10E570004FEA0E4800250193BCE600BF880040002A
:10E58000C8004000F8B500F08FFD294B29482A4CFF
:10E590002A4F2B4DDFF8BCC0DFF8BCE0294E00222B
:10E5A0001A605A609A60DA601A615A619A61DA6197
:10E5B0001A625A629A62DA621A635A639A63DA6377
:10E5C0001A645A649A64DA641A655A659A65DA6557
:10E5D0001A665A669A66DA661A675A679A67DA6737
:10E5E000C3F880200168C3F8842041F480210160D1
:10E5F000C3F307212170C3F30740134938701B0E82
:10E600002B70FF238CF80030104D8EF8003010482E
:10E610000B700123337084F8642070264FF400746B
:10E62000102207F82C3C2E70046081F8F820F8BD09
:10E630000080FF1F348004409C200740B02007402A
:10E64000B4200740942007401020074049E400E030
:10E6500008E100E08020074088200740704700BFA5
:10E6600072B60D480268B2FA82F30F2B10DC4FF03D
:10E670000041D94022EA0102026062B6074803EB7A
:10E68000C303DB00C2180021C1501046516070471F
:10E6900062B60020704700BFA492FF1FBC83FF1F1B
:10E6A0000D4B0E4AC31AA2FB03231B090F2B0CD8D8
:10E6B0000B4A127852B972B60A484FF0004102680C
:10E6C00021FA03F31A43026062B67047064A1278D1
:10E6D000002AF0D0FFF768B9BC83FF1F398EE338FA
:10E6E000D1A0FF1FA492FF1FDCA0FF1F38B50E4B67
:10E6F0000E4C1B68218805468BB1B1F5917F05D280
:10E700000B4A4B1C55549BB2238038BD002208484D
:10E7100098470021064A55540123238038BDB1F59E
:10E72000917FEDD338BD00BF08A1FF1FA2A2FF1F3C
:10E73000A8A2FF1F2DE9F843214E224F3168012383
:10E7400080463B70B1B1204D4B8801EB8302013311
:10E7500000240F2BC2F808802C7004D84B800023B3
:10E760003B70BDE8F88340230B800320FFF780F95E
:10E770003460F4E7DFF8549099F80030002BF0D0C3
:10E78000114D45F6215408E0013C12D02B7883B995
:10E7900000F00AFB99F800307BB10320FFF7EEF898
:10E7A0000528F1D8FFF75CFF014630600028EBD068
:10E7B000CAE701232B70BDE8F883BDE8F88300BFEA
:10E7C00024A1FF1FF8A0FF1F28A1FF1FDCA0FF1F2F
:10E7D0001201F8B5D5B2A1B3012943D0437804465C
:10E7E00000781B0643EA004040F4704045F0040600
:10E7F0008F1E3043FFF79EFF022F04F1020314D94E
:10E80000053414F8023C14F8032C14F8010C1B0412
:10E8100043EA0223334343EA0060033FFFF78AFFE2
:10E82000022F234604F10304EBD8022F23D0012F3B
:10E830000DD045F4774040F00500BDE8F840FFF703
:10E8400079BF14482843BDE8F840FFF773BF187834
:10E8500045F4770545F0060545EA0020BDE8F84097
:10E86000FFF768BF03780C4845EA03452843BDE835
:10E87000F840FFF75FBF1A78587845F0774545F0C4
:10E88000070545EA022545EA0040BDE8F840FFF7E4
:10E8900051BF00BF06F0F70007F000F738B5084B8E
:10E8A0001C7824B9074D296809B14B8803B938BDD4
:10E8B0009B000B800320FFF7DBF82C6038BD00BF06
:10E8C000F8A0FF1F24A1FF1F2DE9F041AD4E3368D2
:10E8D0000746002B00F092801D885A88910803EBB0
:10E8E00081010432AA428C6842D25A8004F00F0699
:10E8F0004FEA1428A449A6F1080208F00F00C4F357
:10E900000313062A00F101050B701AD9B31E012B5F
:10E910005FFA88F04ED9052E48D0042E00F0A4816D
:10E92000731F022B7FD90F2E0ED1F72842D8F02863
:10E9300002D0964B1B883BB1FFF7D8FE0020BDE804
:10E94000F08127B1BD4202D00020BDE8F081082E41
:10E95000C4F3033300F08780092E11D00A2E40F053
:10E9600094800A2BF0D18A4B8A4A1B68A02181E04F
:10E970001846FFF795FE0420FEF7E2FF3060B5E78A
:10E98000092BE1D1270E00F07B81834B814A1B6864
:10E990009021C4F307461170EDB2FCB2002B00F0D9
:10E9A0009D80224631462846984797E0F02843D973
:10E9B000F72841D0F1380E28C6D801A353F820F02B
:10E9C00077EB00005BEB000049EB000049E9000039
:10E9D00049E900003BEB000049E900001BEC0000A6
:10E9E00049E90000E5EB0000FFEB000023EB00002D
:10E9F00049E900000BEB0000EFEA0000674B1B78D1
:10EA0000002BA1D00420FEF79BFF034630600028B6
:10EA10009AD00588002D7FF460AFFFF741FE356086
:10EA20002846BDE8F081FFF761FEC4F30740FFF719
:10EA30005DFE072E02D1200EFFF758FE534B584AB9
:10EA4000198858481468584D524A017000270E0A18
:10EA5000F0201F802E7010700CB301225348A04785
:10EA60000120BDE8F081082B7FF46EAF504B494A7E
:10EA70001B688021C4F307461170EDB2240E6BB3FE
:10EA8000284622463146984728E00B2E11D10B2B01
:10EA90007FF45AAF474B3F4A1B68B021EAE7464B29
:10EAA0001B68002B00F0FB80404898470120BDE820
:10EAB000F0810C2E40F000810C2B7FF445AF3F4BD2
:10EAC000344A1B68C0211170EDB2C4F30746002B15
:10EAD00000F0C88028463146240E98473849314A0C
:10EAE000314B0D7016701C700120BDE8F081354B64
:10EAF0001B68002B00F0D6809847C4F30746254BCF
:10EB0000EDB2240E83F80080E8E72F4B1B68002B42
:10EB1000F2D12E4B1B68A3B1FE209847C4F30746E1
:10EB2000EDE72B4B1B68002BE6D1284B1B6843B14C
:10EB3000FC209847C4F30746E1E7264B1B68002BEF
:10EB4000DAD1C4F30746DAE7234B1B68C4F3074660
:10EB5000002BD4D030469847D1E7204B1A68002AC2
:10EB6000EFD0260C630C06F07F0003F47E531843AD
:10EB7000F6B29047C3E71A4B1B68C4F30746002B55
:10EB8000E8D1BCE730A1FF1FA6A2FF1FA2A2FF1F72
:10EB90000CA1FF1FA0A2FF1F40A1FF1FDCA0FF1FB1
:10EBA00008A1FF1FA4A2FF1FA5A2FF1FA8A2FF1F6D
:10EBB00038A1FF1F3CA1FF1F20A1FF1FFCA0FF1FCA
:10EBC000A7A2FF1FE8A0FF1FECA0FF1FF0A0FF1FE0
:10EBD0002CA1FF1F1CA1FF1F34A1FF1F04A1FF1FB9
:10EBE00018A1FF1F3F4B1B68002B85D13E4B1B68B4
:10EBF000002BA6D0FA209847C4F307467FE73B4B8B
:10EC00001B68002B7FF478AF374B1B68002B98D024
:10EC1000FB209847C4F3074671E7354B1B68002B70
:10EC20007FF46AAF304B1B68002B8AD0F8209847DE
:10EC3000C4F3074663E70E2B7FF486AE2D4A2E4BB6
:10EC40001268E0211970002A47D0260C610C06F0EA
:10EC50007F0301F47E511943EDB2A1F5005128461E
:10EC60009047F6B2240E39E7FFF740FDC4F30740A2
:10EC7000FFF73CFD200EFFF739FD0020BDE8F081D5
:10EC80001E4B1D4A1B6880211170EDB2C4F307466C
:10EC900083B1314628463A4698473C461EE7012054
:10ECA000BDE8F081104B1B68002B3FF44AAFFF20FA
:10ECB000984746E71C4611E70D2EBCD10D2B7FF47B
:10ECC00043AE0F4B0C4A1B68D0211170EDB2C4F358
:10ECD0000746002B7FF4FEAEC4E7C4F30746EDB24F
:10ECE000240EFBE614A1FF1FF0A0FF1FF4A0FF1FDE
:10ECF000E4A0FF1F00A1FF1FA0A2FF1F38A1FF1F5C
:10ED000010A1FF1F38B5164D2868E0B1018844886E
:10ED1000A14213DD03191B7A83B104F10803C21861
:10ED20000C1B002302E012F8011F21B10133A342A2
:10ED3000F9D1204638BD1C46204638BDFFF7B0FC4F
:10ED40000020286038BD074B1B780BB9002038BD68
:10ED50000220FEF7F5FD28600028D7D1F6E700BFB6
:10ED60004CA1FF1FDCA0FF1F0D4B1B78BBB910B5DA
:10ED70000C4C216803F0FF024B883F2B07DC073364
:10ED80000B4401F1470003F8012F8342FBD14023DC
:10ED90000B800120FEF76CFE0023236010BD70473E
:10EDA00044A1FF1F48A1FF1F38B5224C237803B1AF
:10EDB00038BD01232370FFF7A5FF70BB00F048F8B2
:10EDC00040BB00F0DBF810BBFEF7F8FCE0B9002315
:10EDD0002370EFF30583002BEAD1EFF3108172B6B5
:10EDE000154B1868E0B1154C2278CAB945691D6009
:10EDF00001232370C5B1AA6101B962B60025457728
:10EE0000836898472570D3E700F020F8DFE700F02B
:10EE10001BF8D9E700F016F8D3E7FFF71FFCCDE7A2
:10EE20000029C5D162B638BD054B1D600029E5D16A
:10EE3000E3E700BF51A1FF1F689FFF1F6C9FFF1FEB
:10EE4000649FFF1F704700BF704700BF704700BF3F
:10EE5000054A064B10781B78C0B2DBB2984238BF27
:10EE60004030C01A704700BF58A1FF1F59A1FF1FB3
:10EE7000F0B4384B1A7912F0300F2CD072B6997D5D
:10EE800001F0FF0200293DD062B6334F3349387894
:10EE90000D78334E1C46C0B2EDB2431C402BE179D5
:10EEA00028BF0023AB4202F1FF32C9B21CBFF154AC
:10EEB000184612F0FF02F0D12A4B1B68C2B23A701A
:10EEC0004BB1A84236BFC5F14005401B4019272869
:10EED000C4BF01221A701F49CA78D2B2150616D4CF
:10EEE00052060DD51B4B1B795B0609D51E4B1F49DE
:10EEF0001B6800220A7003B11A70164B3C22DA70AC
:10EF0000F0BC70474022D9795A7462B6E3E70B79B6
:10EF10001C06E5D5164B174E1C783378E4B2DBB2ED
:10EF20009C420ED0144D01E0A3420AD00133402B85
:10EF300028BF00230879E85CC0B2C871087D0728A3
:10EF4000F2D9DBB2034933700B79180644BF7C2336
:10EF5000CB70C5E700A0064058A1FF1F59A1FF1FB5
:10EF60009CA1FF1F54A1FF1FE0A1FF1FDCA1FF1FF9
:10EF7000E4A1FF1FDDA1FF1F5CA1FF1F054A064B97
:10EF800010781B78C0B2DBB2984238BF4030C01A4C
:10EF9000704700BF58A2FF1FEDA1FF1FF0B4384B10
:10EFA0001A7912F0300F2CD072B6997D01F0FF0261
:10EFB00000293DD062B6334F334938780D78334E4F
:10EFC0001C46C0B2EDB2431C402BE17928BF0023A0
:10EFD000AB4202F1FF32C9B21CBFF154184612F025
:10EFE000FF02F0D12A4B1B68C2B23A704BB1A84263
:10EFF00036BFC5F14005401B40192728C4BF012278
:10F000001A701F49CA78D2B2150616D452060DD509
:10F010001B4B1B795B0609D51E4B1F491B68002241
:10F020000A7003B11A70164B3C22DA70F0BC7047BC
:10F030004022D9795A7462B6E3E70B791C06E5D50C
:10F04000164B174E1C783378E4B2DBB29C420ED0DC
:10F05000144D01E0A3420AD00133282B28BF00231E
:10F060000879E85CC0B2C871087D0728F2D9DBB224
:10F07000034933700B79180644BF7C23CB70C5E776
:10F0800000B0064058A2FF1FEDA1FF1F18A2FF1FEE
:10F09000E8A1FF1F5CA2FF1FECA1FF1F60A2FF1FE2
:10F0A00059A2FF1FF0A1FF1F70B584B072B6194BB3
:10F0B000194D1A48702241260F2480211A702E7093
:10F0C0001A460470197013781B06FCD5144B186887
:10F0D00062B6144B144C984298BF00EB800001A913
:10F0E00098BF40000A22FDF7CFFE01A92046002369
:10F0F00011F8012B01333AB10A2B20F8022FF7D176
:10F100001623237004B070BD5B00DBB2237004B023
:10F1100070BD00BF00000240070002400600024030
:10F12000080002407F9698007093FF1FFFFFFFFFCB
:10F130002DE9F043DFF8EC808BB006460F4600F077
:10F1400073F898F90030013304460D4637D0304645
:10F15000394600F0DFF9002831D02BA3D3E9002392
:10F160003046394600F026FE814668BB28A3D3E925
:10F1700000233046394600F0FFFD00B398F9003017
:10F18000254ACDF82090042400200021022BCDE94F
:10F190000467CDE9026700940192CDE906012CD005
:10F1A000684600F0BDF940B3089B1BB101F0AAF915
:10F1B000089B0360DDE906010BB0BDE8F083204643
:10F1C00029460BB0BDE8F083134A98F9003001924C
:10F1D00003210022CDE90467CDE90267009108927E
:10F1E0002BB90E4B4FF06042CDE90623D8E70C490E
:10F1F0000020022BCDE90601D2D101F083F92223B0
:10F200000360D1E7AFF30080EF39FAFE422E86406B
:10F2100051302DD5104987C0F43C0100FFFFEF4766
:10F220000000F07F8693FF1F2DE9F04FB04F21F0D3
:10F230000042BA4283B00C464FEAD17605460DD95A
:10F24000AC4FBA4225D9C1F31303034340F0EF801A
:10F250000EB10020014603B0BDE8F08FA64B9A42E4
:10F2600000F2CC80A54B9A4200F2DE808AA3D3E95B
:10F27000002300F05DF90022A14B00F09BFD002867
:10F2800000F005812846214600229D4B00F050F9F0
:10F29000E1E783A3D3E9002300F08CFD002840F0D0
:10F2A000CB802846214680A3D3E9002300F064FDEB
:10F2B0000028CED1934B284603EBC60821467CA3F9
:10F2C000D3E9002300F0E6FAD8E9002300F030F992
:10F2D00000F07AFD804600F077FA77A3D3E90023A7
:10F2E00006460F4600F0D6FA02460B46284621464F
:10F2F00000F01CF972A3D3E90023CDE900013046E8
:10F30000394600F0C7FA82468B4652465B46DDE935
:10F31000000100F00BF905460C462A462346284614
:10F32000214600F0B7FA68A3D3E9002306460F464A
:10F3300000F0B0FA66A3D3E9002300F0F7F83246F4
:10F340003B4600F0A7FA64A3D3E9002300F0F0F8ED
:10F3500032463B4600F09EFA61A3D3E9002300F059
:10F36000E5F832463B4600F095FA5FA3D3E9002367
:10F3700000F0DEF832463B4600F08CFA02460B46BF
:10F380002846214600F0D2F806460F462846214678
:10F3900032463B46B8F1000F56D000F07BFA3246B9
:10F3A00004460D463B4600204FF0804100F0BEF879
:10F3B00002460B462046294600F096FB02460B46C5
:10F3C0005046594600F0B2F8DDE9002300F0AEF8EF
:10F3D0000B4602464A49002000F0A8F86FF47F73FC
:10F3E00098454FDA08F57A7801EB085100224FF082
:10F3F000B87300F04FFA03B0BDE8F08F424B9A4269
:10F400003FF658AF414BF4002344D3E9002300F00A
:10F410008DF83F4BC6F101081C44CDE90001D4E949
:10F4200000ABC6EB080870E74FF0000875E702462E
:10F430000B4600F07DF80EE717A3D3E90023104632
:10F44000194600F027FA06E700F024FA0022804669
:10F4500089464FF080433046394600F067F802464F
:10F460000B464046494600F03FFB2A46234600F043
:10F470005DF802460B460020214900F057F803B022
:10F48000BDE8F08F01EB085103B0BDE8F08F804676
:10F4900043E700BFAFF300809C7500883CE4377EF3
:10F4A000EF39FAFE422E864051302DD5104987C0E3
:10F4B000FE822B654715F73F0000E0FE422EE63F37
:10F4C000763C7935EF39EA3DD0A4BE726937663EA5
:10F4D000F16BD2C541BDBB3E2CDE25AF6A56113F54
:10F4E00093BDBE166CC1663F3E5555555555C53F3B
:10F4F000412E8640FFFFEF7F422ED63FFFFF2F3E7B
:10F500000000F03FF83C0100B1A2F03F183D0100BF
:10F51000083D010041F0004101F58010C00F704727
:10F520000020704781F0004102E000BF83F00043FB
:10F5300030B54FEA41044FEA430594EA050F08BF8E
:10F5400090EA020F1FBF54EA000C55EA020C7FEA52
:10F55000645C7FEA655C00F0E2804FEA5454D4EBCF
:10F560005555B8BF6D420CDD2C4480EA020281EA99
:10F57000030382EA000083EA010180EA020281EAD1
:10F580000303362D88BF30BD11F0004F4FEA013123
:10F590004FF4801C4CEA113102D0404261EB410132
:10F5A00013F0004F4FEA03334CEA133302D05242B8
:10F5B00063EB430394EA050F00F0A780A4F1010474
:10F5C000D5F1200E0DDB02FA0EFC22FA05F28018AE
:10F5D00041F1000103FA0EF2801843FA05F3594194
:10F5E0000EE0A5F120050EF1200E012A03FA0EFC13
:10F5F00028BF4CF0020C43FA05F3C01851EBE3713D
:10F6000001F0004507D54FF0000EDCF1000C7EEB59
:10F6100000006EEB0101B1F5801F1BD3B1F5001F97
:10F620000CD349085FEA30004FEA3C0C04F10104B6
:10F630004FEA445212F5800F80F09A80BCF1004FDF
:10F6400008BF5FEA500C50F1000041EB045141EA61
:10F65000050130BD5FEA4C0C404141EB010111F462
:10F66000801FA4F10104E9D191F0000F04BF01460D
:10F670000020B1FA81F308BF2033A3F10B03B3F1EB
:10F6800020020CDA0C3208DD02F1140CC2F10C027B
:10F6900001FA0CF021FA02F10CE002F11402D8BFD9
:10F6A000C2F1200C01FA02F120FA0CFCDCBF41EAA5
:10F6B0000C019040E41AA2BF01EB0451294330BD74
:10F6C0006FEA04041F3C1CDA0C340EDC04F1140451
:10F6D000C4F1200220FA04F001FA02F340EA030028
:10F6E00021FA04F345EA030130BDC4F10C04C4F16E
:10F6F000200220FA02F001FA04F340EA030029464E
:10F7000030BD21FA04F0294630BD94F0000F83F497
:10F71000801306BF81F480110134013D4EE77FEA7A
:10F72000645C18BF7FEA655C29D094EA050F08BFC6
:10F7300090EA020F05D054EA000C04BF19461046A7
:10F7400030BD91EA030F1EBF0021002030BD5FEAEB
:10F75000545C05D14000494128BF41F0004130BD13
:10F7600014F580043CBF01F5801130BD01F0004567
:10F7700045F0FE4141F470014FF0000030BD7FEADA
:10F78000645C1ABF194610467FEA655C1CBF0B46D5
:10F79000024650EA013406BF52EA033591EA030FEC
:10F7A00041F4002130BD00BF90F0000F04BF0021E4
:10F7B000704730B54FF4806404F132044FF0000517
:10F7C0004FF0000150E700BF90F0000F04BF002190
:10F7D000704730B54FF4806404F1320410F00045F6
:10F7E00048BF40424FF000013EE700BF42004FEAF1
:10F7F000E2014FEA31014FEA02701FBF12F07F436E
:10F8000093F07F4F81F06051704792F0000F14BF6A
:10F8100093F07F4F704730B54FF4607401F00045AE
:10F8200021F0004120E700BF50EA010208BF704705
:10F8300030B54FF000050AE050EA010208BF7047FA
:10F8400030B511F0004502D5404261EB41014FF463
:10F85000806404F132045FEA915C3FF4DCAE4FF067
:10F8600003025FEADC0C18BF03325FEADC0C18BF4E
:10F87000033202EBDC02C2F1200300FA03FC20FA9F
:10F8800002F001FA03FE40EA0E0021FA02F11444EC
:10F89000C1E600BF70B54FF0FF0C4CF4E06C1CEA01
:10F8A00011541DBF1CEA135594EA0C0F95EA0C0F76
:10F8B00000F0DEF82C4481EA030621EA4C5123EAE9
:10F8C0004C5350EA013518BF52EA033541F4801118
:10F8D00043F4801338D0A0FB02CE4FF00005E1FBCB
:10F8E00002E506F00042E0FB03E54FF00006E1FB15
:10F8F00003569CF0000F18BF4EF0010EA4F1FF0458
:10F90000B6F5007F64F5407404D25FEA4E0E6D4197
:10F9100046EB060642EAC62141EA55514FEAC520A8
:10F9200040EA5E504FEACE2EB4F1FD0C88BFBCF524
:10F93000E06F1ED8BEF1004F08BF5FEA500E50F1D5
:10F94000000041EB045170BD06F0004646EA01019B
:10F9500040EA020081EA0301B4EB5C04C2BFD4EBCD
:10F960000C0541EA045170BD41F480114FF0000EC6
:10F97000013C00F3AB8014F1360FDEBF002001F034
:10F98000004170BDC4F10004203C35DA0C341BDCAE
:10F9900004F11404C4F1200500FA05F320FA04F080
:10F9A00001FA05F240EA020001F0004221F00041B4
:10F9B00010EBD37021FA04F642EB06015EEA430E27
:10F9C00008BF20EAD37070BDC4F10C04C4F1200557
:10F9D00000FA04F320FA05F001FA04F240EA02000A
:10F9E00001F0004110EBD37041F100015EEA430EDB
:10F9F00008BF20EAD37070BDC4F1200500FA05F2FB
:10FA00004EEA020E20FA04F301FA05F243EA020379
:10FA100021FA04F001F0004121FA04F220EA020088
:10FA200000EBD3705EEA430E08BF20EAD37070BDCE
:10FA300094F0000F0FD101F00046400041EB0101AE
:10FA400011F4801F08BF013CF7D041EA060195F090
:10FA5000000F18BF704703F00046520043EB03034A
:10FA600013F4801F08BF013DF7D043EA0603704737
:10FA700094EA0C0F0CEA135518BF95EA0C0F0CD042
:10FA800050EA410618BF52EA4306D1D181EA030188
:10FA900001F000414FF0000070BD50EA410606BF82
:10FAA0001046194652EA430619D094EA0C0F02D1C7
:10FAB00050EA013613D195EA0C0F05D152EA03360C
:10FAC0001CBF104619460AD181EA030101F000412A
:10FAD00041F0FE4141F470014FF0000070BD41F073
:10FAE000FE4141F4780170BD70B54FF0FF0C4CF44D
:10FAF000E06C1CEA11541DBF1CEA135594EA0C0F6C
:10FB000095EA0C0F00F0A7F8A4EB050481EA030EB8
:10FB100052EA03354FEA013100F088804FEA03339F
:10FB20004FF0805545EA131343EA12634FEA02226D
:10FB300045EA111545EA10654FEA00260EF000412E
:10FB40009D4208BF964244F1FD0404F5407402D280
:10FB50005B084FEA3202B61A65EB03055B084FEA11
:10FB600032024FF480104FF4002CB6EB020E75EB0E
:10FB7000030E22BFB61A754640EA0C005B084FEA36
:10FB80003202B6EB020E75EB030E22BFB61A7546B3
:10FB900040EA5C005B084FEA3202B6EB020E75EBFE
:10FBA000030E22BFB61A754640EA9C005B084FEA76
:10FBB0003202B6EB020E75EB030E22BFB61A754683
:10FBC00040EADC0055EA060E18D04FEA051545EA72
:10FBD00016754FEA06164FEAC30343EA52734FEA1B
:10FBE000C2025FEA1C1CC0D111F4801F0BD141EA94
:10FBF00000014FF000004FF0004CB6E711F4801FF9
:10FC000004BF01430020B4F1FD0C88BFBCF5E06FD8
:10FC10003FF6AFAEB5EB030C04BFB6EB020C5FEAE8
:10FC2000500C50F1000041EB045170BD0EF0004E3D
:10FC30004EEA113114EB5C04C2BFD4EB0C0541EA6F
:10FC4000045170BD41F480114FF0000E013C90E66C
:10FC500045EA060E8DE60CEA135594EA0C0F08BF30
:10FC600095EA0C0F3FF43BAF94EA0C0F0AD150EA2F
:10FC700001347FF434AF95EA0C0F7FF425AF1046C2
:10FC800019462CE795EA0C0F06D152EA03353FF4EA
:10FC9000FDAE1046194622E750EA410618BF52EA67
:10FCA00043067FF4C5AE50EA41047FF40DAF52EA3B
:10FCB00043057FF4EBAE12E74FF0FF3C06E000BFD8
:10FCC0004FF0010C02E000BF4FF0010C4DF804CDE5
:10FCD0004FEA410C7FEA6C5C4FEA430C18BF7FEAA5
:10FCE0006C5C1BD001B050EA410C0CBF52EA430CD3
:10FCF00091EA030F02BF90EA020F0020704710F153
:10FD0000000F91EA030F58BF994208BF90422CBFE1
:10FD1000D8176FEAE37040F0010070474FEA410CDA
:10FD20007FEA6C5C02D150EA013C07D14FEA430CF8
:10FD30007FEA6C5CD6D152EA033CD3D05DF8040B69
:10FD4000704700BF8446104662468C46194663469B
:10FD500000E000BF01B5FFF7B7FF002848BF10F172
:10FD6000000F01BD4DF808EDFFF7F4FF0CBF0120B7
:10FD700000205DF808FB00BF4DF808EDFFF7EAFF33
:10FD800034BF012000205DF808FB00BF4DF808EDEE
:10FD9000FFF7E0FF94BF012000205DF808FB00BFE3
:10FDA0004DF808EDFFF7CEFF94BF012000205DF86D
:10FDB00008FB00BF4DF808EDFFF7C4FF34BF01207A
:10FDC00000205DF808FB00BF4FEA410212F5001267
:10FDD00015D211D56FF47873B3EB625212D94FEA92
:10FDE000C12343F0004343EA505311F0004F23FA7C
:10FDF00002F018BF404270474FF00000704750EAD1
:10FE0000013005D111F0004008BF6FF0004070478D
:10FE10004FF00000704700BF4FEA4102B2F1E043EB
:10FE200024BFB3F5001CDCF1FE5C0DD901F0004CE1
:10FE30004FEAC0024CEA5070B2F1004F40EB830031
:10FE400008BF20F00100704711F0804F21D113F15D
:10FE50003872BCBF01F00040704741F480114FEA96
:10FE60005252C2F11802C2F1200C10FA0CF320FA1F
:10FE700002F018BF40F001004FEAC1234FEAD3233C
:10FE800003FA0CFC40EA0C0023FA02F34FEA4303A6
:10FE9000CCE77FEA625307D150EA01331EBF4FF02F
:10FEA000FE4040F44000704701F0004040F0FE404A
:10FEB00040F40000704700BF80F0004002E000BF47
:10FEC00081F0004142001FBF5FEA410392EA030F45
:10FED0007FEA226C7FEA236C6AD04FEA1262D2EB8F
:10FEE0001363C1BFD218414048404140B8BF5B4294
:10FEF000192B88BF704710F0004F40F4000020F02D
:10FF00007F4018BF404211F0004F41F4000121F042
:10FF10007F4118BF494292EA030F3FD0A2F101028C
:10FF200041FA03FC10EB0C00C3F1200301FA03F1CA
:10FF300000F0004302D5494260EB4000B0F5000FED
:10FF400013D3B0F1807F06D340084FEA310102F1AC
:10FF50000102FE2A51D2B1F1004F40EBC25008BF5E
:10FF600020F0010040EA03007047490040EB000028
:10FF700010F4000FA2F10102EDD1B0FA80FCACF157
:10FF8000080CB2EB0C0200FA0CF0AABF00EBC25056
:10FF900052421843BCBFD0401843704792F0000F44
:10FFA00081F4000106BF80F400000132013BB5E797
:10FFB0004FEA41037FEA226C18BF7FEA236C21D00D
:10FFC00092EA030F04D092F0000F08BF0846704772
:10FFD00090EA010F1CBF0020704712F07F4F04D140
:10FFE000400028BF40F00040704712F100723CBF53
:10FFF00000F50000704700F0004343F0FE4040F47D
:020000021000EC
:10000000000070477FEA226216BF08467FEA23633A
:100010000146420206BF5FEA412390EA010F40F425
:10002000800070474FF0000304E000BF10F0004371
:1000300048BF40425FEA000C08BF704743F0964358
:1000400001464FF000001CE050EA010208BF704773
:100050004FF000030AE000BF50EA010208BF7047FA
:1000600011F0004302D5404261EB41015FEA010C0F
:1000700002BF84460146002043F0B64308BFA3F107
:100080008053A3F50003BCFA8CF2083AA3EBC253E9
:1000900010DB01FA02FC634400FA02FCC2F1200208
:1000A000BCF1004F20FA02F243EB020008BF20F03F
:1000B0000100704702F1200201FA02FCC2F12002A5
:1000C00050EA4C0021FA02F243EB020008BF20EA9A
:1000D000DC7070474FF0FF0C1CEAD0521EBF1CEAC8
:1000E000D15392EA0C0F93EA0C0F6FD01A4480EAB6
:1000F000010C400218BF5FEA41211ED04FF000639F
:1001000043EA501043EA5111A0FB01310CF00040CA
:10011000B1F5000F3EBF490041EAD3715B0040EAF0
:10012000010062F17F02FD2A1DD8B3F1004F40EBC0
:10013000C25008BF20F00100704790F0000F0CF093
:10014000004C08BF49024CEA502040EA51207F3A57
:10015000C2BFD2F1FF0340EAC250704740F4000032
:100160004FF00003013A5DDC12F1190FDCBF00F023
:1001700000407047C2F10002410021FA02F1C2F1D1
:10018000200200FA02FC5FEA310040F1000053EA6D
:100190004C0308BF20EADC70704792F0000F00F0BB
:1001A000004C02BF400010F4000F013AF9D040EAC1
:1001B0000C0093F0000F01F0004C02BF490011F455
:1001C000000F013BF9D041EA0C018FE70CEAD15353
:1001D00092EA0C0F18BF93EA0C0F0AD030F0004CD3
:1001E00018BF31F0004CD8D180EA010000F0004087
:1001F000704790F0000F17BF90F0004F084691F045
:10020000000F91F0004F14D092EA0C0F01D142027E
:100210000FD193EA0C0F03D14B0218BF084608D147
:1002200080EA010000F0004040F0FE4040F4000091
:10023000704740F0FE4040F4400070474FF0FF0C24
:100240001CEAD0521EBF1CEAD15392EA0C0F93EA6B
:100250000C0F69D0A2EB030280EA010C49024FEABD
:10026000402037D04FF0805343EA111143EA101376
:100270000CF000408B4238BF5B0042F17D024FF42E
:10028000000C8B4224BF5B1A40EA0C00B3EB510F09
:1002900024BFA3EB510340EA5C00B3EB910F24BFF2
:1002A000A3EB910340EA9C00B3EBD10F24BFA3EB77
:1002B000D10340EADC001B0118BF5FEA1C1CE0D13F
:1002C000FD2A3FF650AF8B4240EBC25008BF20F0F2
:1002D000010070470CF0004C4CEA50207F32C2BF46
:1002E000D2F1FF0340EAC250704740F400004FF0E3
:1002F0000003013A37E792F0000F00F0004C02BF14
:10030000400010F4000F013AF9D040EA0C0093F0DD
:10031000000F01F0004C02BF490011F4000F013B37
:10032000F9D041EA0C0195E70CEAD15392EA0C0F9F
:1003300008D142027FF47DAF93EA0C0F7FF470AFD7
:10034000084676E793EA0C0F04D14B023FF44CAF1A
:1003500008466EE730F0004C18BF31F0004CCAD1AF
:1003600030F000427FF45CAF31F000437FF43CAFEB
:100370005FE700BF4FF0FF3C06E000BF4FF0010C0D
:1003800002E000BF4FF0010C4DF804CD4FEA4002EF
:100390004FEA41037FEA226C18BF7FEA236C11D039
:1003A00001B052EA530C18BF90EA010F58BFB2EBEC
:1003B000030088BFC81738BF6FEAE17018BF40F06C
:1003C000010070477FEA226C02D15FEA402C05D120
:1003D0007FEA236CE4D15FEA412CE1D05DF8040BA5
:1003E000704700BF844608466146FFE70FB5FFF738
:1003F000C9FF002848BF10F1000F0FBD4DF808EDF0
:10040000FFF7F4FF0CBF012000205DF808FB00BFE0
:100410004DF808EDFFF7EAFF34BF012000205DF83A
:1004200008FB00BF4DF808EDFFF7E0FF94BF012087
:1004300000205DF808FB00BF4DF808EDFFF7D2FF84
:1004400094BF012000205DF808FB00BF4DF808EDC7
:10045000FFF7C8FF34BF012000205DF808FB00BF94
:100460004FEA4002B2F1FE4F0FD34FF09E03B3EBC1
:1004700012620DD94FEA002343F0004310F0004F01
:1004800023FA02F018BF404270474FF00000704757
:1004900012F1610F01D1420205D110F0004008BFF6
:1004A0006FF0004070474FF00000704742000ED2DE
:1004B000B2F1FE4F0BD34FF09E03B3EB126209D49F
:1004C0004FEA002343F0004323FA02F070474FF055
:1004D0000000704712F1610F01D1420202D14FF0CA
:1004E000FF3070474FF00000704700BF0B460146D9
:1004F000184600F001B800BF13460A460146022024
:1005000000F0B0BE014B1868704700BFB097FF1FE6
:1005100070B50F4E0F4D761BB61018BF002405D0D6
:10052000013455F8043B9847A642F9D10A4E0B4DC9
:10053000761B03F0FBFBB61018BF002406D0013475
:1005400055F8043B9847A642F9D170BD70BD00BF75
:10055000383D0100383D01004C3D0100383D0100AF
:10056000024B0146186800F00BB800BFB097FF1FA0
:10057000024B0146186800F039BF00BFB097FF1F5B
:100580002DE9F04F01F10B05162D83B0064640F220
:100590009F8035F0070500F1BF80A94200F2BC80C2
:1005A00000F058FBB5F5FC7FC0F09C826B0A00F0B0
:1005B000BA80042B00F28381A80900F1390E4FEABA
:1005C0004E033830C44F07EB8303A3F108015C6886
:1005D000A14207D1ACE0002A80F2AC80E468A142DD
:1005E00000F0A680636823F003035A1B0F2AF2DD94
:1005F000B9493C6901F1080E744500F0B3816368A4
:1006000023F003035A1B0F2A00F39981002AC1F833
:1006100014E0C1F810E080F29E80B3F5007F80F016
:100620006781DB0803F1010C01229B1002FA03F33E
:100630004A6851F83C80C4F8088001EBCC091A43A1
:10064000A9F10803E3604A6041F83C40C8F80C4057
:10065000831001249C40944200F28A80144206D107
:1006600020F003006400144200F10400FAD007EB0C
:10067000C009CC468046DCF80C108C4507D173E1EC
:10068000002A80F28181C9688C4500F06D814B6839
:1006900023F003035A1B0F2AF2DD0C46D1F80CC0DD
:1006A00054F8088F4B1945F001054D6042F00101E7
:1006B000C8F80CC03046CCF808807B613B61C3F8B9
:1006C0000CE0C3F808E059609A5000F0C5FA1FE04A
:1006D000102921D800F0BEFA1025062302207E4FF3
:1006E00007EB8303A3F108025C68944200F04581A4
:1006F0006368E168A56823F00303234430465A6821
:10070000E96042F001028D605A6000F0A5FA0834F9
:10071000204603B0BDE8F08F00240C232046336050
:1007200003B0BDE8F08F80234FF0400E3F2049E733
:1007300070465DE72344E1685A68A56842F001020B
:10074000E96030468D605A6000F086FA0834204631
:1007500003B0BDE8F08F234430465A6842F00102EE
:100760005A6000F079FA0834204603B0BDE8F08FF3
:10077000BC68636823F00308A84504D3C5EB0803ED
:100780000F2B00F38C80554BDFF860911A68D9F875
:10079000003001332A4404EB080A00F0608102F5BE
:1007A00080520F3222F47F6222F00F02114630464F
:1007B000019200F04BFCB0F1FF3F8346019A00F03C
:1007C0005881824500F2FC80454B1968DA45114496
:1007D000196000F05381D9F80000DFF810E1013012
:1007E0001BBFCAEB0B0A5144CEF800B019601BF0D6
:1007F000070100F01781C1F10800C1F58051834461
:1008000008315A44C2F30B02C2EB01094946304693
:10081000019300F01BFC431C019B00F03F81CBEBDC
:1008200000024A4442F001021968C7F808B049447E
:10083000BC42CBF804201960DFF8A49016D0B8F1C0
:100840000F0F40F2FD806268A8F10C0323F007034C
:10085000E01802F001024FF0050E1A430F2B626000
:10086000C0F804E0C0F808E000F21C811D4BBC6831
:100870001A68914288BF19601B4B1A6891426268DE
:1008800088BF196022F003029542A2EB050301D84C
:100890000F2B04DC304600F0DFF9002438E7621942
:1008A00043F0010345F0010565603046BA605360CE
:1008B00000F0D2F90834204603B0BDE8F08F142BC5
:1008C00071D9542B00F2A480280B00F16F0E4FEA6F
:1008D0004E036E3076E600BFB497FF1F6CA2FF1F79
:1008E00070A2FF1F68A2FF1F64A2FF1FC09BFF1F13
:1008F0005A0A042A5ED9142A00F2B38002F15C017C
:1009000049005B3207EB810C57F82110DFF8DC81DE
:10091000ACF1080C8C4500F088804A6822F0030294
:10092000934202D289688C45F7D1D1F80CC07A681D
:10093000C4F80CC0A160CCF80840CC6088E663190C
:1009400042F0010745F00105656030464B610B61DF
:10095000C3F80CE0C3F808E05F609A50083400F078
:100960007BF9D5E64A6873E608F1010818F0030F31
:100970000CF1080C7FF47FAE30E0DC68A34208BFC6
:1009800002303FF435AEB3E60B440C465A68C968F2
:1009900054F8085F42F001025A603046E9608D6009
:1009A00000F05AF9B4E603F15C0E03F15B004FEA84
:1009B0004E0307E69A0902F1390149003832A1E7EE
:1009C000BC424A4B3FF400AF9C68626822F00302CD
:1009D0005AE759F80839994540F0828010F0030F22
:1009E00000F1FF30F5D17B6823EA04037B606400EB
:1009F0009C423FF6BDAE002C3FF4BAAE1C424046CE
:100A00007FF435AE64001C4200F10400FAD02EE6FB
:100A1000B3F5AA7F18D8E80B00F1780E4FEA4E0321
:100A20007730CFE54FF48051EBE60121D8F8043060
:100A3000921001FA02F21A43C8F80420614677E7DF
:100A40000123CBF8043025E740F25452934220D8DA
:100A5000A80C00F17D0E4FEA4E037C30B2E5103257
:100A6000A4E6542A26D81A0B02F16F0149006E320F
:100A700048E7BC68626822F0030205E7CAF30B008E
:100A800000287FF4A8AE4244BB6842F001025A60DD
:100A9000ECE6FE234FF07F0E7E2093E501224FF01F
:100AA0000009C1E604F10801304600F09FFCD9F8C6
:100AB0000010DBE6B2F5AA7F05D8DA0B02F1780167
:100AC000490077321EE740F254518A4205D89A0C09
:100AD00002F17D0149007C3214E7FE217E2211E7FC
:100AE0007B6884E7E808431C5B00F8E5B497FF1FC8
:100AF0008842F0B50DD98B1898420AD28118002A85
:100B000051D09A1A13F8014D01F8014D9342F9D1D1
:100B1000F0BD0F2A48D941EA00039B0746D100F1F6
:100B2000100401F11003154653F8106C44F8106CD2
:100B300053F80C6C44F80C6C53F8086C44F8086CCF
:100B4000103D53F8046C44F8046C0F2D03F11003AE
:100B500004F11004E8D8A2F1100323F00F0302F00F
:100B60000F0E1033BEF1030F1944034421D91E1F89
:100B70000D467446043C55F8047B46F8047F032C6C
:100B8000F8D8AEF1040424F00304043423442144CF
:100B900002F0030262B1013B0A4411F8014B03F871
:100BA000014F8A42F9D1F0BD0346F3E70346F2E76D
:100BB000F0BD7246EEE700BF70B4840746D0541E05
:100BC000002A41D0CDB2034602E0621EE4B31446CF
:100BD00003F8015B9A07F8D1032C2ED9CDB245EA70
:100BE00005250F2C45EA054519D903F110022646C3
:100BF000103E0F2E42F8105C42F80C5C42F8085C84
:100C000042F8045C02F11002F2D8A4F1100222F0C2
:100C10000F0204F00F041032032C13440DD91E46AA
:100C20002246043A032A46F8045BFAD8221F22F02F
:100C300003020432134404F003042CB1C9B21C446F
:100C400003F8011BA342FBD170BC70471446034656
:100C5000C2E700BF704700BF704700BF024B0A46A3
:100C60000146186800F002B8B097FF1F2DE9F04F59
:100C7000174683B0002900F0C1800E46814607F177
:100C80000B05FFF7E7FF56F804EC162D2EF00304D2
:100C9000A6F1080840D810221546AF4241D8944228
:100CA00075DAC94B996808EB04008842416800F086
:100CB000D98021F0010303445B68DB077DD51EF07A
:100CC000010F35D039464846FFF75AFC0746E0B1D8
:100CD00056F8043C23F001034344A0F108029A4271
:100CE00000F04481221F242A00F23181132A00F2ED
:100CF0000481034632461168196051685960926850
:100D00009A603146484600F071FB4846FFF7A4FF61
:100D1000384603B0BDE8F08F25F00705002D2A46C0
:100D2000BBDA0C230020C9F8003003B0BDE8F08F17
:100D300056F8083CC3EB080ADAF8043023F0030C39
:100D400004EB0C039342BDDB5746DAF80C1057F85E
:100D5000080F221F242AC160886000F21781132A1D
:100D600040F212813168CAF808107168CAF80C1094
:100D70001B2A00F22B8108360AF11002316811603B
:100D800071685160B16891603E461C46D046631B55
:100D90000F2B1DD8D8F8043003F00103234344443B
:100DA000C8F80430636843F0010363604846FFF706
:100DB00053FF304603B0BDE8F08F21F0030121441A
:100DC000914221DBC36882680C46D3609A60DEE7FB
:100DD000D8F8042008EB050102F00102154343F0A6
:100DE00001020B44C8F804504A605A6842F00102FC
:100DF00008315A60484600F0F9FAD7E7114603B0C7
:100E0000BDE8F04FFFF7BCBB1EF0010F7FF45AAFF7
:100E100056F8083CC3EB080ADAF8043023F0030C58
:100E200001EB0C0E96458BDBC36882685746D36096
:100E30009A6057F8081FDAF80C30CB60221F242A7A
:100E4000996000F29980132A62D93368CAF8083091
:100E50007368CAF80C301B2A00F2A08008360AF129
:100E6000100356E021F0030BA34405F11000834565
:100E700059DA1EF0010F7FF425AF56F8081CC1EBBC
:100E8000080ADAF8041021F0030CE34458453FF750
:100E900057AF5746DAF80C1057F8080F221F242ACC
:100EA000C160886000F2B480132A40F2A5803168E6
:100EB000CAF808107168CAF80C101B2A00F2AF803B
:100EC00008360AF110023168116071685160B1682A
:100ED00091600AEB0501C5EB0B0242F0010299603B
:100EE0004A60DAF8043003F001031D434846CAF8AB
:100EF0000450FFF7B1FE38465CE73368036073685F
:100F000043601B2A27D800F1080306F10802F2E625
:100F10003B4632681A6072685A60B2689A603E4610
:100F20007446D04633E708EB0501C5EB0B0B4BF0DD
:100F3000010299604A6056F8043C03F001031D4326
:100F4000484646F8045CFFF787FE304632E73146F4
:100F5000FFF7CEFDD5E6B3688360F368C360242A4B
:100F600028D000F1100306F11002C4E650F8043C4A
:100F700023F003031C440AE7314638467446D04642
:100F8000FFF7B6FD3E4602E73A46F7E631463846F9
:100F90001C46D046FFF7ACFD3E46F8E6B368CAF8FB
:100FA0001030F368CAF81430242A1BD010360AF126
:100FB0001803AEE7336903617369436106F11802F0
:100FC00000F1180397E600BFB497FF1FB168CAF895
:100FD0001010F168CAF81410242A0FD010360AF144
:100FE0001802CBE63369CAF818307369CAF81C30A6
:100FF00018360AF120038CE73A4664E73269CAF8EA
:1010000018207269CAF81C2018360AF12002B5E6C9
:10101000314638460193FFF76BFD019B59E7B168F4
:10102000CAF81010F168CAF81410242A03D0103638
:101030000AF1180247E73269CAF818207269CAF83B
:101040001C2018360AF120023DE700BF38B5074CD6
:101050000023054608462360FBF7E0FE431C00D052
:1010600038BD2368002BFBD02B6038BDCCA3FF1FFD
:10107000FFFFFFFFFFFFFFFFFFFFFFFFFFFFFFFF80
:1010800090F800F06DE9024520F007016FF0000CC8
:1010900010F0070491F820F040F049804FF0000470
:1010A0006FF00700D1E9002391F840F000F108004B
:1010B00082FA4CF2A4FA8CF283FA4CF3A2FA8CF383
:1010C0004BBBD1E9022382FA4CF200F10800A4FAEA
:1010D0008CF283FA4CF3A2FA8CF3E3B9D1E904233E
:1010E00082FA4CF200F10800A4FA8CF283FA4CF375
:1010F000A2FA8CF37BB9D1E9062301F1200182FA2F
:101100004CF200F10800A4FA8CF283FA4CF3A2FA34
:101110008CF3002BC6D0002A04BF04301A4612BA42
:10112000B2FA82F2FDE8024500EBD2007047D1E945
:10113000002304F00305C4F100004FEAC50514F0D4
:10114000040F91F840F00CFA05F562EA05021CBFA5
:1011500063EA050362464FF00004A9E7002A41D084
:1011600040EA010313F00303F0B425D1032A23D985
:1011700004680D68AC421FD1043A35D0A4F10135A2
:1011800025EA040414F0803F31D1071D0D1D0DE048
:1011900057F8043B0E68A3F10134B34224EA030478
:1011A0000AD1043A20D014F0803F23D1032A2946E3
:1011B000384605F10405EBD803780C789C4202F11F
:1011C000FF320CD182B114B916E06AB17BB110F8CC
:1011D000013F11F8014FA34202F1FF32F5D0181B75
:1011E000F0BC7047104670471046F0BC7047184678
:1011F000F0BC70470020F3E72046F1E740EA010326
:101200009B0770B42BD1032A29D90C4603462146EB
:1012100054F8046BA6F1013525EA060515F0803F68
:1012200006D1043A032A43F8046B2146EFD8A2B151
:101230000C781C70013A013301313CB16AB111F8EC
:10124000014B03F8014B013A002CF7D12AB11A44A3
:10125000002103F8011B9A42FBD170BC7047034682
:10126000E5E700BF2DE9F047254C2568D5F8484152
:101270000646884692469946C4B360681F2817DC24
:10128000431C76B104EB80050122C5F888A0D4F890
:10129000881182401143022EC4F88811C5F80891C4
:1012A0001ED00230636044F820800020BDE8F08743
:1012B000144B03B34FF4C870FFF752F90446D0B192
:1012C000D5F84831002780E88800C5F848413846FD
:1012D0000123C4F88871C4F88C71002EE1D0D1E7E5
:1012E000D4F88C110A43C4F88C21DAE705F5A6740A
:1012F000C5F84841C1E74FF0FF30BDE8F08700BFB7
:10130000283D010061050100024B13B1024800F0C5
:1013100005B87047000000002913010000230146B2
:101320001A461846FFF79EBF38B5074D074C2C1BD1
:10133000A41005D0013C55F8043D9847002CF9D184
:10134000BDE8384002F002BD0000000000000000CF
:10135000F8B5234F0C460646FFF77CFCBB685D687A
:1013600025F00305291B01F6EF7121F47F6121F0BF
:101370000F01A1F58054B4F5805F07DB00213046F2
:10138000FFF764FEBB682B44984204D03046FFF759
:1013900063FC0020F8BD61423046FFF757FE013084
:1013A0000DD0104BBA6819682D1B45F00105304669
:1013B000091B55601960FFF74FFC0120F8BD0021A3
:1013C0003046FFF743FEBA68831A0F2BDEDD064C6A
:1013D0000449246843F00103001B53600860D5E70B
:1013E000B497FF1F70A2FF1FC09BFF1F002945D0AD
:1013F0002DE9F0410D468046FFF72CFC55F8047CA2
:101400006A4927F00103A5F10804E2188E685068C4
:10141000B24220F0030062D0FE0750600BD455F8B2
:10142000087CE41B01F1080EA56875453B446FD0AC
:10143000E768EF60BD6015186D68ED0742D543F0B1
:1014400001026260E350B3F5007F18D2DB085A1C3A
:101450004D6851F83270A76001209B1000FA03F329
:1014600001EBC2001D430838E0604D6041F8324096
:10147000FC604046BDE8F041FFF7EEBB70475A0AFA
:10148000042A53D89A0902F139077F0002F138057E
:1014900001EB870051F827204449083890424DD08D
:1014A000516821F003018B4202D292689042F7D139
:1014B000D068E060A2608460D4604046BDE8F0413E
:1014C000FFF7CABB95683A4FBD4203443FD0D0688E
:1014D000E86043F0010285606260E350B3E7FF0714
:1014E000034407D455F8082CA41A1344A068E268F2
:1014F000C26090602F4A126843F00100934260601E
:101500008C60B6D32C4B40461968FFF721FFB0E73B
:1015100011184968C90744D49168D268CA60034465
:1015200043F0010091606060E350A2E7142A17D8ED
:1015300002F15C077F0002F15B05A9E7AA104B6886
:10154000012505FA02F213434B600246B1E743F06E
:1015500001024C610C61E560A5606260E35088E7C0
:10156000542A06D81A0B02F16F077F0002F16E05AC
:101570008EE7B2F5AA7F06D8DA0B02F178077F0072
:1015800002F1770584E740F25450824206D89A0C63
:1015900002F17D077F0002F17C0579E7FE277E25B9
:1015A00076E743F001026260E35062E7B497FF1F01
:1015B000BC97FF1FBC9BFF1F6CA2FF1F000078059C
:1015C0003408540B800C3C0F5C12E015FA19141E01
:1015D0006022AC265C2B0C30BC34023AFF3FFFFF8C
:1015E000FDFFFFFFFBFFFFFFF8FFFFFFFDFFFFFF1A
:1015F000FBFFFFFFF8FFFFFFFDFFFFFFFAFFFFFF0D
:10160000F7FFFFFFFDFFFFFFFBFFFFFFF7FFFFFF00
:10161000FCFFFFFFFBFFFFFFF7FFFFFFFDFFFFFFEB
:10162000FAFFFFFFF7FFFFFFFDFFFFFFFBFFFFFFDD
:10163000F8FFFFFFFDFFFFFFFBFFFFFFF8FFFFFFCE
:10164000FDFFFFFFFAFFFFFFF7FFFFFFFCFFFFFFBC
:10165000FBFFFFFFF7FFFFFFFDFFFFFFFBFFFFFFAC
:10166000F7FFFFFFFDFFFFFFFAFFFFFFF7FFFFFFA1
:10167000FDFFFFFFFBFFFFFFF7FFFFFFFDFFFFFF8A
:10168000FBFFFFFFF7FFFFFFFDFFFFFFFAFFFFFF7D
:10169000F7FFFFFFFDFFFFFFFAFFFFFFF8FFFFFF70
:1016A000FDFFFFFFFAFFFFFFF7FFFFFFFDFFFFFF5B
:1016B000FAFFFFFFF7FFFFFFFDFFFFFFFAFFFFFF4E
:1016C000F8FFFFFFFDFFFFFFFAFFFFFFF8FFFFFF3F
:1016D000FDFFFFFFFAFFFFFFF7FFFFFFFCFFFFFF2C
:1016E000FBFFFFFFF7FFFFFFFDFFFFFFFAFFFFFF1D
:1016F000F7FFFFFFFDFFFFFFFAFFFFFFF7FFFFFF11
:10170000FEFFFFFFFBFFFFFFF8FFFFFFFEFFFFFFF6
:10171000FBFFFFFFF8FFFFFFFDFFFFFFFAFFFFFFEB
:10172000F7FFFFFFFCFFFFFFFAFFFFFFF7FFFFFFE1
:10173000FCFFFFFFFAFFFFFFF7FFFFFFFDFFFFFFCB
:10174000FAFFFFFFF7FFFFFFFDFFFFFFF9FFFFFFBE
:10175000F7FFFFFFFDFFFFFFF9FFFFFFF7FFFFFFB1
:10176000FDFFFFFFFAFFFFFFF7FFFFFFFDFFFFFF9A
:10177000FAFFFFFFF7FFFFFFFDFFFFFFFAFFFFFF8D
:10178000F6FFFFFFFDFFFFFFFAFFFFFFF7FFFFFF81
:10179000FEFFFFFFFBFFFFFFF7FFFFFFFEFFFFFF67
:1017A000FBFFFFFFF7FFFFFFFDFFFFFFFAFFFFFF5C
:1017B000F7FFFFFFFDFFFFFFFBFFFFFFF8FFFFFF4E
:1017C000FDFFFFFFFBFFFFFFF8FFFFFFFDFFFFFF38
:1017D000FAFFFFFFF7FFFFFFFCFFFFFFF9FFFFFF2F
:1017E000F7FFFFFFFCFFFFFFF9FFFFFFF7FFFFFF22
:1017F000FDFFFFFFFAFFFFFFF7FFFFFFFDFFFFFF0A
:10180000FAFFFFFFF7FFFFFFFDFFFFFFF9FFFFFFFD
:10181000F6FFFFFFFDFFFFFFFAFFFFFFF7FFFFFFF0
:10182000D01E0100AC1E0100881E0100641E0100D4
:10183000BC190100781801009C180100C0180100B3
:101840009819010054180100E01C0100BC150100AA
:10185000101B01000000580246056608540BD80E04
:101860005C127017FC21F82A70305834DC37663A65
:101870008C3C803EFF3FFFFF000058024605660893
:10188000540BD80E5C12E015FA19141E6022AC2617
:101890005C2B0C30BC34023AFF3FFFFF000090018C
:1018A00020031405D0075A0AAC0DCC10B4146A18E2
:1018B000E81C342180252A2B70301437FF3FFFFFAE
:1018C0000000C800F4018403140508072E091C0C4D
:1018D000D80EF811AE159619401F1C25F22B58345E
:1018E000FF3FFFFFFBFFFFFFF8FFFFFFF4FFFFFFDE
:1018F000FAFFFFFFF7FFFFFFF4FFFFFFFDFFFFFF12
:10190000F9FFFFFFF4FFFFFFFAFFFFFFF7FFFFFF05
:10191000F4FFFFFFFCFFFFFFF7FFFFFFF4FFFFFFF8
:10192000FBFFFFFFF8FFFFFFF4FFFFFFFDFFFFFFDF
:10193000FAFFFFFFF4FFFFFFFDFFFFFFF9FFFFFFCF
:10194000F4FFFFFFFDFFFFFFF8FFFFFFF4FFFFFFC6
:10195000FCFFFFFFF7FFFFFFF4FFFFFFFBFFFFFFB1
:10196000F8FFFFFFF4FFFFFFFCFFFFFFF7FFFFFFA4
:10197000F4FFFFFF40067805B004E803840320036A
:10198000BC025802F40190012C01FA00C800960034
:10199000640032001900FFFF00006400C8009001DD
:1019A000BC021A04DC059E07F609800CA00F241364
:1019B000A2174C1D5424442FFF3FFFFF0000FF03DC
:1019C000FF07FF0BFF0FFF13FF17FF1BFF1FFF2377
:1019D000FF27FF2BFF2FFF33FF37FF3BFF3FFFFFAB
:1019E00001020101000101010201010201010101E5
:1019F00001010201010201010201010100000102D5
:101A000001010201010101000102010102010100C5
:101A100002020102010102010002020201020101AF
:101A200002000102020201020101000000020202A2
:101A30000102010101000002020201020100020292
:101A4000020202020102000202010202020201027B
:101A5000000202020102020201010002020202026D
:101A60000202010000020200020202020002010260
:101A7000020202020202000200020202020202024A
:101A8000FBFFFFFFF7FFFFFFF4FFFFFFFBFFFFFF81
:101A9000F7FFFFFFF4FFFFFFFDFFFFFFF7FFFFFF73
:101AA000F4FFFFFFFDFFFFFFF8FFFFFFF4FFFFFF65
:101AB000FAFFFFFFF7FFFFFFF4FFFFFFFBFFFFFF52
:101AC000F7FFFFFFF4FFFFFFFBFFFFFFF7FFFFFF45
:101AD000F4FFFFFFFBFFFFFFF7FFFFFFF4FFFFFF38
:101AE000FDFFFFFFF8FFFFFFF4FFFFFFFDFFFFFF1C
:101AF000F8FFFFFFF4FFFFFFFDFFFFFFF8FFFFFF11
:101B0000F4FFFFFFFAFFFFFFF8FFFFFFF4FFFFFF07
:101B10000000D007800CD80E0010C012EC130C1778
:101B2000FA19141E6022AC265C2B0C30BC34023A2D
:101B3000FF3FFFFF00000000070000000C00000056
:101B40001000000013000000180000001C0000003E
:101B500000000000070000000C000000130000005F
:101B6000180000001F00000024000000000000001A
:101B70000C000000180000002400000030000000ED
:101B80003C0000004800000000000000FBFFFFFFD9
:101B9000F4FFFFFFEFFFFFFFE8FFFFFFE3FFFFFFA3
:101BA000DCFFFFFF00000000F4FFFFFFE8FFFFFF86
:101BB000DCFFFFFFD0FFFFFFC4FFFFFFB8FFFFFF09
:101BC000FBFFFFFFF8FFFFFFF4FFFFFFFAFFFFFF40
:101BD000F7FFFFFFF4FFFFFFFDFFFFFFF9FFFFFF30
:101BE000F4FFFFFFFAFFFFFFF7FFFFFFF4FFFFFF28
:101BF000FCFFFFFFF7FFFFFFF4FFFFFFFBFFFFFF0F
:101C0000F8FFFFFFF4FFFFFFFDFFFFFFFAFFFFFFFD
